:020000040800F2
:1000000000000120217E0508A57E0508C93F0208E1
:10001000A57E0508A57E0508A57E05080000000050
:10002000000000000000000000000000A57E0508A0
:10003000A57E050800000000A57E0508A54701086B
:10004000A57E0508A57E0508A57E0508A57E0508F0
:10005000A57E0508A57E05087F010108830101082A
:10006000870101088B0101088F010108E1B6000832
:10007000F5B6000809B700081DB7000831B7000839
:1000800045B7000859B70008A57E0508A57E0508F4
:10009000A57E0508A57E0508A57E05089301010833
:1000A00075BF000899BE000889BF000885BE00081A
:1000B000C1BE0008D5BE0008E9BE0008E5AC0008D6
:1000C000D9AC0008FDAC0008F1AC0008A57E05081D
:1000D000A57E050851C200085DC2000869C200087B
:1000E00097010108A57E0508A57E05089DBF0008AB
:1000F00025BF00084DBF000811BF00086DB70008FC
:10010000A57E0508A57E0508FDBE0008A57E05089C
:1001100075C2000881C20008A57E05086DD00008E0
:1001200081B7000895B70008A9B70008BDB7000857
:10013000D1B700080000000000000000000000002F
:1001400000000000000000000000000009C40008DA
:10015000E5B70008F9B700080DB800088DC200081F
:1001600015AD000809AD0008A57E0508A57E0508A7
:10017000A57E0508A57E050800000000000000001F
:10018000A57E0508A57E0508A57E0508A57E0508AF
:10019000A57E0508A57E050800000000A57E0508CF
:1001A000000000000000000000000000A57E05081F
:1001B000A57E0508A57E05080000000000000000DF
:1001C000000000000000000000000000000000002F
:1001D000000000000000000000000000A57E0508EF
:0801E0006C790500010000002C
:1001E800C87602200201000001001400E87602200F
:1001F800020700000100140008770220020800002E
:100208000100140028770220010C0000000076008D
:1002180048770220010D010000007700687702206E
:100228000112000000007600887702200114000007
:1002380000001E00A8770220011A000000000D002F
:10024800C87702200115000000000C00E8770220A2
:100258000116000000000C0008780220011B0000B5
:1002680000000E0028780220011C000000001E007B
:10027800487802200117000000000C00687802206E
:100288000118000000000E00887802200119000003
:1002980000000C00A8780220011E000000000C00DD
:1002A800C8780220011F000000000C00E878022036
:1002B8000128010000001800087902200120000030
:1002C80000004800287902200121000000004900B0
:1002D800487902200122000000004A0068790220C3
:1002E8000123000000004B0088790220012400004F
:1002F80000004C00A87902200125000000004D00F4
:10030800C87902200126000000004E00E87902208A
:100318000127000000004F00087A0220012B00008E
:1003280000002900287A0220012C01000000290081
:10033800487A0220012D010000007000687A02202E
:10034800012E010000005200887A0220012F0100CE
:1003580000002800A87A02200130010000002800CF
:10036800C87A02200229050000012C00E87A022040
:100378000231000000021F00087B02200133000048
:1003880000003C00287B022001360000000020000D
:10800000836B1A6C12F0500F21D11A6C42F400727B
:108010001A641A68916811F0405F1BD19969C9B957
:10802000D16A11F4700F02D09168490512D45168D9
:1080300021F0200151601A6C22F480721A641A6CCB
:10804000D20407D41A6C42F001021A6470479B6B89
:10805000DB6C184770477047836B40221A645A6C78
:1080600042F004025A64704790F83530022B03D076
:1080700080234365012070470268052380F835306E
:108080000020136823F00103136070470268436BFC
:108090009169126803B118477047836B19684A6881
:1080A00042F400424A600022996B0A65D96B0A6566
:1080B00093F84120602A02D1202283F841207047A2
:1080C000F0B5059D06680C4FB46931EA04040CBF95
:1080D00001240024944201D000200CE03C68641B81
:1080E0009C42F1D9202380F84130002380F84230AF
:1080F00080F840300320F0BDE826012030B5046848
:10810000039D60682B4320F07F700B4320F45930AF
:1081100043EA024320F47F7020F0030003436360CE
:1081200030BD836B0022A3F85A20A3F85220704779
:10813000436ADA0710B506D50168846A4A6822F4F2
:10814000003222434A609C0706D50168C46A4A6827
:1081500022F4803222434A60590706D50168046B35
:108160004A6822F4802222434A601A0706D5016831
:10817000446B4A6822F4004222434A60DC0606D57A
:108180000168846B8A6822F4805222438A609906CF
:1081900006D50168C46B8A6822F4005222438A60C3
:1081A0005A0610D50168046C4A68B4F5801F22F4A1
:1081B000801242EA04024A6005D14A68446C22F403
:1081C000C00222434A601B0606D50268816C5368D0
:1081D00023F400230B43536010BD0F4B984215D07E
:1081E000A3F57843984213D003F58063984211D0E9
:1081F00003F57843984208D10323084A142101FB70
:108200000322138A01339BB2138270470023F4E7E1
:108210000123F2E70223F0E70030014000000120D3
:10822000D0E907239A422FBFD01AC0688018C01A1D
:108230007047D0E9092300699A4238BF1218013803
:10824000D31AC01A7047D0E90902131A584258418C
:1082500070470246036A4169C85C0133D1688B42AA
:1082600028BF002313627047436A8269D154436A6E
:1082700002690133934228BF0023426B43621368B3
:1082800043F0800313607047436BD86910F010000F
:1082900002D0102201201A627047704770470120F7
:1082A0007047014B58687047E8260120034B93F84C
:1082B0000402C31E58425841704700BFE8260120FF
:1082C000012380F84930704708B5D0F814320BB953
:1082D000022008BD1B6898470028FAD0F8E7D0F8BC
:1082E00018321BB10020C3F81402704702207047F7
:1082F000D0F8302201F00F01D0F8183210B51C244C
:1083000004FB012203F50371B2F81022C3F80C221A
:10831000D0F81C22D3F80402D2689047002010BD88
:10832000D0F81C3210B56BB1D0F8184294F80002A6
:10833000FF2807D09B68214694F801229847FF2325
:1083400084F80032002010BD4323038000487047AA
:10835000500001204323038000487047940001200F
:108360004323038000487047D80001200A2303807C
:10837000004870471C0101202023038000487047FB
:108380002801012020230380004870474801012074
:108390002023038000487047680101200A230380DE
:1083A0000048704788010120042301480B80704772
:1083B00094010120002370B54D1C1E46040FB0F13E
:1083C000204F4FEA001034BF3034373401F81340E7
:1083D00005F813600133DCB2A242EFD870BD1A2356
:1083E00010B50B80094BD3F8100AD3F8182A80185F
:1083F0000AD0D3F8144A08220549FFF7DBFF04220C
:1084000010312046FFF7D6FF024810BD0070F01F64
:108410009A0101209801012000207047212808B509
:108420001CD022282CD0202816D1A9B1072A13D17C
:108430001A4B08790A6883F8B80148798979C3F832
:10844000B42183F8B90183F8BA11154BD3F83C3243
:1084500013B1114600209847002008BD0029FBD029
:10846000072AF9D10D4BD3F8B4210A6093F8B8214B
:108470000A7193F8B92193F8BA314A718B71EBE71D
:108480000029E9D0022AE7D1054BD3F84032002B6E
:10849000E2D0098800209847DEE700BF00000120F5
:1084A000E8260120064AD2E99132934203F1FF33D4
:1084B0008CBF002001209B1A03EB0030704700BFE7
:1084C000E8260120EEE74FF4007300201380024BF2
:1084D000D3F858320B607047E8260120002070471F
:1084E00001207047012070470020704730B41446C7
:1084F0001A69A24209D30D199B69AA4238BF111B00
:108500000A46E11830BC54F085BD30BC704738B520
:108510000025044680F8425090F84130292B0AD1BA
:108520002823012180F84130212303634EF088FB8A
:1085300084F8405038BD90F841302A2BFAD12823D6
:10854000022180F8413022230363EFE7154B2022FC
:1085500010B5C362002304460363436380F84120DF
:1085600080F842304B0711D503685A6A436A591C98
:1085700041621A70038D4BB1013B0385438D013B72
:108580009BB24385436C43F00403436407212046B8
:108590004EF056FB23681022DA61002384F8403045
:1085A00010BD00BF0000FFFF0022304B10B580F867
:1085B00042200446C3624285436C1943416490F8EB
:1085C0004130282B07D090F84130292B03D090F868
:1085D00041302A2B21D1032120464EF031FB2823A4
:1085E00084F8413000232363214B636323681968B7
:1085F0001A6811F480411DD022F48042A06B1A60E9
:108600001C4B0365002384F84030FFF72DFD58B361
:10861000A06B036DBDE81040184707214EF010FB1A
:1086200094F84130602B02D0202384F8413000239D
:108630002363DAE712F400420DD01A68E06B22F4EB
:1086400000421A600B4B036584F84010FFF70CFDE5
:1086500050B1E06BDDE794F84130602B02D120236C
:1086600084F8413084F8402010BD00BF0000FFFFB7
:1086700099A100089B800008036899691A6810B4E2
:10868000CC0508D5140606D5446C44F001044464B6
:108690004FF48074DC614C0508D5140606D5446C93
:1086A00044F0080444644FF48064DC61890508D513
:1086B000120606D5426C42F0020242644FF4007288
:1086C000DA61436C13F00B0F03D0416C5DF8044B7F
:1086D0006AE75DF8044B704703682DE9F04F13F02B
:1086E000010885B000F0C881AC4A916821F400010E
:1086F0009160C16A94680C43B1FA81F149099460B0
:1087000013F4002600F0BA81A44D426BD5F88C40DA
:10871000B2F5801F24F4401444EA0204C5F88C40EA
:1087200000F0AE81B2FA82F2520913F4801401947F
:1087300011D0DFF868C2856BDCF88C40B5F5800F8E
:1087400024F4400444EA0504CCF88C4000F09B81FA
:10875000002D08BF01229F0638D5904CDFF844C297
:10876000256C45F080552564246C04F080540394F6
:10877000039C8B4C256845F480752560DCF800E08F
:108780002568ED0540F18181844C856AD4F870E05C
:1087900005F440791EF4407E40F08281B9F5407FB7
:1087A0007E4C40F0A981D4F808C025F0704E2CF41E
:1087B000F81C2EF4407E4CEA0E0CC4F808C0C5F339
:1087C0000B05D4F870C045EA0C052567DC060CD50E
:1087D000724DD5F88C4024F08074C5F88C40D5F8E3
:1087E0008C40076B3C43C5F88C405F0409D5DFF82B
:1087F000ACC1C46DDCF8905025F440352C43CCF866
:1088000090401D0409D5DFF894C1046EDCF8905047
:1088100025F440252C43CCF89040DC0309D5DFF843
:108820007CC1446EDCF8905025F440152C43CCF804
:1088300090405F0609D5DFF864C1C46BDCF8905046
:1088400025F003052C43CCF890401D0609D5DFF830
:108850004CC1046CDCF8905025F00C052C43CCF88E
:108860009040DC0509D5DFF834C1446CDCF8905049
:1088700025F030052C43CCF890409F0509D5DFF852
:108880001CC1846CDCF8905025F0C0052C43CCF85A
:1088900090405D0509D5DFF804C1C46CDCF8905048
:1088A00025F440752C43CCF890401C0509D5DFF821
:1088B000ECC0046DDCF8905025F440652C43CCF8F6
:1088C0009040DF0409D5DFF8D4C0446DDCF8905047
:1088D00025F440552C43CCF890409D0409D5DFF891
:1088E000BCC0846DDCF8905025F440452C43CCF896
:1088F000904013F400150FD0DFF8A0E0D0F874C05A
:10890000DEF89040BCF1006F24F0006408BF012243
:1089100044EA0C04CEF890405C030AD5DFF87CE012
:10892000DEF8904024F0407CC46E4CEA0404CEF89B
:1089300090401F020AD5DFF864E0DEF8904024F092
:10894000805C846F4CEA0404CEF890405C0140F1F6
:10895000D880DFF848E0DEF8904024F0005CC46F77
:108960004CEA0404CEF89040002940F0CF80012A60
:1089700040F08080094B0B491A6822F080521A603F
:108980000C681A68970000F178810EB1426B5AB1F9
:10899000019A002A38D0826BB2BB05E00038024051
:1089A00000700040E8260120D3F888404FF440369C
:1089B00096FAA6FE47F6C072BEFA8EFE92FAA2F2B0
:1089C000B2FA82F796FAA6F64FF0706CB6FA86F60F
:1089D0009CFAACFC0269BCFA8CFC04F44034BA404A
:1089E000476924FA0EF407FA0CF7B4403A432243DD
:1089F000C3F88820D3F88C20046A22F4F852013C92
:108A000042EA0422C3F88C2055B3436FB3F1006FE0
:108A100026D1A04D4FF0706CD5F888209CFAACF7A9
:108A200047F6C073B7FA87F793FAA3F34FF44034CD
:108A3000B3FA83F694FAA4F4B4FA84F49CFAACFC86
:108A4000036902F070628069BCFA8CFCB340FA40A2
:108A500000FA04F402FA0CF223431343C5F88830F9
:108A60008C4B1A6842F080521A6008681A689200AB
:108A700040F10981002010E0414641E6324654E6CB
:108A80000022012151E6012165E6DCF80050A5EB4A
:108A90000E05642D7FF674AE032005B0BDE8F08F9F
:108AA000F1453FF47BAED4F870E0D4F870A02EF41A
:108AB000407E4AF4803AC4F870A0D4F870A02AF43A
:108AC000803AC4F870A0C4F870E0D4F870E01EF0EA
:108AD000010F3FF463AEDCF800A041F2883BD4F80C
:108AE00070E01EF0020F7FF459AEDCF800E0AEEB50
:108AF0000A0EDE45F3D9CFE7D4F808C02CF4F81CF1
:108B00005BE619B9B3F1007F7FF431AFDFF884E1A0
:108B1000DFF884C1DEF8001021F08061CEF800108B
:108B2000DCF80040DEF800100F0100F19F80B8F182
:108B3000000F2AD0C16A41BBDEF884404FF0706854
:108B400098FAA8F947F6C07BB9FA89F99BFAABFB0A
:108B5000BBFA8BFB98FAA8F84FF0E04AB8FA88F80D
:108B60009AFAAAFA4168BAFA8AFA04F0706401FA29
:108B70000BFB816824FA09F401FA0AF104FA08F4FB
:108B80004BEA01012143CEF884101EB1416BB1F5CF
:108B9000801F05D00199B9B3816BB1F5800F33D136
:108BA000DFF8F0E04FF0E048DEF8844098FAA8F9EA
:108BB00047F6C07BB9FA89F99BFAABFB4FF0706AB4
:108BC000BBFA8BFB9AFAAAFABAFA8AFA98FAA8F8C8
:108BD000416804F0E044B8FA88F801FA0BFBC16878
:108BE00024FA09F401FA0AF104FA08F44BEA010143
:108BF0002143CEF88410DEF88C40C16924F01F04B4
:108C000001392143CEF88C109C011ED547F6C07364
:108C100093FAA3F34FF07061B3FA83F491FAA1F1E0
:108C20004FF0E04EB1FA81F19EFAAEFE4368BEFA13
:108C30008EFEA340C46804FA01F10B43816801FA77
:108C40000EF10B431349C1F88430124B196841F0FF
:108C500080611960DCF80040196809013FF587AEB2
:108C6000DCF80010091B6429F6D915E7DCF80010C0
:108C7000091B64297FF656AF0EE70A68121B642AA7
:108C80007FF67FAE08E70A68121A642A7FF6EEAE16
:108C900002E700BF00380240E82601202DE9F34733
:108CA00006690546C3680C464FF0004901F15007BC
:108CB0001E4001F1380816B902B0BDE8F087B6FAD7
:108CC00086F329FA03F21B3BD24316402A61002C9B
:108CD00042D0042BEFD8DFE803F03B363029030005
:108CE0002369D5F82CA033B19B6823B11FFA8AF110
:108CF00004F108009847A36A33B19B6823B11FFAB7
:108D00008AF104F120009847236C2BB19B681BB1BA
:108D10001FFA8AF140469847A36D002BCBD09B6881
:108D2000002BC8D01FFA8AF1384604E0236904F109
:108D30000800696B5B689847BDE7A36A04F12000EF
:108D4000A96B5B68F7E7236C4046E96B5B68F2E769
:108D5000A36D296C5B68E7E7042B06D8DFE803F016
:108D60000D0B09070300EB6A0193019BA3E76B6BF3
:108D7000FAE7AB6BF8E7EB6BF6E72B6CF4E737B58C
:108D8000224B0025224C234AC4F8883242F20F734A
:108D900004F52270C4F89852C4F894321E4BC4F8FB
:108DA0009052D3F8BC31B3FBF2F3013BC4F88C32E0
:108DB0004DF0B6FE194B062137201A6C42F0200206
:108DC0001A641B6C03F020030193019B4AF0F6F92F
:108DD000134B4FF4000228465A60D4F88832DA6800
:108DE00042F00102DA601A6842F001021A60D4F817
:108DF00020320C4AC3F81052C3F808220A4AC4E9C8
:108E00008F55C3F8042203B030BD00BF00140040EA
:108E1000E826012080841E00000001200038024066
:108E200000E100E0B4670120B457012010B5012033
:108E30000C4609F0D1FF054B122103F114022180E9
:108E400002280CBF1846104610BD00BFC00101200B
:108E5000436BDA69910670B5044613D5586AE36A24
:108E6000C0B2002B4AD0216B9847636B1A6822F47A
:108E700080721A609A6822F001029A609A6942F040
:108E800008029A61636BDA69D20701D501221A627E
:108E9000DA69960701D502221A62DA69550701D507
:108EA00004221A62DA69100701D508221A62DA6907
:108EB00011060ED594F89D20212A0AD0D4E9091272
:108EC0008A4227D10022A4F886201A6822F0800264
:108ED0001A60DA69520640F19380DA6904F13400CD
:108EE000196816079D6821D1960640F18A808D0683
:108EF00040F18780BDE870404DF0AEBDE369626926
:108F0000D054E369E2680133B3FBF2F102FB1133A1
:108F1000E361AAE7A169895C0132C9B2996221695A
:108F2000B2FBF1F001FB1022A262D2E705F00105CD
:108F300001F490762E4364D0D60709D5CE0507D527
:108F400001261E62D4F8A06046F00106C4F8A060B5
:108F5000960708D53DB102261E62D4F8A06046F0FF
:108F60000406C4F8A060560708D53DB104261E6269
:108F7000D4F8A06046F00206C4F8A06016070AD52F
:108F800001F02006354306D008251D62D4F8A03034
:108F90002B43C4F8A030D4F8A030002B30D0960674
:108FA00003D58D0601D54DF057FDD4F8A020636B95
:108FB000110703D49A6812F040021FD01A6822F4F5
:108FC00090721A609A6822F001029A60202284F856
:108FD0009E209A68520613D59A68D4F8980022F019
:108FE00040029A6060B1254B0365FFF73DF838B148
:108FF000D4F89800BDE87040036D1847C4F8A0206D
:1090000070BD16062ED50D062CD594F89D20212A6C
:10901000F6D1B4F8862092B242B91A6822F08002E2
:109020001A601A6842F040021A60E9E7E16BD4F86E
:109030008020B1F5805F0FD1616C69B932F8021BF5
:10904000C1F308019962C4F88020B4F88630013B6E
:109050009BB2A4F88630D3E7511CC4F88010127874
:109060009A62F2E75006CBD54A06C9D51A6822F0B3
:1090700040021A60202384F89D30C1E72381000854
:1090800070B500260E4CD4F8C8329BB9FEE712F832
:10909000016B013B4FF00105C4F8C822636007D1A2
:1090A0004AF04CFA6368D4F8C8222BB1002DEED0F8
:1090B000304670BD0025F5E7002DE3D0F8E700BF8E
:1090C000E826012008B5054A0B68C2F8C8025360BB
:1090D0000BB94AF033FA002008BD00BFE826012092
:1090E00090F84820531C0244DBB280F8483082F8E4
:1090F000341090F849200AB1132B01D94DF09EBBD2
:109100007047002280F849204DF098BBF8B504461E
:10911000D0F83002237C93BB4FF4007302228121EC
:109120004DF022FB4FF4007302220121D4F83002EB
:109130004DF01AFB082303228221D4F830024DF0AF
:1091400013FB4FF4077056F0FDF80546C4F81802FB
:1091500030B3D4F81C3200271B689847267CC5F82A
:109160001472C5F818728EB94FF40073D5F8042242
:109170000121D4F830024DF073FA3046F8BD402397
:10918000022281214DF0F0FA4023CDE74023D5F8AB
:1091900004220121D4F830023E464DF061FAECE79A
:1091A0000126EAE710B504468121D0F830024DF0DF
:1091B00098FA0121D4F830024DF093FA8221D4F8C4
:1091C00030024DF08EFAD4F8183253B1D4F81C3274
:1091D0005B689847D4F8180256F0BCF80023C4F82E
:1091E0001832002010BD10B504460121D0F830021D
:1091F0004DF077FA8121D4F830024DF072FAD4F8AC
:10920000280256F0A7F80020C4F8280210BD37B590
:109210000B7804460D4613F060022BD0202A21D192
:10922000CA8848780AB31B06D4F818120AD5D4F8AD
:109230001C3201919B689847EA88019920464DF0BD
:10924000F2FA0FE0032381F8012281F80002C4F84A
:10925000F4311346D4F83002C4E942220A46002110
:109260004DF0FEF9002003B030BDD4F81C329B68ED
:109270009847F7E74B780A2BF4D101220049DEE743
:10928000B429012070B50446D0F83002237C93BB8A
:109290004FF40073022201214DF066FA4FF400737F
:1092A00002228121D4F830024DF05EFA4FF41B7097
:1092B00056F048F80646C4F8280218B30025D4F83A
:1092C0002C320581A0F85C5228461B689847012182
:1092D000D4F830024DF05EFB8121D4F830024DF01D
:1092E00059FBD4F830021F2306F5037201214DF01B
:1092F000B7F9284670BD4023022201214DF034FA0F
:109300004023CDE70120F5E770B5D0F82852044698
:1093100095F818324BB9D5F8143233B16B7A23B9BA
:109320000121D0F830024DF0E8FA8121D4F8300262
:109330004DF0E3FA6B7A022B09D105F50372D4F8EC
:1093400030021F230121BDE870404DF089B970BD86
:1093500070B50E4B0446D0F82852C5F82C320023C5
:1093600085F8381205F50B722B7281210D23D0F888
:1093700030024DF097F905F50372D4F830021F233F
:109380000121BDE870404DF06BB900BF5553425309
:109390002DE9F0410B7804460D46D0F8287213F001
:1093A000600634D0202E7DD14A78FE2A05D0FF2ACF
:1093B00017D0022649F01EFE26E04E887EB9CD88E1
:1093C000012D0CD11A060AD5D0F82C329B6998478A
:1093D0002A463860394620464DF025FA14E02046EA
:1093E000E7E74A88002AFAD1CE88002EF7D11B067B
:1093F000F5D44FF4807307F5037201213B811F23DD
:10940000D0F830024DF02CF93046BDE8F08191F8EB
:109410000180B8F10A0F2AD0B8F10B0F2AD0B8F1A9
:10942000010FF1D10979D0F830024DF0B3FAD4F838
:10943000300229794DF055F995F90430D4F830020D
:10944000002B237C1BDAC3B94FF400730222812165
:109450004DF08AF9D4F828727B7A022B17D181213A
:10946000D4F830024DF049FA00237B72CCE7012298
:10947000391DB1E78B787B60C6E74023E6E723B967
:109480004FF4007302224146E2E74023FAE795F9E0
:109490000420002AB8DA012BB6D001212046FFF7BC
:1094A00057FFB1E70026AFE72DE9F74313780646EB
:1094B0000D4617462F2BD0F828423DD8192B08D837
:1094C000032B6BD0122B00F09380002B4BD020226B
:1094D00007E21A3B152BFAD801A252F823F000BF7D
:1094E0002F96000829960008CF940008CF94000812
:1094F00029960008CF940008CF940008CF94000864
:10950000CF94000859960008CF940008AB96000845
:10951000CF940008CF940008E5960008CF94000887
:10952000BF970008CF940008CF940008CF9400089C
:10953000CF940008D99800085A2BC8D10823B74AFD
:109540006381D2F80F30E360D2F813302361D0F892
:109550002C320846DB689847002847D0E37B63F04D
:109560007F03E37342E0D4F81432002BAFD1D0F87C
:109570002C3208469B689847054650B13A22022192
:10958000D6F828024AF09FF9052323724FF0FF35E1
:1095900000E06081284603B0BDE8F083122200217C
:1095A00004F10C0055F0DEFE702394F85D22237365
:1095B0000C23E37494F85C329A4211D004EBC3029A
:1095C000013392F83C12DBB2A173042B92F84112E2
:1095D00008BF0023217692F8402284F85C3262763C
:1095E000122363813B79122B98BF63810025D1E759
:1095F0005378DB0715D4D0F82C3201EBC105127972
:10960000DB6903EB85052B790533934228BF1346AD
:109610006381002BEAD0013B9BB2E95CE218117335
:10962000F7E707237D4DF3E700206081DEE708239D
:109630007A4A6381D2F80730E360D2F80B302361B5
:10964000D0F82C320846DB6898470028CED0A37BA0
:1096500063F07F03A373C9E700230DF1020201A9A0
:10966000E36023616361D0F82C3228465B68984739
:10967000054630B13A220221D6F828024AF023F9F1
:1096800084E70823E373019B013B1A0EE374227401
:109690001A0C62741A0ABDF80230A27402225BBA74
:1096A000A282E3820C23638174E7D0F82C3204F2A7
:1096B0005E22284604F518715B6898470546002825
:1096C000D8D1D4F860322082013B1A0EE3732273A2
:1096D0001A0C62731A0AB4F85E32A2735BBA638220
:1096E0000823E0E7237A6BBB94F91832002BBFF60E
:1096F000EEAED0F82C3208469B6898470028B9D1C6
:10970000D7F80220D6F8280212BAD0F86012C4F8AE
:109710006422B7F807305BBA9BB29F18C4F868326E
:109720008F4277D802212172B4F85E124A434B432C
:10973000C4F86422D4F81422C4F86832934201D0E9
:10974000202268E04FF40073D6F82C026381D6F82B
:109750002842D0F810902846D4F8687204F10C081A
:10976000B4F85E229F42D4F8641228BF1F46B7FBAC
:10977000F2F3B1FBF2F29BB24146C847002802DA8D
:109780001122042178E7BBB2D6F83002424681218B
:109790004CF088FFD4F86432D4F868023B44C51B0F
:1097A000C4F86432D4F83432C4F86852DB1BC4F80D
:1097B0003432002D7FF41AAF03232372EAE6237AB2
:1097C000002B49D194F91832002BFFF680AED0F867
:1097D0002C3208469B68984700287FF44BAFD6F898
:1097E0002C322846DB689847054608B1272242E715
:1097F000D7F80220D6F8280212BAD0F86012C4F8BE
:109800006422B7F807305BBA9BB2D718C4F8683245
:109810008F4205D92122052130E700BF1804060830
:10982000B4F85E124A434B43C4F86422D4F81422BD
:10983000C4F86832934283D1B3F5007F4FF0010141
:1098400004F10C0228BF4FF400732172D6F83002E5
:109850009BB24CF005FF9DE6D4F8687204F10C0849
:10986000B4F85E22B7F5007FD4F86412D0F82C0269
:1098700028BF4FF40077D0F814902846B7FBF2F3D6
:10988000B1FBF2F29BB24146C847002801DA03223D
:1098900077E7D4F86432D4F868523B44ED1BC4F83F
:1098A0006432D4F83432C4F86852DB1BC4F8343262
:1098B00025B929463046FFF74BFD6BE6B5F5007F2D
:1098C00042464FF00101D6F8300228BF4FF4007530
:1098D000ABB24CF0C5FE89E6787810F0020003D0F8
:1098E000242205212046C9E6D4F86422B4F868325F
:1098F0001344D4F8602293427FF697AE2122F0E71A
:10990000D0F8281210B50B7A0446022B07D0033B7F
:10991000012B02D80021FFF71BFD002010BD01F232
:109920001B2291F81912FFF7BFFD0028F5DA01217B
:109930002046F0E770B5D0F828420546267A1EB1D9
:10994000012E55D0002070BDD4F81032C4F830324A
:10995000D4F81432C4F83432D0F83032B3F82C32A0
:109960001F2B0DD1D4F80C22264B9A4208D194F823
:109970001912012904D894F81A32013B0F2B0AD985
:1099800020220521204649F09EFF022363722846CB
:10999000FFF7BAFCD6E704F21B22FFF785FD00288B
:1099A000237A06DA052BF2D101212846FFF7D0FCF5
:1099B000C8E7013B022BC5D961890029F5D0D5F84C
:1099C0002832D3F8142283F83862914228BF114616
:1099D000D3F83422521AC3F8342204221A728BB2FA
:1099E00004F10C028121D5F830024CF05BFEA9E7AE
:1099F00004F21B2294F81912FFF756FD0028A1DA91
:109A0000D2E700BF5553424308B520B9034849F097
:109A1000C1F9034808BD0348F9E700BF39B006089B
:109A2000B82901205AB00608024808B549F0B2F931
:109A3000014808BD7BB00608B8290120024808B5D6
:109A400049F0A8F9014808BD80B00608B8290120EE
:109A5000024808B549F09EF9014808BD8BB00608D8
:109A6000B8290120002008B549F05CFA002008BDA3
:109A70002DE9F843089D0E46174600212022044692
:109A8000984655F06FFC4DB12B681A0CE3816B685A
:109A90002282E3821A0C6B892283638230464DF066
:109AA000B1F9FB0604D400F1FF39B9F1FF3F42D10F
:109AB000082802464FF0FF394FF00005A8BF0822E2
:109AC0004FF02033314620462360636053F0A2FA02
:109AD00004F10803214A09F10101184622813144A9
:109AE000A2722A4653F096FA621E0346E01D12F84F
:109AF000011FA1F16105192D9CBF2039117082420F
:109B0000F5D1184604F10B0210F8013BA3F16101F5
:109B100019299CBF203B00F8013C9042F4D1182346
:109B2000E772A4F81A8023734FEA1843A382099BB3
:109B3000E361BDE8F88316F809302E2B02D009F155
:109B4000FF39B2E74A46A0EB0905082A05F1FF35BF
:109B5000A8BF0822032DA8BF0325B1E720202000BD
:109B60002DE9F04F0D46B94F85B00120043516465A
:109B7000994649F0D7F92C1FB9F1000F06D1484694
:109B800049F0D0F9484605B0BDE8F08FD7F870220B
:109B9000B24200F2B780A6EB0208D7F880A24FEAE3
:109BA000D803DAF8302008F007080233934203D3D1
:109BB000DAF83820934218D951461846039349F0F1
:109BC0007DF8039B824670B9A5F1080305F5FC7288
:109BD0009F4943F8041F9342FAD109F1FF39013636
:109BE00005F50075C7E7C7F880029AF80420002A37
:109BF0006DD04FF400720021204655F0B3FBDAF827
:109C00004030B8F1000F47D105F11C0BCDE90088B9
:109C100043BB434620460822D7F85C12FFF728FFD3
:109C20005C464FF4F073DAF8448004EB030AB8F1B1
:109C3000000FD2D05445D0D098F8042004F1200B66
:109C4000D8F8001008F11C00D8F83030B2B3002268
:109C5000CDE90002112220465C46FFF709FFD8F843
:109C60004880E4E7DAF83030112220467949FFF7DE
:109C7000FFFEDAF8403005F13C041A6CCDE90088AB
:109C800042B94346112274495846FFF7F1FE4FF49A
:109C9000E073C8E71B6BF5E7002B0CBF0122022223
:109CA000C2EB0812DAF84480B8F1000F03D0013A91
:109CB000D8F84880F8D14FF40073B6E798F805C09B
:109CC000D8F81020CDE900024CF02102C3E7DAF801
:109CD00028B0BBF1000F06D14FF4007200212046DE
:109CE00055F040FB79E7DAF830204FF40071204658
:109CF0009B1ADAF80C2008EBC308534602EB482203
:109D0000D8476AE7002E64D14FF4007231462046EE
:109D100055F028FB8023514985F8BA310C2385F88A
:109D2000BE31D7F86022D7F858328A42C4F8C6212B
:109D3000C4F8CA3118DDFF2285F8BB2185F8BD21A2
:109D400085F8BC21013B454A934228DDFF2385F875
:109D5000BF3185F8C13185F8C031552385F8FA3116
:109D6000AA2385F8FB3138E73F2143F6C16492FB13
:109D7000F1F192FBF4F4C1EB811C85F8BD41A01018
:109D8000A2EB0C0220F03F000132024385F8BC2117
:109D9000FF2291FBF2F2114485F8BB11D2E73F227A
:109DA00043F6C16093FBF2F293FBF0F0C2EB821436
:109DB00085F8C10181101B1B21F03F0101330B43CA
:109DC00085F8C031FF2392FBF3F31A4485F8BF21D5
:109DD000C3E7D7F864329E4242D152234FF00008C5
:109DE000412272212370284663706123E270A370C0
:109DF00084F8E731D7F8783284F8E411C4F8E83110
:109E00004FF0FF3384F8E511414684F8E6214FF422
:109E1000F07284F8EC3184F8ED3184F8EE3184F896
:109E2000EF3155F09FFA5523C5F8EC81C5F8F08164
:109E3000C5F8F48184F8FE316FF0550384F8FC8195
:109E400084F8FD8184F8FF31C7E600BFE8260120D1
:109E5000DEADBEEF14E5060813E50608FF03FB00C0
:109E6000D7F860329E426BD14FF400720021204639
:109E700055F078FAEB233A4A4FF0080C05F8043C09
:109E80005823F82105F8033C902305F8023C136899
:109E900045F8013C53680222C5F8033000232273C1
:109EA000E37285F809C0A273E37369743F212A73D2
:109EB00021764FF0FF31D7F86002A1763E2184F879
:109EC0002C2001222177D7F858126376091AE376FD
:109ED00063772162A377E37784F82D3084F82E30FE
:109EE00084F82F30D7E99A01091A616284F830208A
:109EF00084F83130802385F842C085F83C3029232E
:109F000085F83E30942385F83F300E2385F84030A5
:109F10000D2385F84130134B1A68C5F843205A6861
:109F2000C5F847201A899B7AA5F84B200E4A85F878
:109F30004D301368C5F84E305368C5F852300CE701
:109F4000D7E99A138E4206D39E4207D2711A204651
:109F500048F0D8FE41E69E42FFF4BEAEF11AF6E7A5
:109F600099B00608A2B00608AEB0060813460A4625
:109F70000146184633F056B882B0054A0190106881
:109F8000136801991B1A8B42FAD302B0704700BFC5
:109F9000E8260120002808DB4209012300F01F0009
:109FA00003FA00F0014B43F82200704700E100E0A3
:109FB0002DE9F04F002385B0DFF8B8816B4ADFF858
:109FC000B89101270C689F4007EA040537EA0404AA
:109FD00040F0B6804C6824F0100ABAF1020F16D196
:109FE0004FEAD30E03F0070B4FF00F0C00EB8E0E71
:109FF0004FEA8B0BDEF820600CFA0BFC26EA0C0C07
:10A000000E6906FA0BF646EA0C06CEF820604FEA17
:10A01000430E4FF0030CD0F800B00AF1FF3A0CFAEF
:10A020000EFCBAF1010F6FEA0C062BEA0C0B04F0E0
:10A03000030C01960CFA0EFC4CEA0B0CC0F800C0A5
:10A0400015D8D0F808C006EA0C0CCE6806FA0EFA4D
:10A050004AEA0C0CC0F808C0D0F804C02CEA070784
:10A06000C4F3001C0CFA03FC4CEA07074760C768FE
:10A07000019E37408E6806FA0EF63E43C660E60043
:10A080005ED5D8F8446023F0030703F0030C4FF0CB
:10A090000F0E46F4804607F180474FEA8C0CC8F853
:10A0A000446007F59C37D8F8446006F48046039670
:10A0B000039E0EFA0CF6D7F808A02AEA060E2C4EDC
:10A0C000B04244D006F58066B04242D006F58066C4
:10A0D000B04240D006F58066B0423ED006F58066BC
:10A0E000B0423CD048453CD006F50066B0423AD07C
:10A0F00006F58066B0420CBF0726082606FA0CF665
:10A1000014F4803F46EA0E06BE606FEA0507166843
:10A110000CBF3E402E4314F4003F166056680CBF3F
:10A120003E402E4314F4801F566096680CBF3E409C
:10A130002E43A4029660D66854BF3E402E43D6609C
:10A140000133102B7FF43DAF05B0BDE8F08F002642
:10A15000D4E70126D2E70226D0E70326CEE704267D
:10A16000CCE70526CAE70626C8E700BF003C014049
:10A1700000000240003802400014024003689A695F
:10A18000910701D500229A629A69D20703D49A698D
:10A1900042F001029A61704770B590F84030044671
:10A1A0000D461646012B00F01881012380F840303F
:10A1B000CB0640F19780D00640F19480638D9BB22E
:10A1C000002B40F08780E36AB3F1007F03D0E36A9D
:10A1D000B3F1007F6AD194F84130282B66D129462B
:10A1E0002046FEF7B3F9AB065CD5B6065AD5236810
:10A1F000202207212046DA610822DA614CF020FD96
:10A20000236820465A6842F400425A605A6822F095
:10A21000FF7222F48B3222F4FF7222F001025A60A4
:10A22000FFF7ACFF22681368580402D413681904BE
:10A2300009D594F84130212B0CBFA36BE36B1B684D
:10A240005B689BB26385638D9BB21BB1636C43F00B
:10A25000040363646B0710D5636A526A591C616218
:10A260001A70238D4BB1013B2385638D013B9BB25B
:10A270006385636C43F004036364002323636363B7
:10A2800084F84230636C002B00F09A80616C2046A9
:10A29000FEF78AF994F84130282B03D1294620464D
:10A2A000FEF754F9002084F8400070BDE26A23688C
:10A2B00012F5803F0BD094F84120292A07D11022B3
:10A2C0002046DA61FFF75AFFFEF721F98BE71022EB
:10A2D000DA6188E723681022DA61636C43F00403D3
:10A2E000636480E769071DD572071BD5638D9BB238
:10A2F00063B123685A6A636A591C61621A70238DBC
:10A30000013B2385638D013B9BB26385638D9BB2CB
:10A31000002B7FF468AFE36A13F5803F3FF463AF2F
:10A320002046D1E72B072CD530072AD594F84130A9
:10A33000226803F02803282B20D193699169936840
:10A34000D068E068022813D1C3F3C21383EA114333
:10A3500013F006030CD1A16C0131A164A16C022998
:10A360007FF441AF0821A364D16184F840303AE71B
:10A37000042120464CF064FC0023F6E70823D36157
:10A38000FAE7A9077FF52FAFB2077FF52CAF638DF2
:10A390009BB26BB1636A5A1C626222681B7893623B
:10A3A000638D013B9BB26385238D013B23851AE7B7
:10A3B000E36AB3F1807FB3D0E36A002BB0D012E739
:10A3C000E36A13F5803F05D0054BE362202384F850
:10A3D000413067E794F84130F8E7022065E700BFB5
:10A3E0000000FFFF194B9A6802F00C02042A28D0E3
:10A3F000082A28D15A68596802F03F02586811F4B7
:10A40000800F47F6C07191FAA1F3B3FA83F300EA23
:10A41000010020FA03F014BF0D4B0E4BB3FBF2F218
:10A420000A4B50434FF440325B6892FAA2F2B2FA00
:10A4300082F203F44033D34001335B00B0FBF3F00E
:10A440007047034870470348704700BF0038024018
:10A4500000127A000024F400094B4FF4E0529B688C
:10A4600092FAA2F2B2FA82F203F4E053D340054A20
:10A470001344054ADB7DD2F8BC01D840704700BFC9
:10A48000003802401804060800000120094B4FF470
:10A4900060429B6892FAA2F2B2FA82F203F460433D
:10A4A000D340054A1344054ADB7DD2F8BC01D840AD
:10A4B000704700BF00380240180406080000012061
:10A4C00038B5C26904460368816800691D680143A4
:10A4D00060690143A04811432840256A0143E068B0
:10A4E0001960596821F4405101435960A169986885
:10A4F000294320F430600143996098498B421ED172
:10A5000001F59431D1F8901001F0030101390229CD
:10A5100000F2038192480144C97FB2F5004F40F038
:10A52000AE80082900F2A880DFE811F0E500FA000B
:10A530000001A6000C01A600A600A600350089496E
:10A540008B420AD101F5FA31D1F89000844900F02C
:10A550000C00014491F82210DFE783498B421FD1A0
:10A5600001F5F831D1F8901001F03001202900F008
:10A57000DA800AD8002900F0BB80102900F0DF80C3
:10A58000B2F5004F78D00120C6E03029F8D1B2F5FD
:10A59000004F40F0A8806268530803F58033CBE099
:10A5A00072498B4210D101F5F631D1F8901001F0CB
:10A5B000C001802900F0B78004D8002900F09880FD
:10A5C0004029DBE7C029E1E769498B4213D101F556
:10A5D000F431D1F8901001F44071B1F5007F00F032
:10A5E000A28005D8002900F08380B1F5807FC5E7FF
:10A5F000B1F5407FCAE75F498B4213D101F5923133
:10A60000D1F8901001F44061B1F5006F00F08B803B
:10A6100005D8002900F08180B1F5806FAEE7B1F573
:10A62000406FB3E754498B4211D101F5E031D1F8C5
:10A63000901001F44051B1F5005F74D004D80029A6
:10A6400056D0B1F5805F99E7B1F5405F9EE74B4981
:10A650008B4295D101F5DE31D1F8901001F44041E3
:10A66000B1F5004F5FD004D8002941D0B1F5804F3B
:10A6700084E7B1F5404F89E70120002345E0082930
:10A6800081D801A252F821F0ADA60008C5A60008A5
:10A69000CBA6000887A50008E1A6000887A500084A
:10A6A00087A5000887A50008E7A60008FFF7D4FEE5
:10A6B000D4E9002300EB5300B0FBF3F080B2D0608C
:10A6C000002029E0FFF7E2FEF2E761684A0802F5A0
:10A6D000740202F51052B2FBF1F292B2DA60EFE7C7
:10A6E000FFF780FEE4E761684A0802F50042F2E7FE
:10A6F000B2F5004FDAD1FFF7AFFE63685A0802EBFC
:10A700004000B0FBF3F39BB2002023F00F02C3F331
:10A71000420321681343CB6038BDB2F5004FD1D15D
:10A72000FFF7B4FEE9E7B2F5004FCED162685308F7
:10A7300003F1F47303F59043B3FBF2F3E3E7B2F5EF
:10A74000004FCDD1FFF74EFE61684A0802EB40038F
:10A75000B3FBF1F3D7E700BFF369FFEF001001404F
:10A76000180406080044004000480040004C004027
:10A77000005000400014014000780040007C004080
:10A78000044B194491F82F20835823F00103835080
:10A79000704700BF180406080269202341681F2A79
:10A7A00070B504462DD94968203A93400B4227D012
:10A7B000A5692B7C022B01D100232B746B68134EEF
:10A7C0001B69EA68C3F30323506806EB8303996BA4
:10A7D000FFF7D6FF6A6811685279CB6806EB42062C
:10A7E000B6F8582002F4F05223EA020322691F2A25
:10A7F000CB604FF02003616805D9203A9340CB60CD
:10A8000070BD0968D1E793408B60F9E7180406082A
:10A81000A348A44AA449121A70B5A4B052F0FAFB96
:10A82000A24A0020D2F8883043F47003C2F888307E
:10A830009F4B196841F0010119609860196821F077
:10A84000847121F4803119609A495960196821F4A2
:10A85000802119609849D8609160BFF34F8FBFF392
:10A860006F8FC2F85002BFF34F8FBFF36F8F5169E4
:10A8700041F400315161BFF34F8FBFF36F8F1A6CFA
:10A8800042F080521A641A6C02F080520292029ACC
:10A890008A4A116841F440411160126802F4404252
:10A8A0000192019A9A6802F00C02042A07D09A6871
:10A8B00002F00C02082A65D15A68520262D57C4B1C
:10A8C0001B687B4A936803F00C03082B68D013685D
:10A8D0007B4C23F080731360216813689D0160D462
:10A8E00047F6C07393FAA3F3B3FA83F04FF44033FF
:10A8F00093FAA3F34FF0706191FAA1F14FF4D8737A
:10A90000B1FA81F18340092000FA01F10B4343F0D1
:10A91000015343F008035360136843F080731360DE
:10A92000634B21681A68900140D51A6C42F080523E
:10A930001A641B6C03F080530393039B5F4B1A68EC
:10A9400042F480321A6021685A68D20333D51A68FB
:10A9500042F400321A60594A216853689B0330D58B
:10A960004FF400134FF4C07C04A804934FF000632D
:10A9700021930723CDE908C303230A93FDF7ACFE17
:10A9800028B3FEE71A684A4942F480321A604C4AFA
:10A9900010680B689E0394D413681B1A642BF8D9B3
:10A9A000FEE723685B1A022B97D9F9E72268521A4F
:10A9B000022AB7D9F4E72268521AB2F57A7FC3D9CE
:10A9C000FEE723685B1AB3F57A7FC6D9F8E73D4AFC
:10A9D000136803F00F03062B08D9354B9A6822F051
:10A9E000F0029A601A6890010CD4FEE7136823F015
:10A9F0000F0343F007031360136803F00F03072BE3
:10AA0000F3D1EAE79A6841F2883022F0030242F07B
:10AA100002029A6021689A6802F00C02082A39D171
:10AA2000284A1368190755D4214CA36823F4E0532E
:10AA300043F4A053A360A36823F4604343F40043AA
:10AA4000A360FFF7CFFCA368F02292FAA2F2B2FA59
:10AA500082F203F0F0031C4ED3401C4D334493F8B4
:10AA60006030D840C5F8BC0148F03AFD184B04A846
:10AA700004930023CDE91333CDE91533CDE9173322
:10AA8000CDE91933CDE91B33CDE91D33FDF724FEA4
:10AA900060B3FEE72268521A8242BCD9A5E700BF24
:10AAA0000000000078230000C41C070800ED00E04F
:10AAB0000038024010300024000000080070004000
:10AAC000E8260120003C024018040608000001208E
:10AAD000C0FF0300136823F00F0343F00703136064
:10AAE000136803F00F03072B9ED07EE7D4F88C3059
:10AAF00023F08073C4F88C30D4F88C3043F080732A
:10AB0000C4F88C30A36803F00C03042B14D0082B7A
:10AB100014D0184BC5F8BC31174B9B68C3F3031313
:10AB20001E44D5F8BC3196F86020D340134A9342B6
:10AB3000C5F8BC311BD0FEE7114BEBE763686268D8
:10AB400013F4800F636802F03F0218BF0C49C3F38F
:10AB5000881308BF0749B1FBF2F25343064A526813
:10AB6000C2F3014201325200B3FBF2F3D2E724B048
:10AB700070BD00BF0024F4000038024000E6DF0C86
:10AB800000127A0003682DE9F041C3F30D04054675
:10AB900088464D4F002C62D14C4A93421ED302F599
:10ABA0008042934219D302F5804293421ED3484A11
:10ABB00093421DD902F5803293421BD902F500322F
:10ABC000934219D902F50032934217D902F50032A7
:10ABD000934215D9052009F09BFE012497F8E43330
:10ABE000012B0FD14FF0FF30BDE8F0810224F5E7D3
:10ABF0000324F3E70424F1E70524EFE70624EDE757
:10AC00000724EBE7012387F8E43348F081FA68BBB7
:10AC1000304E336923F440733361336943F4007376
:10AC20003361336923F0F8033361782393FAA3F394
:10AC3000B3FA83F332699C40144344F00204346154
:10AC4000336943F480333361BFF34F8F48F060FAC8
:10AC5000336923F07A03336140B987F8E40397F846
:10AC6000E433012B06D16FF00100BDE7002387F824
:10AC7000E433B7E701232E68D8F8008087F8E4337F
:10AC800048F046FAB0B9134C236923F440732361AA
:10AC9000236943F400732361236943F001032361B3
:10ACA000C6F80080BFF34F8F48F032FA236923F0D3
:10ACB00001032361002387F8E4330028D3D12B68F4
:10ACC00004332B6090E700BFE82601200040000815
:10ACD000FFFF0008003C02400148FDF7CDBC00BF6B
:10ACE000D82A01200148FDF7D1B900BFD82A012098
:10ACF0000148FDF7C1BC00BF282B01200148FDF72A
:10AD0000C5B900BF282B01200148FDF7B5BC00BF25
:10AD1000782B01200148FDF7B9B900BF782B01203D
:10AD20002DE9F8438F4F0C26054606FB0076D6F832
:10AD3000E831002B00F0108196F8EE0148F0D0F8D1
:10AD400096F8EC0106F01CFF044696F8ED0106F0BB
:10AD500017FF6B1C0646DBB21CB140F60C122372C7
:10AD6000E2801EB140F60C223372F28020464FF092
:10AD7000090905F084FA304605F081FA11212046D0
:10AD800006F0B2FE1121304606F0AEFE4FF0650827
:10AD900003E00520002109F095FD204605F05EFA4C
:10ADA00010B9B8F10108F4D1204606F0E5FD002104
:10ADB000052009F087FD204605F061FA05200021F5
:10ADC00009F080FDB9F10109E0D120464FF00C08EF
:10ADD00006F0D2FD0021052008FB057809F072FD80
:10ADE000304606F0C9FD0021052009F06BFD204624
:10ADF00005F045FA0021052009F064FD304605F014
:10AE00003EFA204698F8F2213E2106F093FE5024A7
:10AE10003046554E98F8F2213E2106F08BFE04FB99
:10AE20000564D8F8E831C4F8F033FFF715FB98F85B
:10AE3000EF31022B00F09280032B00F09180012B68
:10AE400014BF4FF4C8714FF4487147F0C1FF50224E
:10AE50000021C4F8F40302FB05630120C3F80014C9
:10AE6000C3F80414C3F80C14C3F81014C3E9FE109B
:10AE700093F8311401F0FF0009B983F8300402FBA4
:10AE800005622424D2F8F03382F83144196821F0A5
:10AE900001011960D2F8F41321F070611961996809
:10AEA00021F4004199604FF400419960596841F0E4
:10AEB000007141F400415960D96821F40041D96022
:10AEC000D2F808140902D96000211960186840F00E
:10AED000010018602020C2F8341482F83104C2F84E
:10AEE000201482F8321492F8310420285FFA80FC92
:10AEF00017D192F83004012813D082F83144186831
:10AF000020F001001860186820F48050186018685C
:10AF10001860186840F00100186082F831C482F8A7
:10AF200030140C24022104FB057494F9F10148F05B
:10AF300045F994F9F101FFF72DF8022194F9F00198
:10AF400048F03CF994F9F001FFF724F85020012370
:10AF500000FB056585F8EC33BDE8F883642174E7F0
:10AF6000C82172E700000120E82601202DE9F04FFA
:10AF7000984685B0431C064689469DF83C5003928E
:10AF800000F02081AA4F502303FB007393F8ECB329
:10AF9000BBF1000F6ED0FF2A03D0B8F1000F40F0D4
:10AFA000BE80002D00F0BB805024744307EB040AE0
:10AFB0009AF83134202B40F0FC809AF83034012B81
:10AFC00000F0F7809B4B0122D7F800B04FF400410E
:10AFD0001C448AF830241923CDF800B02046FDF730
:10AFE0006FF8002840F0E58021231FFA88F809FA5D
:10AFF00002F9CAF824048AF8313410238AF832346A
:10B000000E9BCAF83404CAF81434AAF81A84BAF8A1
:10B010001A349BB2FF2B31D94FF40053FF22AAF808
:10B02000182400934FF080734FF050084946204693
:10B0300008FB0678FDF762F8B8F81A34594620463E
:10B040009BB23BBB48F01CF838BBD8F8F03320214A
:10B05000AB46D9615A6822F0FF7222F48B3222F497
:10B06000FF7222F001025A6088F8311488F8300427
:10B0700088F83204584605B0BDE8F08FBAF81A24B3
:10B080004FF4005392B2AAF81824D2B200934FF0B2
:10B090000073C9E748F018F810B1D8F8343488E0E4
:10B0A000D8F814345A1CC8F81424D8F8F0231B78A4
:10B0B0009362B8F81824B8F81A34013A013B92B2F6
:10B0C0009BB2A8F81824A8F81A34002AB4D1B8F80A
:10B0D0001A349BB2002BAFD00A2380212046CDF832
:10B0E00000B0FCF7EDFF002863D1B8F81A349BB22A
:10B0F000FF2B0AD9FF224FF08073A8F81824009084
:10B1000049462046FCF7FAFF96E7B8F81A244FF0B4
:10B11000007392B2A8F81824D2B20090F0E750243D
:10B1200074433D1995F83134202B42D1B8F1000F0A
:10B130003FD095F83034012B3BD03E4B0122D7F85D
:10B1400000A04FF400411C4485F830241923CDF8A9
:10B1500000A02046FCF7B4FF58BB212309FA02F9EE
:10B160001FFA88F8C5F8240485F83134402349468D
:10B1700085F832340E9BC5F834042046C5F81434E3
:10B180004FF40053A5F81A8400934FF08073FCF736
:10B19000B5FF5146204647F097FF0246A8B1D5F8C3
:10B1A0003434502303FB0673D3F83424002283F88D
:10B1B0003024B7F8DC34304601339BB2A7F8DC34D6
:10B1C000FFF7AEFD4FF0000B54E7D5F8F033204603
:10B1D000039999620A238021CDF800A0FCF770FF43
:10B1E0000028DED1B5F81A349BB2FF2B09D8B5F888
:10B1F0001A244FF0007392B2A5F81824D2B200902E
:10B2000005E0FF224FF08073A5F8182400904FF05E
:10B2100050084946204608FB0675FCF76FFF51466B
:10B22000204647F051FF38B108FB067835E700BFEC
:10B23000E8260120D82A0120D5F814345A1CC5F874
:10B240001424D5F8F0231B789362B5F81824B5F8C8
:10B250001A34013A013B92B29BB2A5F81824A5F822
:10B260001A34DAB9B5F81A349BB2BBB10A2380217B
:10B270002046CDF800A0FCF723FF002899D1B5F8AF
:10B280001A349BB2FF2B16D9FF224FF08073A5F81A
:10B290001824009049462046FCF730FFB5F81A34D0
:10B2A0009BB2002BBBD15146204647F0E9FE60B16E
:10B2B000D5F834347DE7B5F81A244FF0007392B214
:10B2C000A5F81824D2B20090E4E7D5F8F033202195
:10B2D000D9615A6822F0FF7222F48B3222F4FF7295
:10B2E00022F001025A6085F8311485F8300485F89F
:10B2F0003204BFE62DE9F04FB0F1FF3F85B0804644
:10B3000093469DF83C9000F09A805024B74F4443F8
:10B310003D1995F8ECA3BAF1000F00F0FB809BB249
:10B32000FF2A05F57C744FEA4106039340F0F6804E
:10B33000B9F1000F00F0F28095F83134202B75D16F
:10B3400095F83034012B71D00122D7F800A01923D1
:10B350004FF4004185F830242046CDF800A0FCF7DA
:10B36000AFFE002862D12223C5F8240485F83134C9
:10B37000102385F832340E9BC5F83404C5F8143414
:10B38000039BA5F81A34B5F81A349BB2FF2B1DD9CC
:10B390004FF41053A5F818B45A4600934FF0807339
:10B3A00050253146204605FB0875FCF7A7FEB5F889
:10B3B0001A349BB2002B56D15146204647F060FE0E
:10B3C000002800F09280D5F834342FE0B5F81A2424
:10B3D0004FF4105392B2A5F81824D2B200934FF054
:10B3E0000073DDE75146204647F012FEC8B9D5F894
:10B3F000F0339A6912F0200224D02021D9615A68D2
:10B4000022F0FF7222F48B3222F4FF7222F001024A
:10B410005A60C5F8340485F8300485F8311485F88D
:10B420003204502303FB0873D3F83434B7F8DC3408
:10B43000404601339BB2A7F8DC34FFF771FC4FF0B4
:10B44000000A67E03B68A3EB0A030A2B0BD9D5F887
:10B45000343485F8302443F02003C5F834342023F5
:10B4600085F83134DDE7D5F8F0339A695207B9D55C
:10B470005A6AD5F81434591CC5F814141A70B5F862
:10B480001824B5F81A34013A013B92B29BB2A5F8E0
:10B490001824A5F81A34002A89D1B5F81A349BB2B9
:10B4A000002B84D00A2380212046CDF800A0FCF791
:10B4B00007FE0028BAD1B5F81A349BB2FF2B0AD97F
:10B4C000FF224FF08073A5F81824009031462046E3
:10B4D000FCF714FE6BE7B5F81A244FF0007392B234
:10B4E000A5F81824D2B20090F0E7D5F8F033202167
:10B4F000CA46D9615A6822F0FF7222F48B3222F4D4
:10B50000FF7222F001025A6085F8311485F8300488
:10B5100085F83204504605B0BDE8F08F502505FB94
:10B52000087595F83134202B80D10E9B002B3FF409
:10B530007DAF95F83034012B3FF478AF0122D7F876
:10B54000009019234FF4004185F830242046CDF8AF
:10B550000090FCF7B5FD00287FF468AF2223C5F802
:10B560002404314685F831344FF0400385F83234F5
:10B570000E9BC5F83404C5F81434039BA5F81A349F
:10B580004FF40053009303462046FCF7B7FD4946AD
:10B59000204647F099FD024650B1D5F83434502387
:10B5A00003FB0873D3F83424002283F830243DE7EA
:10B5B000D5F8F03340212046C3F828B00A23CDF84F
:10B5C0000090FCF77DFD0028E9D1B5F81A349BB254
:10B5D000FF2B0DD8B5F81A244FF4105392B2A5F8EA
:10B5E0001824D2B200934FF0007309E0E82601203E
:10B5F0004FF41053FF22A5F8182400934FF08073E6
:10B6000050253146204605FB0875FCF777FD0A23D7
:10B61000002204212046CDF80090FCF751FD0028BF
:10B620007FF404AFD5F8F033596AD5F81434581CB8
:10B63000C5F814041970B5F81834B5F81A14013B9C
:10B6400001399BB289B2A5F81834A5F81A14E3B9E8
:10B65000B5F81A349BB2C3B10A2380212046CDF835
:10B660000090FCF72DFD00287FF4E0AEB5F81A3409
:10B670009BB2FF2B2AD9FF224FF08073A5F8182424
:10B68000009031462046FCF739FDB5F81A349BB2DC
:10B69000002BBCD14946204647F0F2FC00287FF43D
:10B6A00092AED5F8F0332021D9615A6822F0FF72AA
:10B6B00022F48B3222F4FF7222F001025A6085F8E4
:10B6C000311485F8300485F8320423E7B5F81A24DC
:10B6D0004FF0007392B2A5F81824D2B20090D0E7D0
:10B6E0000348D0F8183213B100F5037018477047BB
:10B6F000000001200348D0F8383213B100F50B7078
:10B7000018477047000001200348D0F8583213B1A1
:10B7100000F5137018477047000001200348D0F867
:10B72000783213B100F51B701847704700000120F4
:10B730000348D0F8983213B100F5237018477047CA
:10B74000000001200348D0F8B83213B100F52B7087
:10B7500018477047000001200348D0F8D83213B1D1
:10B7600000F5337018477047000001200348D0F8F7
:10B77000F83213B100F53B70184770470000012004
:10B780000348D0F8183313B100F5437018477047D9
:10B79000000001200348D0F8383313B100F54B7096
:10B7A00018477047000001200348D0F8583313B100
:10B7B00000F5537018477047000001200348D0F887
:10B7C000783313B100F55B70184770470000012013
:10B7D0000348D0F8983313B100F5637018477047E9
:10B7E000000001200348D0F8B83313B100F56B70A6
:10B7F00018477047000001200348D0F8D83313B130
:10B8000000F5737018477047000001200348D0F816
:10B81000F83313B100F57B70184770470000012022
:10B8200038B5446844F4805444603BB9012004E0D6
:10B83000013C05D1FCF7D1FC002038BD40F2E934D1
:10B840008568AD07F4D56AB112F8014B047340F274
:10B85000E9348568ED0707D5C46809B101F8014BE3
:10B86000013BE2E7FF24F1E7013CF2D1E2E70023EC
:10B87000054A52F83310814201D1D8B270470133E2
:10B880000E2BF6D1FE2070478804060870B507EE2F
:10B89000902A0E46002800F088800368F8EE677A48
:10B8A000D3E900341D68414B93ED6F7AB8EE477AC7
:10B8B00087EE270ADFED3E7A30EE270A4EF0BCFD18
:10B8C00023680138711E9D4280B289B205D1636838
:10B8D000834202D1E3688B4267D00023E160C4E970
:10B8E0000433A3608023C4E90050A36120464BF0D9
:10B8F00017F9304B9D4216D0B5F1804F13D0A3F508
:10B900007C439D420FD003F580639D420BD003F52D
:10B9100080639D4207D003F578439D4203D003F531
:10B9200070539D4241D194F83C30012B3DD002230D
:10B93000214A84F83D30236899680A409A609A68E1
:10B9400022F4803222F007029A60012284F83D201E
:10B95000002284F83C20174A954212D0B5F1804F5E
:10B960000FD0A2F57C4295420BD002F58062954241
:10B9700007D002F58062954203D002F578429542E5
:10B9800013D10C485A688342996803D000F580604F
:10B99000834201D122F4700222F0700221F0800172
:10B9A0005A609960002384F83C3070BD000001208B
:10B9B0000AD7233C000001408800FEFF2DE9F04734
:10B9C00007460068FFF753FF0D28054608DD0024F1
:10B9D000274A0021052003F095FA2046BDE8F087AC
:10B9E000DFF898904FEA800809EB800ADAF8E06403
:10B9F0005EBB0721682003F051FB0446CAF8E0044F
:10BA000028B901461B4A052003F07CFAE5E73146D8
:10BA1000682253F0A7FC18482AB2DAF8E04400F193
:10BA2000700300EBC500A46003EBC203006F246247
:10BA30002360A4632465FFF71AFF0D289EBF09F554
:10BA4000A36600B206EB80166660C84478791821B8
:10BA50000023D8F8E04401FB0042D760C2E9043378
:10BA600000FB0112A35401FB00440834B5E700BFFA
:10BA7000B7B00608DCB0060818040608E82601205E
:10BA80000A4B30B51A4600241D79854208D1DD687D
:10BA9000294203D0142000FB042030BD0029F9D036
:10BAA00001341433052CEFD10020F6E70C040120FB
:10BAB00043680068F0B540685C799A79974B12F05A
:10BAC0000202234490F83C400EBF1546022208258E
:10BAD000012C93F8E03017D001240C2B80F83C4067
:10BAE0004FF0020480F83D4000F0C6800DD8042BD2
:10BAF00065D0082B00F09080002B32D0012380F815
:10BB00003D30002380F83C30F0BD102B00F0DB808E
:10BB1000142BF3D103681C6A24F480141C621D6A80
:10BB20005E6825F400155C6D45EA025224F08074CD
:10BB30007B4D24F4E044AB4244F4C04403D005F50B
:10BB40008065AB4201D146F480265E605C65D965B4
:10BB50001A625A6D42F400625A655A6D22F480628C
:10BB6000D7E003681C6A24F001041C621C6A5F6849
:10BB700024F002049E69224326F48036684C26F0A5
:10BB80007306A34246F0600603D004F58064A34226
:10BB900006D122F0080247F440772A4322F004023B
:10BBA0005F609E6159631A629A6942F008029A6165
:10BBB0009A6922F004029A619A699A619EE7036881
:10BBC0001C6A24F010041C621C6A5F6824F02004C4
:10BBD0009E6944EA021226F08076514C26F4E6462D
:10BBE000A34246F4C04603D004F58064A34207D1C3
:10BBF00022F0800247F4406742EA051222F0400238
:10BC00005F609E6199631A629A6942F400629A6168
:10BC10009A6922F48062CEE703681C6A24F4807477
:10BC20001C621C6A5F6824F40074DE6944EA022224
:10BC300026F480363A4C26F07306A34246F060069E
:10BC400003D004F58064A34207D122F4006247F4D4
:10BC5000405742EA052222F480625F60DE61D963C8
:10BC60001A62DA6942F00802DA61DA6922F0040243
:10BC7000DA61DA69DA6141E703681C6A24F4805406
:10BC80001C621D6A5E6825F40055DC6945EA0232D3
:10BC900024F08074224D24F4E644AB4244F4C044C2
:10BCA00003D005F58065AB4201D146F480465E6065
:10BCB000DC6119641A62DA6942F40062DA61DA69F5
:10BCC00022F48062D4E703681C6A24F480341C6286
:10BCD0001D6A5E6825F400355C6D45EA024224F475
:10BCE00080340F4D24F07004AB4244F0600403D064
:10BCF00005F58065AB4201D146F480365E605C6537
:10BD000099651A625A6D42F008025A655A6D22F01E
:10BD100004025A655A6D5A65F0E600BF1804060819
:10BD20000000014043685A79032A0FD8DFE802F087
:10BD30000205080B186834307047186838307047AF
:10BD400018683C30704718684030704700207047D2
:10BD5000D0E9003251795868054B0B4493F8E01054
:10BD600093795B0701D54AF0AABE4AF0BCBE00BF7A
:10BD7000180406082DE9F84343680446274E884610
:10BD80001B69C3F3032306EB83039F6BC3685D68E2
:10BD9000EFF31189102383F3128842682846116853
:10BDA0005279CB6806EB4202B2F8582002F4F05206
:10BDB00023EA0203CB603946FEF7E2FCE26813692E
:10BDC000516820221F2B25D9203B9A40CA605FFA78
:10BDD00089F989F311883E44204696F82F10666948
:10BDE00029444B681B0C1B0443EA08034B60FFF714
:10BDF00099FF0B4BDB5D5A19D66090605A5942F09F
:10BE000010025A515A5942F001025A510123237427
:10BE1000BDE8F8839A408A60D9E700BF1804060895
:10BE2000470406080268137E012B26D102231376ED
:10BE30004FF4007392F83010012904D1022143F429
:10BE4000806382F8301092F84810012904D1022151
:10BE500043F4006382F8481092F8601001290ED173
:10BE6000022143F4805382F86010126800211268A6
:10BE70005162D1680B43D36003E00023DAE7002B63
:10BE8000F3D17047024B0348D3F8E014FCF706BF28
:10BE9000E82601200000014010B5064C0648D4F801
:10BEA000E014FCF7FBFED4F804150448BDE810408C
:10BEB000FCF7F4BEE82601200000014000440140E8
:10BEC000034B4FF08040D3F8E414FCF7E7BE00BF0B
:10BED000E8260120024B0348D3F8E814FCF7DEBE45
:10BEE000E826012000040040024B0348D3F8EC147C
:10BEF000FCF7D4BEE826012000080040024B0348AE
:10BF0000D3F8F014FCF7CABEE8260120000C00406C
:10BF1000024B0348D3F8FC14FCF7C0BEE82601200E
:10BF20000004014010B5064C0648D4F8FC14FCF798
:10BF3000B5FED4F810150448BDE81040FCF7AEBEBD
:10BF4000E826012000040140001C004010B5064C0A
:10BF50000648D4F8FC14FCF7A1FED4F814150448E4
:10BF6000BDE81040FCF79ABEE8260120000401401D
:10BF700000200040024B0348D3F80015FCF78EBEAA
:10BF8000E826012000400140024B0348D3F8081581
:10BF9000FCF784BEE826012000480140024B03481C
:10BFA000D3F80C15FCF77ABEE826012000180040F3
:10BFB000704710B501208EB006F00EFF012809D1A0
:10BFC000002106F00FFF614B1A6882F308885B6856
:10BFD0009847FEE75E4A00245E4BD1685E4821F434
:10BFE000E0610904090C0B43D3605C4B596F196B7A
:10BFF00041F480211963196B01F480210D910D9991
:10C00000196B41F480111963196B01F480110C91C3
:10C010000C99196B41F480011963196B01F48001CB
:10C020000B910B99196B41F000511963196B01F0D9
:10C0300000510A910A99196B41F080411963196BFB
:10C0400001F0804109910999196C41F4003119649A
:10C05000196C01F4003108910899196C41F48021A0
:10C060001964196C01F4802107910799196C41F446
:10C0700000211964196C01F4002106910699196CCC
:10C0800041F480111964196C01F48011059105992E
:10C09000196C41F080411964196C01F080410491E0
:10C0A0000499196C41F000411964196C01F00041C8
:10C0B00003910399596C41F010015964596C01F0D6
:10C0C000100102910299596C41F020015964596C98
:10C0D00001F0200101910199596C41F4006159640A
:10C0E0005B6C1F4903F400630093009B1D4BD3F866
:10C0F000BC31B3FBF1F1C0F89818D2F8FC101A4823
:10C1000041F08071C2F8FC101849C1F8B00F4C60C2
:10C11000086840F0010008604FF47A71B3FBF1F356
:10C12000013BB3F1807F08D24FF0E0214B61F02357
:10C1300082F8233007238C610B614FF0E0221369F2
:10C1400043F0040313610EB010BD00BF0000F01FE8
:10C1500000ED00E00003FA05E82601200038024067
:10C1600040420F000000012055CEACC5001000E099
:10C17000074B03EB8000D0F8E43033B193F8AD20E7
:10C180004A7093F8AC300B7070474B70FBE700BF00
:10C19000180406082DE9F04117462C4A9846054632
:10C1A00002EB8003D3F8E44084B304F1AE0302F55C
:10C1B000827294F8AD00261DA36104F5D773626006
:10C1C000E3614FF48073E160C4E904332368C4F889
:10C1D000A830A36305F0D4FC18F0080F19D001357E
:10C1E000EDB218B140F20673C380057294F8B6221E
:10C1F000022105F09FFC94F9B702D4F8B81246F07A
:10C20000DDFF94F9B7023446FDF7C4FE2046BDE8D1
:10C21000F081BA0794F8AC800BD56B1CDBB218B177
:10C2200040F206520372C28094F8B622022105F051
:10C2300081FCFB07DFD50135404605F0A1FCEDB2DE
:10C240000028D3D040F20663CEE700BF18040608EA
:10C250000148FCF7FDBD00BF740401200148FCF754
:10C26000F7BD00BF300701200148FCF7F1BD00BF5A
:10C27000EC0901200148FCF7EBBD00BFA80C012030
:10C280000148FCF7E5BD00BF640F01200148FCF741
:10C29000DFBD00BF20120120426B2423816870B5EE
:10C2A00080F89D300446136800F1340523F0010343
:10C2B0001360002313605360936081638179C0F839
:10C2C000A03080F89C3080F89D3080F89E30880245
:10C2D000A36400F48050E3646365E063080363795A
:10C2E00000F4005013F0010620644FEA012000F42E
:10C2F000806060641CBF0420A06413F002031EBFB2
:10C30000A06C40F00800A064C8070FD536B1A06D3E
:10C3100040F00200A0654FF48030206633B1A36D79
:10C3200043F00103A3654FF40033E365242311F0C8
:10C33000080F94F89D10284684F89D30136823F068
:10C340000103136036D0FEF7BBF8012818D0A36DA7
:10C3500013B12846FBF7ECFE636B5A6822F4904257
:10C360005A609A6822F022029A609A6842F00802A3
:10C370009A6028461A6842F001021A604AF03EFBB1
:10C380006179CA070DD5D4F8A4301A6842F48072D6
:10C390001A609A6842F001029A601A6842F020021C
:10C3A0001A608B0705D5D4F8A420136843F08003E6
:10C3B000136070BDFEF784F80128E1D0A36D13B1BE
:10C3C0002846FBF7B5FE636B5A6822F490425A6028
:10C3D0009A6822F02A02CBE781605DE741715BE752
:10C3E000704710B51C2005F0CBFB0446112105F069
:10C3F0007BFB204605F0C0FAC82008F074FA2046FE
:10C40000BDE8104003F03BBF934B2DE9F04FD3F84C
:10C410009C5887B06B6913F00103029340F0AA8126
:10C420006A69AB691A4200F0A5816B69AA69134079
:10C430009C0701D502236B616B69AA69134018033D
:10C4400000F19B81844CD4F89C385A6999690A4060
:10C45000510311D5D3F8182803F5006304F69C079F
:10C4600005F5106ADB694FF0000913409BB2019398
:10C47000019B002B40F02584D4F89C084269836915
:10C480001A4216D5D5F8043823F00103C5F804384C
:10C4900094F8883C012B15BFD4F8983C002393F8FE
:10C4A000FD2184F8883C18BF83F8FC214FF000433D
:10C4B00043614369826913401B050FD5D5F80838DD
:10C4C000DF0708D5D4F8983C93F8FC2183F8FD21C8
:10C4D000042283F8FC214FF40063436143698269BD
:10C4E00013401E010FD54FF00063436194F8883C60
:10C4F000002B40F0F684012384F8883C436DC3F39D
:10C500008303C4F88C3C436982691340D9043AD54B
:10C51000D5F80438102105F5006623F00103736097
:10C520004AF02AFAD4F8A00805F510630022FF218A
:10C53000824240F0E1844FF0FF33B361F36943F08E
:10C540000113F361D4F8CC38002B00F0DC84D6F86A
:10C55000843043F00B03C6F88430736C43F00B0354
:10C560007364D5F800383D4A23F4FE6394F8AC18A0
:10C57000D4F89C08C5F800384AF0A0F9D4F89C38E3
:10C580004FF480525A61D4F89C385A6999690A402C
:10C59000920473D5D3F8002922F4FF6222F0070237
:10C5A000C3F8002903F50062916801F0060104292F
:10C5B00005D1D3F8001941F00301C3F800195168FF
:10C5C00041F480715160D96821F47051D96091684B
:10C5D00011F0060F11D0916801F00601022900F058
:10C5E0009C84916801F00601062900F09684926807
:10C5F00002F00602042A00F090844FF40072002733
:10C60000C4F8B028DA68C4F8A87842F41052DA60A6
:10C61000D4F8986C00224FF0400840231146D6F819
:10C6200030024AF0A1F8434600228021D6F83002B9
:10C63000C6F810814AF098F80123C6F8208086F8E1
:10C64000FC31D6F818325BB9D6F8203243B9D6F8A7
:10C6500028325BB104E000BFE8260120403301200E
:10C66000D6F81432304631795B689847D4F8983C54
:10C670004FF400521F74D4F89C385A61D4F89C28A7
:10C68000536991690B40DB062FD5936923F01003A2
:10C6900093612B6AC3F3434003F00F07022840F075
:10C6A000AB8447F6F0710B421BD01C20C3F30A1376
:10C6B00005F5805C00FB0740DE1CD0F8A01AB61020
:10C6C0000298864240F08E841C2101FB0741D1F87C
:10C6D000A05AD1F8AC0A1D441844C1F8A05AC1F8B8
:10C6E000AC0A936943F01003936153699269134054
:10C6F0001F070ED5D4F8980C90F8FC31032B04D109
:10C70000D0F81432DB6903B19847D4F89C3808227A
:10C710005A61D4F89C28536991690B40DE0202D516
:10C720004FF480135361536991690B409D0202D508
:10C730004FF400135361536991690B40580002D5BF
:10C740004FF080435361536991690B40590711D5EC
:10C7500055686B0709D5D4F8980C012380F8FC3193
:10C76000D0F8143201795B689847D4F89C385A683D
:10C7700015435D6007B0BDE8F08FD5F8183805F5B2
:10C780003068D5F81C284FF0000AB24F1340A7F6C6
:10C790009C061B0C0193019B002B3FF453AE019BA5
:10C7A000DA0740F14C81D6F89C385FFA8AF103F53C
:10C7B000306203F5006302EB411292685B6902EAA2
:10C7C000030919F0010F3BD00123C8F80830D6F84F
:10C7D000AC38012B0DD1D8F81030D7F80022C3F3B4
:10C7E0001203D31AC7F81032D7F804321344C7F82B
:10C7F0000432D6F8984C002979D1D4F8F431032BBF
:10C8000010D1D4E94303984263D9C01AD6F8A02ABC
:10C810008342C4F80C0128BF0346D4F830029BB20F
:10C8200049F01EFFD6F8AC18012909D1D6F8A83A6C
:10C830005AEA030304D1884AD6F89C084AF03EF825
:10C8400019F0080F00F0EF80D6F8984C96F858CC05
:10C8500004F5027B84F808C296F859EC84F809E2E2
:10C8600096F85B1C96F85A3C03EB01239BB2A4F8A4
:10C870000A3296F85D2C96F85C0C00EB022080B230
:10C88000A4F80C0296F85F1C96F85E2C02EB0122CD
:10C89000012192B2C4E97D120CF01F01A4F80E220E
:10C8A000012900F04881022900F05A81002940F056
:10C8B0000582BEF1090F00F28F80DFE81EF015013E
:10C8C00031018D0026018D00870024008D000501B7
:10C8D000CF00D4F814321B692BB194F8FC21032A41
:10C8E00001D120469847204649F094FF9AE7D4F8B2
:10C8F00014329B69002B95D094F8FC21032A91D126
:10C90000204698478EE71A0A013A062A64D8DFE8DB
:10C9100002F0041D2A63634A5300D4F810321B68E6
:10C920000DF11601207C9847BDF81620002A77D01B
:10C93000B4F80E32002B73D09A42014628BF1A4633
:10C94000ADF81620204649F06EFF69E0227CD4F84D
:10C95000143232B99B6A0DF11600984702234370D6
:10C96000E2E7DB6AF7E7DBB2052B35D8DFE803F057
:10C9700003070B0F1317D4F810325B68D0E7D4F815
:10C9800010329B68CCE7D4F81032DB68C8E7D4F8E3
:10C9900010321B69C4E7D4F810325B69C0E7D4F8E1
:10C9A00010329B69BCE7237CB3B9D4F814320DF183
:10C9B00016005B6B9847B7E7237C6BB9D4F8143249
:10C9C0000DF116001B6B98470723C8E7024303D1FC
:10C9D00094F8FC11032901D1204665E003F07F0B98
:10C9E000D4F8303284F8FEB193F8B81301290ED090
:10C9F0001968D1F8000820F4FE60C1F80008D1F8E9
:10CA0000000840EA0B10C1F8000883F8B82320465C
:10CA100049F000FFBBF1000F1AD0022384F8FC316B
:10CA20000823C8F8083019F0100F02D01023C8F8F6
:10CA3000083019F0200F02D02023C8F80830019BDD
:10CA40000AF1010A08F120081C375B080193A2E6ED
:10CA50000123E3E7842F012040330120D9B20129CB
:10CA600086F89C1CB8D894F8FC31022B0FD0032B0D
:10CA7000B2D1E1B902232046616084F8FC31D4F8D8
:10CA800014325A689047204649F0C4FEC8E700298E
:10CA9000F9D001210323616084F8FC312046FBF7C3
:10CAA00013FC02282046EFD146F0A4FAB8E76168EB
:10CAB0000129E8D0D4F81432C9B220465B689847FF
:10CAC00096F89C1C6160E9E7012A85D194F8FC3155
:10CAD000022B04D0032B7FF47FAF211D32E72146C8
:10CAE000002341F8083F2DE794F8FC31023B012B6D
:10CAF0003FF672AF0123E360D4F804320BB1032395
:10CB0000E360022204F10C011CE7012B88D1C4F878
:10CB10000432D4F81432594620469B689847B2E74D
:10CB200094F8FC21023A012A3FF656AF012B7FF41C
:10CB300077AF0023EBE794F8FC31032B7FF44CAF85
:10CB4000C0B203283FF648AFD4F814325946204605
:10CB50009B689847B4F80E32002B7FF461AF92E7E0
:10CB60000CF0600CC1B2BCF1200F06D1D4F8143225
:10CB7000594620469B68984752E7BEF1010F44D0C2
:10CB8000BEF1030F31D0BEF1000F7FF449AF94F82E
:10CB9000FC31022B00F08A80032B7FF41DAF40B2E2
:10CBA00001F07F0210234FF0040E0028B4BF02F101
:10CBB000010C02F1100C00284FF01C0013FB0CE3D9
:10CBC000D4F830C2A8BF00FB01C12344B4BF00FBAE
:10CBD00002C291F8FA211946B8BF92F83A20003AF9
:10CBE00018BF01221A600222ACE694F8FC21022A46
:10CBF0005CD0032A7FF4F0AE002B8AD14B0688D09C
:10CC0000D4F8300249F079FE83E794F8FC21022A37
:10CC10004CD0032A7FF4E0AE002B7FF401AF11F07B
:10CC20007F0C3FF430AF40B2D4F830221C230028F0
:10CC30004FEAD070B4BF03FB0C2103FB01214FF07E
:10CC40000003B4BF383101F5FC718B7081F800C06E
:10CC5000487092F8B833012B3FF45BAF01234FF0DB
:10CC6000200E82F8B8331368A0B1C87803F51063BA
:10CC7000097802381EFB01330128196821F40011DC
:10CC8000196003D8196841F080511960002382F8B7
:10CC9000B8333EE703F530631EFB0C33186820F40D
:10CCA00000101860C97802390129EAE748063FF404
:10CCB000B7AED4F8300249F020FEB1E60CF08001A6
:10CCC000F7E7019BDA0740F1A980D4F89C285FFAC6
:10CCD00089FBD2F8101802F5106252F8CC3C02EB36
:10CCE0004B1223FA0BF892684FEAC8185FFA88F8DB
:10CCF00048EA010808EA020818F0010F4AD00121A9
:10CD0000D5F8343801FA09F123EA0103C5F83438BB
:10CD10000123CAF80830D4F8AC38012B02BFD7E998
:10CD200010239B187B6419F0FF01D4F8986C40F035
:10CD3000A780D6F8F431022B17D1D6E90730834209
:10CD400076D91C221B1AD6F8300202FB0B42039143
:10CD5000D2F8E028F3619BB249F0A4FC03990B469A
:10CD60000A46D6F8300249F07BFC96F80032012BD7
:10CD700002D1002386F80032D4F8AC18012909D179
:10CD8000D4F8E83859EA030304D1A74AD4F89C0838
:10CD900049F094FD18F0080F02D00823CAF80830B3
:10CDA00018F0100F02D01023CAF8083018F0400F06
:10CDB00002D04023CAF8083018F0020F02D0022334
:10CDC000CAF8083018F0800F28D0D4F89C08D7E9AA
:10CDD000133200F5106600F580519B1A3A6C06EB91
:10CDE0004918934201EB0B3BA8BF1346DA1C48BF1E
:10CDF0009A1D9210D8F8181089B2914203D9D7E938
:10CE000013218A424AD8002B08DC0122D0F834389A
:10CE100002FA09F223EA0203C0F83438019B09F14F
:10CE200001091C370AF1200A5B080193FFF720BBB8
:10CE3000B269B2FBF0F300FB132393B9904210D810
:10CE4000D6F8F8118A420CD21A461946D6F83002A2
:10CE5000039349F027FC039BC6F8F8311A4619469C
:10CE60007FE7D6F81432DB682BB196F8FC21032A51
:10CE700001D1304698470523C6F8F4310023EDE789
:10CE8000D6F814325B69002B3FF476AF96F8FC219C
:10CE9000032A7FF471AF304698476DE7521A3B6C16
:10CEA00094F8AC189342A8BF1346DA1C48BF9A1DE9
:10CEB000921031B1796C19447964396D194439652E
:10CEC00098E71FFA83FCD7F844E00CF1030C4FEA13
:10CED000AC0C8C45EED05EF821600131CBF80060DF
:10CEE000F7E7D4F8983C93F8FC2183F8FD2104225D
:10CEF00083F8FC21FFF707BB99600132C3F80812E1
:10CF00002033FFF715BB736943F02B03736133695B
:10CF100043F00B033361FFF724BB0322434944482A
:10CF2000C4F8A8284022C4F8B028424AD2F8BC214C
:10CF30001144814206D8DA6842F470520127DA605F
:10CF4000FFF766BB3C493D481144814203D8DA688B
:10CF500042F46052F2E7A2F574013948A1F510518C
:10CF6000814203D8DA6842F45052E7E7A2F18371B4
:10CF70003448A1F5E741814203D2DA6842F44052D5
:10CF8000DCE7314931481144814203D8DA6842F480
:10CF90003052D3E72E492F481144814203D2DA6838
:10CFA00042F42052CAE72C492C481144814203D252
:10CFB000DA6842F41052C1E7A2F1B7712848A1F52E
:10CFC0005851814203D2DA6842F40052B6E725494B
:10CFD0001144254A9142DA6834BF42F4E05242F4E7
:10CFE000C052ABE7029DDCF8000041F8250028465E
:10CFF00001300290FFF764BB06287FF472AB05F5A1
:10D000008055C3F30A132968C4F8581C2968C4F86A
:10D010005C1C1C2101FB0741D1F8AC0A0344C1F898
:10D02000AC3AFFF75EBB00BF40330120405327FFFF
:10D03000FF340C0000000120401E1BFF3F420F0088
:10D040007F4F120020D6130060B6E5FE5FE31600A6
:10D0500000D3CEFE40771B00C05BB3FEC091210021
:10D0600020753800E05459FEE09C410070B5484CF2
:10D07000D4F888321A69910709D5DA68920706D57B
:10D080006FF002021A619A69002284F8A4221A69D8
:10D09000560709D5DA68550706D56FF004021A61FC
:10D0A0009A69002284F8A4221A69100709D5DA685F
:10D0B000110706D56FF008021A61DA69002284F8B8
:10D0C000A4221A69D20609D5DA68D60606D56FF009
:10D0D00010021A61DA69002284F8A4221A69D507BD
:10D0E0002ED5DA68D0072BD56FF001021A61294AD4
:10D0F000934225D1D4E99125AA4221D0264B8CBF59
:10D10000C2F58055AD1A1A44D4F82032A9B2D3F82A
:10D110001462C3F80822C3F810128EB90121D4F8A2
:10D120003802C3F81412ABB2812149F0BBFAD4F82B
:10D1300044321D44B5F5805F18BF2E46C4F84462E2
:10D14000D4F888321A69110605D5DA68120602D5B4
:10D150006FF080021A611A69D60505D5DA681506DE
:10D1600002D56FF080021A611A69540605D5DA6893
:10D17000500602D56FF040021A611A69910605D572
:10D18000DA68920602D56FF020021A6170BD00BF06
:10D19000E826012000140040B46701202DE9F04189
:10D1A000114E0D46D6F82022D2F81432002BFBD1B6
:10D1B00004464719DFF83480BC4202D12846BDE856
:10D1C000F081D6F8483214F8012B08F80320013317
:10D1D000C3F30B03C6F84832FBF764F90028EBD120
:10D1E000012007F080FBF7E7E8260120B467012063
:10D1F000F8B50D461446FBF759F878B1084ED6F845
:10D20000A07C002C0ADD21462846FFF7C7FFD6F890
:10D21000A03C241A0544DB1B322BF2D9F8BD00BF19
:10D22000E82601202DE9F04F4FF00008DFF8349395
:10D230002DED028B8FB044462FF034FF47462FF080
:10D240000BFF45460646BE4200F3A380642C40F027
:10D250004D816825DFF8E4824C22B54B0021D8F8D7
:10D260004C7155430534C3F8E07308EB05031846C9
:10D2700052F078F84C22002152F074F8AD4A48F888
:10D280000520012247628260AB4AC0E904668262DF
:10D29000C0E90777A64BA94DD3F8E0737300B3F14B
:10D2A000805F18DA4C220021C6F1006654432B1926
:10D2B000184652F057F84C22002152F053F8A04A79
:10D2C0002A51022247624271012296408260C0E9DF
:10D2D0000466C0E907774FF498729A4997484FF06F
:10D2E00099FE964A0421134601395F62C3E9077724
:10D2F00003F14C03F8D1AE68002E45D12B79002BF9
:10D3000042D02B68002B3FD00C468C488C462964B9
:10D31000E963C5E91111C76C00F14C03002F40F01F
:10D32000238102231068002840F04E8186489C1E0D
:10D33000864B3E22C0F88462C0F85C323F23C0E9CD
:10D3400098234023C0E99D41C0F86832A100A30F93
:10D35000002C00F0668140F2FF128A1843F10003AE
:10D36000520A42EAC35202F14003C0F86C3213443D
:10D37000C0F8703203EBC403DA0DC0F858325B0218
:10D38000C0E99F55C0E994320FB0BDEC028BBDE8F7
:10D39000F08F202206A938462FF044FE12226C4955
:10D3A00006A851F071FF0090002840F08D80AF4238
:10D3B0001DD068490C20621CCA4600FB0414664953
:10D3C0000192A7EB050B204601F086FD01214AF8EA
:10D3D0004C4B019AC9E9021557491446C9F828105F
:10D3E000D9F81C10C9E904BBC9E90811D146504B52
:10D3F0003D46D3F8E023C9F81C20122202F138037D
:10D40000501C0DEB0302554B12F8201C18F803209A
:10D4100091425CD108F10108B8F1150F59D12022D1
:10D4200006A9284400252FF0FDFD05AA4C4906A8B1
:10D4300050F000FE05AAAA46AB4608EE102A019558
:10D44000CDE9025538B30BF1FF32042A04D8DFE8E6
:10D4500002F00F13171B1F0002F0F2F9824618EEBC
:10D46000102A3F4900200BF1010B50F0E3FDE9E7E2
:10D4700002F0E6F90190F2E702F0E2F90290EEE73D
:10D4800002F0DEF90390EAE702F0DAF90546E6E792
:10D4900002F0D6F90090BAF1000F12D0AAF2BC7ACD
:10D4A000DDE9012343EA4210039B40EA4A2A68016E
:10D4B00040EAC320009B40EA630040EA0A40C9F802
:10D4C0001C00642C2ED03D4607F50067BBE64FF0EC
:10D4D0000008202808D12035AE42F2DB024606A91A
:10D4E00028462FF09FFD0020024687E7AF4219D063
:10D4F000A7EB0508174A0C27174907FB0427013437
:10D500003846224601F0E8FC0122C9F80070C9E95A
:10D510000225094AC9F82820D9F81C20C9E904883D
:10D52000C9E90822251D002C7FF494AE0424B1E63D
:10D53000F810012032B106086D9F00083C38012028
:10D540003FB106084C050608E82601204CB1060844
:10D55000F6B006088C33012009B1060817B1060899
:10D560002DB106086C3901209F6804F1FF3EC3F815
:10D5700040C07745C3F83CC0C3E911CC05D1002CAD
:10D580003FF402AF53F80C0C3C4604F1010E774512
:10D5900008D10479002C3FF4F7AE43641864744654
:10D5A0001846B8E6A7427FF4EFAE002F3FF4ECAE8A
:10D5B000D0F840E0DEF83C400134CEF83C40C3F8FF
:10D5C00040E0BE468364EAE7107903F1FF3CA0B176
:10D5D0001363D36B5B0116BF03F6FF7301231B0BB1
:10D5E0006344C2E90477C2E90D33D2E90D03013681
:10D5F0004C32181A0133014494E61469136364B180
:10D6000004F6FF74240B64445069546338B100F687
:10D61000FF70000B60449063E7E70124F3E701200B
:10D62000F8E701229FE6F0B59C080E461546270153
:10D6300000EB0414A04206F1100605F1100508D114
:10D6400003F0030339443A4404EB83039C4223D19F
:10D65000F0BD844616ED045AD0ED016A10309CED01
:10D66000006A56ED037A26EE056A10ED027A56ED51
:10D67000025A66EEA76A50ED017A05ED046A27EEBC
:10D68000257A16ED016A45ED036A67EE867A05EDA7
:10D69000027A45ED017ACDE7F4EC017AB1EC017A3A
:10D6A00067EE877AE2EC017AD0E700BF4FF40063BF
:10D6B000838170472DE9F74FCDE900124F4AD38996
:10D6C00011681B025689178AC91A93896EEB0E0ED0
:10D6D000A3FB010403FB0E44C009138940EA446024
:10D6E0001B04E411C018A6FB013506FB0E554FEADA
:10D6F0001323D68844F1000443EA0563F6032D1290
:10D700009B19A7FB012607FB0E664FEAD25245F193
:10D71000000542EA4622F61512F5FA6C46F1000BB6
:10D72000BCF5FA6F7BF100074CDAA2FB02784FF0F0
:10D73000050A02FB06F908EB4909A7FB0A780AFB70
:10D7400009884FEA5709BF0849EAC87947EA887744
:10D75000B0EB090064EB6804DB1B294F65EBA805FF
:10D76000BC454FF0FF377BEB070720DA40F6AC579C
:10D77000D21946F100065643A2FB027202EB46069E
:10D78000FA004FEAC608BA1A48EA577866EB080862
:10D79000101844EB08044FF00B08A7FB087208FBB5
:10D7A00006267F0847EAC677DB1B65EB660501FBAB
:10D7B0000EFEA1FB011202EB4E0EC90F41EA4E0113
:10D7C000BCEB010C009A8AB10C4A5169A1FB0323FE
:10D7D00001FB0535520D009B42EAC5226D15121A58
:10D7E00065EB0404D20B42EA44421A60019B0BB180
:10D7F000C3F800C0012003B0BDE8F08FB877012066
:10D8000024FAFFFF31B10A4BD3ED0C7AFDEEE77A33
:10D81000C1ED007A52B1064B9FED067AD3ED0D7A39
:10D8200067EE877AFDEEE77AC2ED007A0120704755
:10D83000B87701200000C84231B10C4BD3ED0E7A0D
:10D84000F8EEE77AC1ED007A72B1084BDFED086AB5
:10D85000DB6BA3F5D543333B07EE903AF8EEE77A5E
:10D8600087EEA67A82ED007A704700BFB877012074
:10D870000000C842014B1B6C5B681847B877012059
:10D88000024B08301B6C9B68184700BFB87701201B
:10D89000007970470079C0F3401070470079400963
:10D8A00070477047704703685A1C026019707047D0
:10D8B00003690133012B036106D1002380ED010AC6
:10D8C00080ED000A8360704790ED006A07EE903AA1
:10D8D00070EE466AF8EEE77A86EEA77A77EE067A79
:10D8E00090ED027A30EE670AC0ED017AC0ED007A61
:10D8F000A6EE807A80ED037A80ED027A70470368A5
:10D900005A1C02601970704790F83C20034602F0E0
:10D91000FF0012B1002283F83C2070474FF40063EF
:10D92000838170474FF4006383817047064A042364
:10D93000002110B552F8044B844208BF42F8041C81
:10D94000013BF7D110BD00BFFC77012001207047DB
:10D9500001207047012070472DE9F8435F4F1546BD
:10D960000E467C6DB7F85820B7F85E90C2EB2413D2
:10D970005200C2EBE402B7F95A40624303FB03F4DE
:10D98000B7F95C3024135C43B7F96230A4134FEA53
:10D99000E37804EBE224A4F5FA313C6781FB01CE85
:10D9A00003FB0EF20CFB0822A3FB0C389044B7F9E2
:10D9B00060201B0A82FB010243EA0863120342EA69
:10D9C000105200031B184FF0000042EB2822A3FB6B
:10D9D000093802F5004209FB02884FEAE8734FEA72
:10D9E000680253EA68086CD0B7F968904FEAE978A2
:10D9F00009FB0EFE0CFB08EEA9FB0C9CE644B7F9F4
:10DA000066C08CFB01814FEA414C4FEA48414CEA29
:10DA1000D83C11EB0909796F4EEB0C0CC1F5801E57
:10DA200010EB0900B7F964100EF000480CEBC101CF
:10DA300048EA5E084FEACE7EBEEB000068EB010CC0
:10DA400040F63548A0FB080108FB0C114AF002F82B
:10DA5000B7F96E304FEA613E80464FEA503C03FB17
:10DA60000EF24FEAE3794CEAC14C0CFB0929A3FB07
:10DA70000C324A4403FB0EFE0CFB02EEB7F96C209D
:10DA8000A3FB0C3C4FEAE279E6445B0E43EACE137B
:10DA900013EB000C02FB01F3A2FB082841EB6E6EB6
:10DAA00009FB0031D00CB7F96A30414440EA4130FB
:10DAB0001CEB00004EEBE141000A40EA016000EB84
:10DAC00003100EB1000A306025B104EB84048034E9
:10DAD00024122C600120BDE8F88300BFB877012034
:10DAE000F0B50D4B04460D4EB34201D30020F0BDFE
:10DAF000587988420DD11D79A54200D04CB9D8790A
:10DB0000904206D118680779AF4202D105689D425C
:10DB1000EDD00C33E8E700BFE801000898030008E7
:10DB2000B0F90000084B4143994208DBB1F5000F02
:10DB300007DA0029B8BFFF31081200B27047034866
:10DB4000FBE747F6FF70F8E701FF7FFF0080FFFF6C
:10DB500001207047054B002201209A67DA67C3F85D
:10DB600080200022C3F88420704700BFB8770120CE
:10DB7000104B1A68104BD3F88410521AFA2A16D890
:10DB8000D3ED1E7AFDEEE77A17EE902AD3ED1F7AD9
:10DB9000FDEEE77AC28617EE902AD3ED207AFDEEED
:10DBA000E77A028717EE903A4387012070470020FA
:10DBB000704700BF88330120B877012012B10B0EE7
:10DBC00000F8013B0B0C817003700B0A4370704727
:10DBD00000487047E014012010B50446901C8842AC
:10DBE0009DBFA354A4189DF808306FF0004098BF63
:10DBF000637010BD012070470120704701207047FD
:10DC000001207047012070470120704701207047B4
:10DC100030B5094A0546052400201368AB4205D1FA
:10DC2000D3688B421EBF431CD160D8B2013C02F1C5
:10DC30001402F2D130BD00BF0C0401202DE9F041E7
:10DC40000C4D0127DFF830802C686B691C400CB943
:10DC5000BDE8F081B4FA84F3C3F11F0307FA03F6B9
:10DC600008EB8303D3F8880024EA06040368984786
:10DC70006E61ECE7003C0140B87701200C4B10B519
:10DC80000C4C1B68D4F8C8001B1AFA2B06D90420C8
:10DC900019F06CFE002084F8CC0010BD11B1D4F84E
:10DCA000D0300B6012B1D4F8D43013600120F4E707
:10DCB00088330120B877012008B5006848F09FFB41
:10DCC000014B1860012008BDB877012008B5006835
:10DCD00048F095FB014B5861012008BDB877012041
:10DCE000024BD3F8D80006F089BC00BFB8770120FA
:10DCF00003682DE9F04113440446406883421AD872
:10DD00000D468E18002704F10C08B542606901D158
:10DD1000BDE8F08123695A1C23442261042A15F8C6
:10DD2000011B1973F1D118B941462046FCF72AFFAF
:10DD3000C4E90470E9E74FF0FF30E9E707B58DF873
:10DD40000700012305480DF107020021D0F8DC008F
:10DD500048F020FB03B05DF804FB00BFB87701205A
:10DD600013B50C4C94F8E00068B10523D4F8DC003E
:10DD70006A4601A9ADF80030022348F00BFB9DF87C
:10DD8000050000F0010084F8E00080F0010002B01E
:10DD900010BD00BFB877012038B558B9094BD3F88A
:10DDA000E440094DFFF7DCFF40B1064B0022C3F809
:10DDB000E42006E0044B1C680444F2E72B689C4214
:10DDC000F0D838BDB87701208833012010B5002085
:10DDD000FFF7E2FF80B10620084CFFF7AFFF0123F9
:10DDE000C72084F8E030FFF7A9FF054B1B6803F557
:10DDF000A4430833C4F8E43010BD00BFB877012055
:10DE000088330120F0B5044689B000200F4615463E
:10DE1000FFF7C2FF58B30620164EFFF78FFF01230E
:10DE200096F8E8200DF1010086F8E0300223CDF8E5
:10DE30000CD0009300239A428DF80430029314BF53
:10DE400005210421CDE904132146CDE90675FFF72C
:10DE5000B5FED6F8DC000379022B02D102A946F008
:10DE6000F7F8054B2C441B680633C6F8E43020460F
:10DE700009B0F0BDB877012088330120F0B5054620
:10DE800089B000200E461446FFF786FF002308B332
:10DE90000322114F0DF101008DF80430009297F824
:10DEA000E82002939A42CDF80CD014BF052104213A
:10DEB000CDE904162946CDE90634FFF77FFED7F8F1
:10DEC000DC000379022B02D102A946F0C1F82046FA
:10DED00009B0F0BD0446FAE7B877012073B50546EE
:10DEE0000020FFF759FF18B30620124CFFF726FF5A
:10DEF0000123002694F8E82084F8E030D82329464E
:10DF00000DF1010000938DF80460FFF757FEB24257
:10DF100031466A46D4F8DC0014BF0523042348F0D8
:10DF200039FA054B1B6803F59C530833C4F8E430F9
:10DF300002B070BDB87701208833012010B50A4CBB
:10DF400003210A4AD4F8EC00FDF7A0FCD4F8EC0059
:10DF50000021FDF7ADFDD4F8EC0040F62B4204495A
:10DF6000BDE8104045F056B9B8770120009F240065
:10DF700080AF012010B5114C6421114AD4F8EC0097
:10DF8000FDF784FC0021D4F8EC00FDF791FDD4F8F6
:10DF9000EC00FDF7DDFED4F8EC3002221B685B6874
:10DFA000196883F83D200A6842F001020A600122E4
:10DFB00083F83D2084F8F02010BD00BFB877012021
:10DFC000009F240013B5044601A90120FEF7D0F8F4
:10DFD000012022F0A3FF58B123799DF805209A4231
:10DFE00002D1012002B010BD9DF804209A42F8D061
:10DFF000022001A9FEF7BCF8022022F08FFF40B1F9
:10E0000023799DF805209A42EBD09DF804209A428E
:10E01000E7D0032001A9FEF7ABF8032022F07EFF32
:10E0200040B123799DF805209A42DAD09DF804206A
:10E030009A42D6D0042001A9FEF79AF8042022F0D3
:10E040006DFF40B123799DF805209A42C9D09DF813
:10E0500004209A42C5D0052001A9FEF789F80520C1
:10E0600022F05CFF40B123799DF805209A42B8D098
:10E070009DF804209A42B4D0094B1B68DB0308D5F5
:10E0800000211820FDF7FCFC18B1226803689A42B1
:10E09000A7D02079313801288CBF00200120A1E7CA
:10E0A000000000202DE9F84F394D4FF0000B0646D7
:10E0B000384FAA465C46A946DFF8E080DAF800103F
:10E0C000002357F83320914241D1DBB2434493F807
:10E0D000F130012B40D0022B49D05046FFF772FFA0
:10E0E00078B9142303FB0B93D96801F00C03042BBC
:10E0F00007D10134DAF80000FFF78AFDE4B20444E6
:10E10000E4B20BF1010B0AF1140ABBF1050FD5D1F2
:10E11000214F2846FFF756FFA0B9E9684B0711D5F4
:10E1200001F00C03042B0DD0A64229D921F00801DF
:10E130000134286841F00401E4B2E960FFF768FDAA
:10E140000444E4B21435AF42E3D1BDE8F88F0133A3
:10E150000E2BB6D1FF23B9E7DAF80C301907BCD57E
:10E1600023F0080343F00403CAF80C30B5E7DAF8EB
:10E170000C305A07B1D523F0040343F00803F3E74A
:10E1800021F004012868E960FFF742FDDAE700BFEB
:10E190000C0401208804060870040120B8770120CF
:10E1A000DFED0A7AB7EE007A0023C0ED020A20EE16
:10E1B000270A0360C7EE007AC0ED017A70EEA77AF5
:10E1C00080EEA77A80ED037A704700BFDB0FC9406D
:10E1D0004A09012301F01F0103FA01F150F822302E
:10E1E0000B4340F8223070474A09012301F01F0118
:10E1F00003FA01F150F82230194214BF0120002027
:10E2000070474A09012301F01F0103FA01F150F898
:10E21000223023EA010340F82230704730B54D091F
:10E2200002444FF0FF3300EB8504A24223D901F0F2
:10E230001F018B4050F825100B4093FAA3F3B3FA5B
:10E2400083F3DBB2202B02D003EB451030BD211D40
:10E2500091420C4602D34FF0FF30F7E704312368B8
:10E2600093FAA3F3B3FA83F3DBB2202BF0D0201A96
:10E2700003EBC000EAE71846E8E780EA012008233C
:10E2800041F2210210F4004F4FEA400018BF504005
:10E29000013B80B2F6D1704738B50C468D18AC42C0
:10E2A00000D138BD14F8011BFFF7E7FFF7E770B5A1
:10E2B000124C0122124E00201249FFF7EDFF228876
:10E2C00062B1A31DB34217D2A518B54214D2052AD4
:10E2D00012D921462C46FFF7DFFFF0E72146022244
:10E2E000FFF7DAFF63880849C31A084A641A5842DC
:10E2F000A2F80041584170BD0020FCE70140000831
:10E300000080000800400008FC3F0008B8770120AA
:10E310004840082310F0800F4FEA400018BF80F0FB
:10E32000D500013BC0B2F5D1704710B50A440C4688
:10E33000944200D110BD14F8011BFFF7E9FFF7E785
:10E3400038B50A46044605680020AA4203D36B1C70
:10E350002360287038BD12F8011BFFF7D9FFF4E7DE
:10E3600090ED017AD0ED007A30EE877AC0ED020AA6
:10E37000C0EE876A30EE677AE6EE877AB0EE670A1B
:10E38000C0ED007A7047012303700023C3648364E7
:10E390000365036443644365836283657047DFED0F
:10E3A000157A80ED010AF4EEE70AC0ED020A80ED6D
:10E3B000031AC0ED051AF1EE10FA18DDB4EEE70A03
:10E3C000F1EE10FA10DD81EE007AC0EE207AF0EE68
:10E3D000006A77EE877A86EEA77A80ED047A80ED80
:10E3E0000F2AC0ED0E2ACEE700230361F7E70023D2
:10E3F0008360FAE7BD378635FDEEC07A17EE903AB6
:10E400002033402B43D8DFED237A9FED237AB4EEFF
:10E41000E70AF1EE10FA28DCDFED207A9FED1E7A94
:10E42000B4EEE70AF1EE10FA22D4DFED1D7AB4EE75
:10E43000E70AF1EE10FA1EDD30EE670A37EEC00A89
:10E4400060EE007ADFED176A9FED177AA7EEA67AE5
:10E45000DFED166A20EE276AE7EE876A9FED147AF1
:10E46000A7EEA67AA6EE070A704730EE470ACEE777
:10E4700030EE070AD4E79FED0F7AB4EEC70AF1EE4B
:10E4800010FA44BF30EE270A37EE400AD8E79FED76
:10E490000A0A7047DB0F4940DB0FC940DB0F49C058
:10E4A000DB0FC93F9A7C2E36FAAF4FB93587083C4F
:10E4B000A4AA2ABEDB0FC9BF00000000DFED027A6C
:10E4C00030EE270A98E700BFDB0FC93F38B51D467D
:10E4D000304BB0EE405A0024F7EE005AB3FBF2F393
:10E4E00099424FD207EE901A9FED2B7ADFED2B6AFF
:10E4F000F8EE677A67EE877A07EE102AB8EE477A69
:10E5000027EE267AC5EE876A87EEA64AB0EE440A61
:10E51000FFF772FFF0EE404AB0EE440AFFF7CEFF7D
:10E5200035EE055AF0EE407A012DB8EE000A84EE81
:10E53000854A19BF35EEE76AF6EE006AF0EE656AC5
:10E5400027EE806A18BF66EE266A67EE807A34EEA0
:10E55000257A75EEC45A86EE875AC6EE076A80EDB4
:10E56000005A80ED025AC0ED016AC7EE876AC5EE17
:10E57000877AC0ED036AC0ED047A84614461046265
:10E58000C46138BDC0ED005A44608460C460046159
:10E59000F3E700BF20A10700DB0FC940BD37863578
:10E5A00000239FED010A91E7F304353FF0EEE06AA6
:10E5B000B0EEC07AF0EE405AF4EEC76AF1EE10FA0F
:10E5C00036FE876AB5EE406AF1EE10FA44D0F4EEFA
:10E5D000C76AF1EE10FA54BFB0EE475AB0EE665A71
:10E5E000C5EE067A9FED1E6A9FED1E5ADFED1E4AAC
:10E5F000A7EE865A9FED1D6AF4EEC76AF1EE10FA97
:10E60000F5EEC00AA5EE276A9FED195AA6EE275A25
:10E610009FED186AA5EE276A9FED175AE7EE854A27
:10E62000B7EE005AA4EEA75AF1EE467A87EE850AB5
:10E6300044BFDFED127A37EEC00AF1EE10FAF5EEC4
:10E64000C05A44BFDFED0E7A37EEC00AF1EE10FA81
:10E6500048BFB1EE400A7047DFED0A7AC2E700BF5B
:10E6600039094E3DE3B59EBE69A2163E88FA16BE34
:10E6700045FE7FBFA7DFA8B499FB243FDB0FC93F4E
:10E68000DB0F49400000000044F25063984203DD74
:10E69000A0F50C40A0387047034B9842BCBF00F572
:10E6A0000C40A030704700BFB0B9FFFF48F69F4351
:10E6B000984203DDA0F50C40A03870470028BCBF8D
:10E6C00000F50C40A030704791ED005A08B5B0EE4F
:10E6D000450AFFF7F3FEF0EE405AB0EE450AFFF7A9
:10E6E0008BFE91ED015AF0EE404AB0EE450AFFF77D
:10E6F000E5FEF0EE403AB0EE450AFFF77DFE91ED03
:10E70000023AB0EE405AB0EE430AFFF7D7FEB0EE41
:10E71000404AB0EE430AFFF76FFE25EE806A63EED3
:10E72000C07A80ED025A24EE847A25EE843AC0ED58
:10E73000017AF0EE467A64EE806A23EE844AE5EED2
:10E74000077AA5EE067A64EEE34A80ED004A65EEAC
:10E75000A35AC0ED054AC0ED037AF0EE437A80ED8E
:10E76000077AC0ED085AE5EE667AE5EE436AC0ED39
:10E77000047AC0ED066A08BD034600F1400100229C
:10E780001A6110335A609A60DA609942F8D1102207
:10E79000002150F0E7BD91ED007AD0ED047AE7EE6C
:10E7A000077AC0ED047AD0ED057AD1ED006A91EDDB
:10E7B000017AE6EE877AC0ED057AD0ED067AD1EDE2
:10E7C000006A91ED027AE6EE877AC0ED067AD0ED26
:10E7D000077A91ED007A77EE877AC0ED077AD0ED6F
:10E7E000087AD1ED016A91ED007AE6EE877AC0ED04
:10E7F000087AD0ED097A91ED017AE7EE077AC0ED5B
:10E80000097AD0ED0A7AD1ED016A91ED027AE6EE4D
:10E81000877AC0ED0A7AD0ED0B7A91ED017A77EE26
:10E82000877AC0ED0B7AD0ED0C7A91ED007AD1EDBC
:10E83000026AE6EE877AC0ED0C7AD1ED026A91EDBC
:10E84000017AD0ED0D7AE6EE877AC0ED0D7AD0ED43
:10E850000E7A91ED027AE7EE077AC0ED0E7AD0EDEE
:10E860000F7A91ED027A77EE877AC0ED0F7AD0EDCC
:10E87000107A91ED007A77EE877AC0ED107AD0EDBC
:10E88000117A91ED017A77EE877AC0ED117AD0EDA9
:10E89000127A91ED027A77EE877AB7EE007AC0EDC0
:10E8A000127AD0ED137A77EE877AC0ED137AD1ED34
:10E8B000017AD1ED006A67EEA77A91ED027AE6EE71
:10E8C000A67AE7EE077A90ED007AA6EEA77A80EDB9
:10E8D000007A90ED017AD1ED016AA6EEA77A80ED7B
:10E8E000017A90ED027AD1ED026AA6EEA77A80ED68
:10E8F000027A90ED037A77EE277AC0ED037A7047BB
:10E900002DE9F043034685B000F1100705460026C7
:10E910001C46AC4612E0F8EC016A1EED047AD4ED18
:10E92000007AE6EEC77AC4ED007A98450EF1100E33
:10E93000F1D104340CF1040CBC4203D0A7F110084F
:10E94000E646F2E701361C46B646BEF1040F1FD07C
:10E9500000EB0E1CA84604F1100909E0FCEC016A6A
:10E9600018ED047AD4ED047AE6EEC77AC4ED047AA1
:10E97000CC4508F11008F1D1D4ED046A0EF1010E76
:10E9800093ED007AC6EE877AC4ED047A6446DCE73C
:10E99000042E03F1140305F1040507F11007B7D1A4
:10E9A00000236C46142700930193029303930023E2
:10E9B00052F8045B07FB030C6E4644F8045B00EB63
:10E9C000031565451FD10133042BF1D104AD10317E
:10E9D00000F1400255F8044D0E4600EB031741F8D4
:10E9E000044D1446A742D1ED007A17D152ED016AC9
:10E9F000013BA2F1140287EEA67A81ED007AE9D1FB
:10EA000005B0BDE8F083B6EC017A54ED017AF5EC7F
:10EA1000016AE6EEC77A44ED017AD2E7F4EC016AC6
:10EA2000B6EC017AE6EEC77AC1ED007ADAE700F1DA
:10EA30000C039FED0B7AF0EC017AF4EE677AF1EEBD
:10EA400010FA06D7F0EEE77AF4EE477AF1EE10FA14
:10EA500003DC9842EFD1012070470020704700BFCF
:10EA6000FFFF7F7F1FB50C46024669461030FFF757
:10EA700047FFB6EE007ADDED007A204667EE877A32
:10EA8000C4ED007ADDED017A67EE877AC4ED017A94
:10EA9000DDED027A67EE877AC4ED027AFFF7C7FFF1
:10EAA00004B010BD60EEA00A20EE400A70EEA00A8D
:10EAB000C0EE200A9FED010A4BF0C0BD54F82D4076
:10EAC000B5EEC00A08B5F1EE10FA06DB4BF014FE05
:10EAD000B4EE400AF1EE10FA01D79FED010A08BD2D
:10EAE00000000000F8B504461C30254604F164021D
:10EAF0002DED028B50ED017AB1EC010A77EE807AB0
:10EB000040ED017AFEF7D4FE18309042F2D123692D
:10EB10002B4E01336268236133689B1AA2689342CB
:10EB20002BD904F130079FED278AEB6A012BC5BF73
:10EB300003F1FF3395ED0A7AB0EE480A07EE903AFA
:10EB4000C4BFF8EEE77A87EE270AFFF7B9FFBD42A8
:10EB5000D4ED057A14D01835F4EEC07AF1EE10FA3F
:10EB6000E3D5237B4BBB3268236162600022E36202
:10EB7000A26122636364A264E365BDEC028BF8BD0D
:10EB8000F4EEC07AF1EE10FAEBD4D4ED047A02235D
:10EB9000D4ED066AF8EE677A86EEA77AD4ED0C6AB1
:10EBA00084ED067A86EEA77AD4ED126A84ED0C7AAB
:10EBB00086EEA77A84ED127A00E003232370DCE767
:10EBC000883301200000000038B503780446012B8B
:10EBD00039D10369244D1BB942680AB92A684260D9
:10EBE000D4ED067A013304F11C0077EE807A2361BC
:10EBF000C4ED067AFEF75CFE62682B689B1AA26879
:10EC0000934220D9E36A012BC5BF03F1FF3394ED92
:10EC10000A7A9FED160A07EE903AC4BFF8EEE77A3B
:10EC200087EE270AFFF74CFFD4ED057AF4EEC07AA1
:10EC3000F1EE10FA0BD5237B33B92A6823616260A9
:10EC40000022E362A26138BD03232370FBE7D4ED09
:10EC5000047A0223D4ED066AF8EE677A86EEA77A84
:10EC600084ED067AF1E700BF883301200000000040
:10EC700008B52DED028BF0EEC08AB0EE408AB7EEFB
:10EC8000000A30EE680AFFF71BFF9FED0E7ADFEDFA
:10EC90000E7AB5EEC08AE8EE877A9FED0C7AF1EE37
:10ECA00010FAA7EEA87ADFED0A7AE7EE287ABDEC33
:10ECB000028B20EE270A44BFDFED067A37EEC00A4A
:10ECC00008BD00BF306E99BC2716983D843459BEEC
:10ECD000A40DC93FDB0F494060EEA00AE0EE000A38
:10ECE000B0EE600AECE660EEA00AE0EE000AE1EEAB
:10ECF000010AB0EE600AE3E670B52DED028B82B03A
:10ED00000E46154640F09EFB002869D0364B374C26
:10ED10005B6894F8022103F00203002A45D0002B1F
:10ED200059D00DF1060021F00BFA314ABDF806303A
:10ED3000F0EE405AD2F8EC1302F580629FED2D7A86
:10ED40005B1A07EE903AF8EEE77A87EE870ADFED76
:10ED50002A7A20EE270AFFF7B1FB92ED008AA0EE97
:10ED6000658A3AF0D1FAD4ED430AD0ED057A70EE17
:10ED7000A70AB0EE480AFFF7AFFF7EB120EE000A07
:10ED8000DFED1E7A9FED1E7A20EE270AC0EE077A8D
:10ED90009FED1C7A77EE877AC6ED007A0DB11A4B9B
:10EDA0002B6002B0BDEC028B70BDA3B1B4F932315F
:10EDB00001EE103AB4F9303100EE903AB4F92E3148
:10EDC000B8EEC11A00EE103AF8EEE00AB8EEC00A4A
:10EDD000FFF789FFD1E7D4F8483193ED340ACCE747
:10EDE0009FED0A0AC9E700BF00000020B8770120A4
:10EDF00030E001200000C84235FA8E3CCDCC9C3F6B
:10EE000000409C4682E6C547331390430000000053
:10EE10002DE9F74F90469DF8302005460F46002A11
:10EE20000D9A14BF4FF030094FF020091C1EBABFD5
:10EE300064420123002312F8011B01B12CB9A24640
:10EE400063B100240D9EA41B12E0013CF3E7BD4218
:10EE500004D2494628460193C047019BBAF1010AF2
:10EE6000F5D2EFE7BD4203D228460193C047019B8C
:10EE700006EB040B16F8011B0029F3D133B15446FD
:10EE8000002C07DCBAF1000FA8BFD344584603B0EA
:10EE9000BDE8F08FBD4202D249462846C047013C3A
:10EEA000EEE70FB437B506AB0A4D53F8042BD5E99E
:10EEB0005301019345F0D6FD0446D5F8D80005F07E
:10EEC00000FC0028F9D0204603B0BDE8304004B073
:10EED000704700BFB87701200EB403B503AB0849F3
:10EEE00053F8042BCDE9003001A845F0BBFD019B90
:10EEF00000221A7002B05DF804EB03B0704700BF47
:10EF0000FFD800080CB430B52C4CA5B0D4F854315F
:10EF10001BB9D4F85831002B39D094F85C319942A0
:10EF200006D9012303FA00F0D4F8603118422ED03C
:10EF3000234B04A819684FF47A73B1FBF3F203FB77
:10EF400012132049FFF7C8FF04AB289A0546034473
:10EF50001D4903A8039329AB029345F083FD039B4E
:10EF60000246D4F85401591C03910A211970039BDD
:10EF7000591C03910021197090B103681B6A03B1F9
:10EF80009847D4F8545104AC14F8011B21B925B0AA
:10EF9000BDE8304002B07047284605F02FFBF3E78C
:10EFA000D4F85831002BF2D002212A44FD200A4423
:10EFB000009104A923F054FCE9E700BFB8770120D1
:10EFC0008833012074B10608A7D8000810B54FF4A3
:10EFD000004086B021F0F2FD044690B34FF40041AA
:10EFE00021F04EFF02281AD1226848F201039A420A
:10EFF00027D14FF4004043F097FC10B31F4BD3F8D8
:10F00000642182421FD0D3F84022904230D0D3F8FE
:10F010001C2390422FD00022C3F8582111E0002376
:10F02000022294F904004FF40041CDE901234FF48A
:10F03000612200921A4621F07AFF104BC3F8540166
:10F0400028B906B010BD03F5B272C3F858210C4BB5
:10F0500002210C4A002004930B4B03930B4B0293A9
:10F060000B4B01930B4B00930B4BFFF74BFFE8E768
:10F0700003F51072E9E703F54772E6E7B877012078
:10F0800080B10608E8C1060889B1060892B10608F1
:10F090009EB10608A4B106087BB00608174A0330E3
:10F0A00038B5D2F8F84304EB9003B3F5007F18D8D5
:10F0B00002F57F75C2F8F83302EB810220F00300FD
:10F0C000C3F5007305EB8404D2F8FC1B9B000844D5
:10F0D0000421C2F8FC0B0020094AFFF713FF204669
:10F0E00038BD0021074A00240846FFF70BFF064AF7
:10F0F000936843F000739360F1E700BFB877012095
:10F10000B7B10608DBB10608000000202DE9F04386
:10F11000062587B092F9007014466B4312F80580FB
:10F12000A0EB070C02EB05090635A0EB080E16460E
:10F13000BEF1000FB8BFCEF1000EBCF1000FB8BF9A
:10F14000CCF1000CE645BCBF4FFA88F74C46AB4209
:10F15000E4D11A443378BB420CD1658873884D1BC7
:10F16000CB1A002DB8BF6D42002BB8BF5B429D4249
:10F17000C8BF34460636B242ECD16379084A0493DC
:10F1800023790393638802932378CDE90013034620
:10F1900003210120FFF7B6FE204607B0BDE8F0834B
:10F1A000E9B106084B1EDBB2062BF0B594BF1C4A32
:10F1B0004FF480721B4C87B098BFD25C04F15803A7
:10F1C000002808BF1C46234613F9087B1888C8B9D5
:10F1D000154B93F8840CA3790593A3880493A37823
:10F1E0000393238800910321CDE901230F4A104B9B
:10F1F000002808BF13460F4A0120FFF783FE204670
:10F2000007B0F0BD161AD51B002EB8BF7642002DF0
:10F21000B8BF6D42AE42BCBF1C4647B20833D5E70B
:10F220008C110608F0140120B8770120130007089C
:10F2300057C6060822B2060803685A1C02601970F5
:10F24000090A03685A1C02601970704703685A1C47
:10F250000260197003685A1C02600A0A1A70036877
:10F260005A1C02600A0C090E1A7003685A1C0260CC
:10F270001970704703685A1C02600A0A1A70036802
:10F280005A1C02601970704738B50446006815466C
:10F2900050F068F823682B44236038BD38B5044625
:10F2A000006815464DF0B6FE23682B44236038BD38
:10F2B00003685A1C02601878704703685A1C026081
:10F2C0001A4612F8021B0260587841EA0020704783
:10F2D00002681146531C10B50360D31C11F8024B91
:10F2E00001605178036093781B0443EA0123111DE8
:10F2F00023430160D07843EA006010BDD1E90032B9
:10F300009A4206D05A1C0A6008B11B78037001208B
:10F31000704700207047D1E9002310B59B1A0446BE
:10F320000846012B04DDFFF7C8FF2080012010BD37
:10F330000020FCE730B50A440446914201D1002088
:10F3400011E014F8013BA3F14100192811F8010B59
:10F35000A0F1410598BF2033192D98BF20301B1A0A
:10F3600002D10028E9D130BD1846FCE76FF0004219
:10F37000E0E7028810B5A2F5FA62C37840F2B5540E
:10F380009108013B02F0030204FB013381780C2455
:10F39000013904FB02120C49847901EB4202182165
:10F3A00012891344027901FB03223C21437900892D
:10F3B00001FB0233054A224401FB03224FF47A7316
:10F3C0000021C2FB030110BD8C11060880436D387B
:10F3D0002DE9F04190461F4605464FF47A7200230E
:10F3E0004046394648F036FB274B3C21034493FB0B
:10F3F000F1F201FB1233AB7192FBF1F301FB13222B
:10F4000040F2B5516A71182293FBF2F402FB1433F7
:10F4100094FBF1F201FB12442B719300B4F5896F58
:10F420002DDA40F2DA2294422BDCB4F5B77FB4BF78
:10F4300000210121154A18200B2600FB012232F879
:10F440001600A04201DD013EF9D103F5FA63013453
:10F450004FF47A7240460B442B80731CAB700C2324
:10F4600003FB01660A4B394603EB46063389E41A6F
:10F470000023EC7048F0EEFA2A81BDE8F081032108
:10F48000D8E70221D6E700BF80BC92C794110608D6
:10F490008C110608F0B5274D8DB006460F466C4618
:10F4A0000FCD0FC40FCD0FC495E80F0084E80F00F7
:10F4B00016F0030339D1642196FBF1F201FB1262CD
:10F4C00042B94FF4C87296FBF2F302FB1363003BA0
:10F4D00018BF0123721EC3F11D0369460024002AD0
:10F4E000019340F26D131046B8BFB01C072573435B
:10F4F000013F03EBA0006FF0630392FBF3F31844AA
:10F500004FF4C87392FBF3F21044063051F8042B09
:10F51000A74202EB000393FBF5F0C0EBC000A3EBA6
:10F52000000004D1101A0DB0F0BD0123D2E7013460
:10F53000ECE700BFF4110608084B53E9021251EA48
:10F54000020308D0064B1B685B1842F10002C0E9B9
:10F550000032012070470020704700BF488401201E
:10F560008833012037B505466846FFF7E5FF0446B6
:10F5700038B12846DDE90023FFF72AFF204603B013
:10F5800030BD40F201132880A8806B80A8712881CB
:10F59000F4E71FB50190FFF7E5FF0199044648B174
:10F5A000064B0DF10E020846B3F8903CADF80E3054
:10F5B00042F0AAFC204604B010BD00BFB87701207D
:10F5C000F0B50124B0FBF4F58D4203D200261CB93E
:10F5D0001C70F0BD4C43F5E7B0FBF4F5B4FBF1F75C
:10F5E00004FB15002EB9002D03DC8C420CD33C46E5
:10F5F000EDE7092D08DD002A14BF372457242C44D9
:10F60000013603F8014BF2E73024F8E7A0F13003AC
:10F61000DAB2092A01D818467047A0F16103052B18
:10F6200001D857387047A0F14103052B94BF3738F4
:10F630004FF0FF30704770B50446154608469442B7
:10F64000B4FBF2F602D33046FFF7F5FF05FB164494
:10F65000024B1B5D00F8013B70BD00BF6CB2060899
:10F66000B5EEC00ADFED2D7A0023F1EE10FA30B5C9
:10F67000C8BF30EE270A87B0D8BF30EE670ADFED8B
:10F68000287A054603A9029320EE270ACDE9003324
:10F69000FDEEC07A17EE904A84EAE470A0EBE470C5
:10F6A00043F03CFF002C03A8ACBF20232D238DF892
:10F6B000003047F0A7FB012822D130238DF801301C
:10F6C0008DF802308DF8033003A9684650F09AFD9A
:10F6D000684647F097FB03386946C4B2284622467D
:10F6E0004DF098FC00230F4928462B5550F08AFD19
:10F6F0000DEB0401284650F085FD284607B030BDCB
:10F70000022805D130238DF801308DF80230DBE777
:10F71000032804BF30238DF80130D5E76F12033A78
:10F7200000007A4414E5060830B50278034601303B
:10F73000202AFAD0092AF8D02D2A4BD1BFEE000A90
:10F740000346F2EE046A1A469FED3B7A134612F81E
:10F75000010BA0F13001CCB2092C41D92E280BD1DC
:10F76000F2EE046A1146B0EE666A0B4611F8012B00
:10F77000303AD0B209283CD91A7802F0DF02452A83
:10F7800054D15A782D2A3FD102330120013B002267
:10F790000A2513F8011F3039CCB2092C3BD9B2F538
:10F7A0009A7F1346F7EE007ADFED246A28BF4FF404
:10F7B0009A731A46072A31D8DA086FF00701F2EE79
:10F7C000046A01FB02336BBB90B3C7EE276A20EEDD
:10F7D000260A30BDB7EE000A2B2A08BF0346B0E761
:10F7E00007EE901AF8EEE77AE7EE267AB0EE677A3F
:10F7F000ACE707EE902AF8EEE77AC7EEA65A66EE77
:10F80000866A37EE257AB0E72B2A4FF0000014BF46
:10F8100001330233BAE705FB0212BAE767EEA67AB4
:10F82000083AC7E767EEA67A013BCCE7F7EE007A25
:10F8300067EE276ACBE700BF0000000020BCBE4C8B
:10F8400070B5034610F8012B202AFAD0092AF8D007
:10F850002D2A4FF000044FF00A060ABF0346012587
:10F860004FF0FF35591E11F8010FFFF7CFFE0928A1
:10F8700002D905FB04F070BD06FB0404F3E7002386
:10F8800010B5802804D893420AD2C854581C10BD21
:10F89000934205D060F07F04C009CC540133F0E7F7
:10F8A0004FF0FF30F3E72DE9F04F7A4B8FB0DFF8E0
:10F8B000F4814FF00309A3EB0802CDE901231022E4
:10F8C00000210AA84FF04EFD019BCDF81C80099342
:10F8D000029B0893704B1A69002A04DA6F4A5A6037
:10F8E00002F188325A6001244FF0000A7E2304A9F5
:10F8F000224607A88DF83440CDF830A08DF810309E
:10F90000FEF7F6F9504513DA0023B9F1010900F0CA
:10F91000BA80002BD3D098F800307E2B40F0B68010
:10F92000FEF7C5FC002800F0B1800FB0BDE8F08FF5
:10F930002246DFF874B15A4C04A95046FEF7ACFCDD
:10F94000ADF812005C453FD30024022205A907A8A8
:10F95000ADF81440FEF7CCF9A042D5DBBDF812009B
:10F96000022205A9FEF798FC0222ADF812000DF163
:10F97000120107A8FEF7BCF9A042C5DB0B98A0B1A5
:10F98000079B089A03449342BED80AABC0F1040215
:10F99000214618444FF0E6FC0C9818B90AA907A8AC
:10F9A000FBF7F0F800230C900B930C9B002BABDBC8
:10F9B0009DF8342022B138490A6942F000420A61B8
:10F9C000B3FA83F35B09A0E762888DF819A0C2F34C
:10F9D0000B06B31DADF814302388C3F30B011B0BCA
:10F9E0008DF818301304ADF8161020D4062205A99E
:10F9F00007A8FEF77DF9002886DBBDF81200062275
:10FA000005A9FEF749FC3246ADF8120007A8616867
:10FA1000FEF76EF90028FFF677AFBDF81200324608
:10FA20006168FEF739FCADF8120014348AE700274C
:10FA30003D460135062205A907A8EDB28DF81950FB
:10FA4000FEF756F90028FFF65FAFBDF81200062258
:10FA500005A9FEF721FC6168ADF812003246394471
:10FA600007A80391FEF744F90028FFF64DAFBDF853
:10FA70001200324603993744FEF70EFC032DADF811
:10FA80001200D6D1D1E7002B7FF445AF052004F05A
:10FA90003FFF00BF00800008003C02402301674593
:10FAA0003C4007080040000878450708034AD2F8A0
:10FAB000943C1843C2F8940C704700BFB8770120FB
:10FAC000034AD2F8943C23EA0000C2F8940C704731
:10FAD000B8770120034606490648884201D3002032
:10FAE00070470288C2F30B029342F9D01430F4E756
:10FAF000784507083C40070842880B4613B5C2F317
:10FB00000B0204460021184601924FF02BFC21699C
:10FB100003460A48814209D30948019A814205D225
:10FB2000184602B0BDE810404DF074BA21B1184635
:10FB300002B0BDE81040084702B010BD7845070884
:10FB4000374A070810B4B0F902400B464288002C2F
:10FB500041685DF8044BBEBFC2F30B02DBB203FB8E
:10FB60000211C9E730B5094B094CA34200D330BD9F
:10FB7000B3F902205988002A06DA5A68C1F30B014A
:10FB8000DD6800FB01222A601433EEE73C400708E1
:10FB90007845070802460144002030B512F8015BA1
:10FBA000082480EA050340086D0813F0010F1CBF0C
:10FBB00080F08C03D8B2631E13F0FF04F1D18A42A7
:10FBC000ECD130BD144901EB8000406C70B500B33E
:10FBD0000C2202FB001292F9993C581C1AD092F8A0
:10FBE000A10CB0B1C8188C2592F8A04C142290F842
:10FBF000EC6C6B4300201D19013A344401EB4505C0
:10FC0000B5F8F05C10FA85F0F5D11423B0FBF3F0F1
:10FC100080B270BD0020FCE7B877012038B50D46F2
:10FC200003201446FFF7CEFF07EE900A8DB1F8EEE1
:10FC3000677A9FED0A7AF0EE006A67EE877AB8EE8F
:10FC4000047AA7EEA67ADFED067A67EE277AC5ED8D
:10FC5000007A0CB1034B236038BD00BF6740533AB4
:10FC600000007A443313904310B5427A044632B10F
:10FC70000146406851F80A3B98470023637210BD63
:10FC800010B4447A621C0444D2B24272A172037A64
:10FC9000934202D85DF8044BE6E75DF8044B7047E9
:10FCA000036810B51A790446022A02D1987A46F000
:10FCB00097FB00232360237110BD73B50279022ADC
:10FCC00038D190F9103014260320083173430025F1
:10FCD00069448DF80300012419488DF80050C35879
:10FCE0008DF801408DF8022011F8086C15498B42FF
:10FCF00022D0A1F578418B4220D001F580618B4262
:10FD000005D0114A934214BF4FF0FF320322196805
:10FD1000142421F0400104FB02021960D068196824
:10FD200021F0380250F826100A431A601A6842F08F
:10FD300040021A6002B070BD2A46E8E72246E6E7B4
:10FD4000000001200030014000340140C36910B5BB
:10FD5000044623B909211420FFF7A0F9E061E06906
:10FD600010BD10B504460068FFF7F0FF8378CBB1F3
:10FD70008388DBBA07EE903AF8EEE77AC4ED047AAE
:10FD8000C388DBBA07EE903AF8EEE77AC4ED057A5D
:10FD900003890120DBBA07EE903AF8EEE77AC4ED6A
:10FDA000067A10BD1846FCE710B504460068FFF758
:10FDB000CDFF8378CBB1B0F9043007EE903AF8EE7E
:10FDC000E77AC4ED047AB0F9063007EE903AF8EE1F
:10FDD000E77AC4ED057AB0F90830012007EE903AD1
:10FDE000F8EEE77AC4ED067A10BD1846FCE738B5A0
:10FDF00000680D461446FFF7A9FFD0F8013007EE62
:10FE0000103ACDB1D0F80530DFED166A07EE903A22
:10FE10009FED156AF8EE677A77EEE67A77EEA77AC5
:10FE2000C7EE866AF7EE007A76EEE77ADFED0F6AC4
:10FE300067EEE67AC5ED007A9CB1B8EEC77ADFEDE1
:10FE40000C7ADFED0C6A27EE277AC7EE267A9FED53
:10FE50000A7A77EEC77A9FED097A77EE877AC4ED52
:10FE6000007A38BD9AC9CC449AC94C460E76D7451B
:10FE70000000484300E0FF440000484233938843B9
:10FE800037B500680D461446FFF760FFD0F805301F
:10FE90009FED237A07EE903AF8EE677A77EEC77A0D
:10FEA0009FED207A67EE877AB3EE097A67EE877A5C
:10FEB000B2EE047AF4EEC77AF1EE10FA06DCBAEE8E
:10FEC000047AF4EEC77AF1EE10FA0CD517EE900A28
:10FED00047F004F9144ACDE9000104210320FFF79B
:10FEE00011F803B030BDD0F8013007EE103A2DB153
:10FEF000DFED0E6A67EEA67AC5ED007A002CF0D031
:10FF0000B8EE477ADFED0A6ADFED0A7AE7EE267A85
:10FF10009FED097A77EE877AC4ED007AE1E700BFBA
:10FF2000000000460000803891B206080AD77843E6
:10FF30000319C83D000048C23393884310B50068D8
:10FF40000C46FFF703FF83784BB14389222201203F
:10FF5000DBBA93FBF2F303F26D13238010BD184656
:10FF6000FCE70368DB6B13B504462BB923685B6BB6
:10FF70003BB9FF23E38202E098470028F6D102B0A4
:10FF800010BD214601A898470028F2D0BDF80630E0
:10FF9000013B9BB2EEE738B58B68044601600D4625
:10FFA00098470B4B2361002323752B6B13B120461D
:10FFB00098472075074B13F8C03C1BB1237D23F0F5
:10FFC0000103237500232046E382BDE83840C8E7DB
:10FFD0000001FF00B0880120036810B59B6804464B
:10FFE000984701236374FF23A37410BD036810B501
:10FFF00004461B689847236820469B689847E37C23
:020000040801F1
:100000000133E37410BD036810B504465B6898477C
:10001000236820469B689847E37C013BE37410BD4E
:10002000F0B5044685B00D4618461646039346F0D3
:10003000E9FE226828440021E673A073204600915F
:10004000294657693246039BB84705B0F0BD30B525
:10005000046885B0E469089D34B10DB90DF10F0550
:100060000095A04705B030BD2046FBE703685B6AFA
:10007000184703689B6A184710B5037B04460BB109
:10008000437B13B92046FFF7F4FF23682046DB6863
:10009000BDE81040184703685B6C03B11847704710
:1000A00003681B6803B11847704703685B6803B1B6
:1000B0001847704703681B6A03B118477047036805
:1000C0005B6A03B11847704730B40468A46A14B17E
:1000D000A44630BC604730BC704730B40468E46A62
:1000E00014B1A44630BC604730BC704703685B6CF9
:1000F00003B11847704703689B6C03B118477047FA
:1001000003689B6F03B1184770470368D3F88030CA
:1001100003B1184770470368D3F8843003B1184718
:1001200070470368D3F8883003B11847704721B18E
:100130000B68D3F88C3003B118470020704738B5EE
:100140000524094B04FB0030A0F1A005013C15F883
:10015000010B45F045FF14F0FF04F7D12046BDE840
:10016000384045F03DBF00BF2412060810B5441EBC
:1001700014F8010F00B910BDFFF7E1FFF8E7FDF734
:100180005DBDFDF75BBDFDF759BDFDF757BDFDF743
:1001900055BDFDF753BDFDF751BD034B53F8BC0CE6
:1001A00008B1436818477047B0880120034850F8E9
:1001B000BC3C0BB11B6A1847B8387047B0880120A7
:1001C00030B500220624064B04FB02F1CD5C8542CB
:1001D00004D00132092AF7D1002030BD5818FCE7BD
:1001E0000888012070B51A4E36221A4C0021A6F15B
:1001F000A8004FF0B7F8D4F8C8300020984705465B
:1002000008B3C83446F8BC4CFFF7D0FF8368D3B1BD
:1002100004880320FFF7D4FFB8B9013C0220A4B240
:10022000FFF7CEFF50B956F8700C08280BD0431CCE
:10023000062246F8703C084B02FB00300223848003
:10024000037000234380284670BD4488E5E700BF63
:10025000B0880120E01401200888012030B1036833
:1002600082881B691A4214BF01200020704718B110
:100270000268838809B1936170471B04FBE710B1E2
:10028000036882889A61704710B504464FF4FA708B
:1002900004F0AAFA6069BDE81040F0E773B590F980
:1002A000103015461422044653430D4AD65883682D
:1002B0009A0704D44069019146F064F801993046E8
:1002C00046F0DEFA2946304646F0DAFAA3689B0784
:1002D00002D42046FFF7D8FF012002B070BD00BF56
:1002E000000001207FB503790D46012B0AD0022BB7
:1002F00019D18368DB0758BF01F07F0104B0BDE866
:100300007040CBE781688DF80F200DF10F0201F0EE
:10031000010100922A460191417C90F91000FAF700
:1003200025FE04B070BD0020FBE7012258210068C3
:10033000D8E7012248210068D4E73122F42100687F
:1003400008B5FFF7CFFF012008BDF022FF210068AC
:10035000C8E7B422FF210068C4E7CA43006841EA45
:100360000212D221D2B2BDE70A460068A521B9E740
:100370005521F9E79622FF210068B3E70A46006895
:100380008721AFE7C901006801F080027821A9E761
:1003900010B57822044600210068FFF7A3FF05206E
:1003A00004F0A1FA202201212068FFF79BFF05201D
:1003B00004F099FA002202212068FFF793FF6420DD
:1003C00004F091FA012010BD10B524220446412109
:1003D0000068FFF787FF80B1202230212068FFF7F7
:1003E00081FF50B1062231212068FFF77BFF20B149
:1003F000002234212068FFF775FF052004F073FA0E
:10040000012010BD10B5072204460A210068FFF73D
:1004100069FF052004F067FA242241212068FFF7D4
:1004200061FF052004F05FFAC02242212068FFF737
:1004300059FF052004F057FA012010BD10B50446FD
:10044000002221210068FFF74DFFFC2220212068B7
:10045000FFF748FF402224212068FFF743FF0C22CA
:1004600023212068FFF73EFF002222212068FFF7AA
:1004700039FF012010BD10B501220446102100688B
:10048000FFF730FF40B1142004F02DFA2068A022BD
:100490001121BDE8104025E710BD10B5012204462A
:1004A0000B210068FFF71EFF20B11D2209212068E3
:1004B000FFF718FF00F0010010BD10B504469422AC
:1004C0000B210068FFF70EFF712201212068FFF762
:1004D00009FF002204212068FFF704FFC82205213C
:1004E0002068FFF7FFFE002206212068FFF7FAFED2
:1004F000C82207212068FFF7F5FE002208212068A6
:10050000FFF7F0FEC82209212068FFF7EBFE01206B
:1005100010BD044B024653F86C0C08B18021E1E693
:10052000704700BFB088012010B5B0204FF4806440
:10053000FFF7EFFF4020FFF7ECFF0020FFF7E9FF98
:100540001020FFF7E6FF013C002045F049FDA4B272
:10055000002CF8D110BD503910B50446C8B2FFF7D1
:10056000D8FF04EB440004EB4404400000F00E000C
:10057000FFF7CFFFC4F3C300BDE810401030C8E759
:10058000503808B5C0B2FFF7C4FF0020FFF7C1FF25
:100590001020BDE80840BCE7054B002113F8612C92
:1005A00053F8680C02F0F70203F8612C9AE600BFDA
:1005B000B0880120F7B515461E46142290F9103078
:1005C000044653430D4AD75883689A0704D44069B8
:1005D000019145F0D7FE0199384646F051F933466E
:1005E0002A4600213846FBF71BF9A3689B0702D473
:1005F0002046FFF749FE012003B0F0BD00000120B6
:10060000F7B507791646012F0AD0022F15D1846855
:10061000E40758BF41F0800103B0BDE8F040C9E7EE
:10062000826802F00102CDE900620A46417C90F93D
:100630001000FAF79BFC03B0F0BD0020FBE7F7B514
:1006400015461E46142290F91030044653430E4AB4
:10065000D75883689A0704D44069019145F092FE07
:100660000199384646F00CF93346002229463846AF
:10067000FBF7D6F8A3689B0702D42046FFF704FED9
:10068000012003B0F0BD00BF00000120F7B50779DD
:100690001646012F0AD0022F15D18468E40758BFEF
:1006A00041F0800103B0BDE8F040C8E7826802F085
:1006B0000102CDE900620A46417C90F91000FAF788
:1006C00019FE03B0F0BD0020FBE713B50623044676
:1006D0006A461F210068FFF7D9FFD0B1BDF800308E
:1006E000DBBA07EE903ABDF80230F8EEE77ADBBAF3
:1006F000C4ED047A07EE903ABDF80430F8EEE77ADC
:10070000DBBAC4ED057A07EE903AF8EEE77AC4ED6D
:10071000067A02B010BD37B50623F7216A46006895
:10072000FFF7B4FF124C1349D8B19DF801209DF892
:10073000003012019DF8035042EA03329DF8023066
:1007400042EA13129DF804301B014A6743EA05335D
:100750009DF8055043EA15134B6544E9172303B090
:1007600030BD54F85C3C4B6754F8583C4B65F6E799
:10077000B0880120B877012007B5012301AAFF2125
:100780000068FFF783FF03B05DF804FBF7B505468B
:100790000068FFF7DBFA00230446FF2103700423FF
:1007A00028680DEB0302FFF771FF10B9002003B0BA
:1007B000F0BD04236A46FF212868FFF767FF002881
:1007C000F4D09DF804108A09023A012AEED99DF866
:1007D000053043F6FF7503EB0123C3F30D03AB4272
:1007E000E4D0002BE2D09DF8061040F2FF779DF890
:1007F000072002EB0122B7EB521F4FEA6211D5D05E
:100800000029D3D09DF800609DF8012002EB06225C
:10081000C2F30D02AA42C9D0002AC7D09DF80260D7
:100820009DF8035005EB0625B7EB551F4FEA6516FB
:10083000BCD0002EBAD09D1A002DB8BF6D42FF2D3E
:10084000B4DC8D1B002DB8BF6D42FF2DAEDC012541
:10085000134431442B4125702941C4F80530C4F8B4
:100860000110A4E773B505460068FFF76FFA00268C
:10087000042304460670FF210DEB03022868FFF7EE
:1008800005FF48B19DF804108B0907D003200D4ADD
:100890000421FEF737FB304602B070BD9DF80520FD
:1008A0009DF8073002EB01229DF8061003EB0123AF
:1008B000012192B25B112170C4F80520C4F8013007
:1008C000EAE700BFB3B2060838B504460068FFF790
:1008D0003DFA0546C21C0D230C212068FFF7D6FE09
:1008E000A870B8B1B5F90A3007EE903AF8EEE77A99
:1008F000C4ED077AB5F90C3007EE903AF8EEE77AD6
:10090000C4ED087AB5F90E3007EE903AF8EEE77AC2
:10091000C4ED097A38BD13B503230C4601AA222180
:100920000068FFF7B3FE30B1BDF9053003EB830378
:100930001B12E633238002B010BD13B50623044614
:100940006A4625210068FFF7A1FED0B1BDF800304E
:10095000DBBA07EE903ABDF80230F8EEE77ADBBA80
:10096000C4ED077A07EE903ABDF80430F8EEE77A66
:10097000DBBAC4ED087A07EE903AF8EEE77AC4EDF8
:10098000097A02B010BD70B5066805463046FFF71B
:10099000DDF90446021D0E233B213046FFF776FEAB
:1009A000A070B8B1A389DBBA07EE903AF8EEE77A07
:1009B000C5ED077AE389DBBA07EE903AF8EEE77AFD
:1009C000C5ED087A238ADBBA07EE903AF8EEE77AAB
:1009D000C5ED097A70BDF0B5816B85B0514F044605
:1009E00005681023504A90F83500B7FBF1F189B241
:1009F000FEF78CFB4388064600212846B7FBF3F739
:100A00002764FFF75AF980226B212846FFF76AFC1A
:100A1000962003F068FF032268212846FFF762FC56
:100A2000962003F060FF03226B212846FFF75AFC53
:100A30000F20002103F046FF10226A212846FFF70D
:100A400051FC0F20002103F03DFF00226C212846BD
:100A5000FFF748FC0F20002103F034FF72791921C1
:100A60002846FFF73FFC0F20002103F02BFF182240
:100A70001B212846FFF736FC0F20002103F022FF40
:100A800018221C212846FFF72DFC0F20002103F01F
:100A900019FF32791A212846FFF724FC0120002192
:100AA00003F010FF03212846FFF707F9062302AAE7
:100AB00043212068FFF7EAFDD0B1BDF80830DBBA6A
:100AC00007EE903ABDF80A30F8EEE77ADBBAC4EDEB
:100AD000077A07EE903ABDF80C30F8EEE77ADBBA09
:100AE000C4ED087A07EE903AF8EEE77AC4ED097A99
:100AF000D4ED087AFDEEE77ACDED017A9DF9043068
:100B000001330CD1D4ED077AFDEEE77ACDED017A11
:100B10009DF90430013302D1062003F0F9FE05B03F
:100B2000F0BD00BF40420F00C814060813B50446CC
:100B300000686A460379022B4FF006030CBF43217D
:100B40000321FFF7A3FD18B9E086A06302B010BD32
:100B5000BDF800305BBAE386BDF802305BBA63874C
:100B6000BDF804305BBA2387F0E713B506230446CB
:100B70006A4611210068FFF789FD18B9E086A06375
:100B800002B010BDBDF90030F7EE086A07EE103A6A
:100B9000B8EEC77A27EE267ABDEEC77A17EE103A7E
:100BA000E386BDF9023007EE103AB8EEC77A27EEB9
:100BB000267ABDEEC77A17EE103A2387BDF90430C6
:100BC00007EE903AF8EEE77A67EEA67AFDEEE77A5E
:100BD00017EE903A6387D3E7002313B5C386044624
:100BE00083636A46062303210068FFF74FFD78B14F
:100BF000BDF8003003EB4303E386BDF902305B42EE
:100C000003EB43032387BDF8043003EB43036387FF
:100C100002B010BD13B50021044606236A46C18602
:100C200081630068FFF732FD40B1BDF80030E38614
:100C3000BDF802302387BDF80430638702B010BDD1
:100C4000002313B504460093ADF804306A468DF8CE
:100C500006304E2107230068FFF718FDBDF801306C
:100C600001205BBAE386BDF803305BBA2387BDF889
:100C700005305BBA638702B010BD73B590F91030D0
:100C800015461422044653430D4AD65883689A07E2
:100C900004D44069019145F075FB0199304645F057
:100CA000EFFD0123002229463046FAF7B9FDA3687B
:100CB0009B0702D42046FFF7E7FA012002B070BD7F
:100CC0000000012073B503791646012B0AD0022BD0
:100CD00015D18368DB0758BF41F0800102B0BDE841
:100CE0007040CAE7826802F00102CDE900620A465C
:100CF000417C90F91000FAF7FDFA02B070BD0020B7
:100D0000FBE7F8B504460E461546071D3A46FF2197
:100D10002068FFF7D7FF30B116B12379DB07F5D490
:100D20000DB123792B70F8BD00220121E9E710B540
:100D30000446FFF70EFB18B12046BDE81040F3E76C
:100D400010BD10B50446FFF70FFB18B12046BDE8F3
:100D50001040E9E710BD73B50546CDE90023FFF764
:100D6000E6FFA8B12846FFF703FB88B12846FFF746
:100D7000DBFF68B16E46082416F8011B2846FFF712
:100D8000E0FF28B1013C14F0FF04F5D102B070BDC2
:100D90000020FBE7CC21D4E770B506460C468D1841
:100DA000AC4201D1012006E014F8011B3046FFF7E8
:100DB000C8FF0028F4D170BD38B505461446FFF7CA
:100DC000DDFA2846FFF7B0FF20B11CB12B79C3F341
:100DD0004013237038BD10B50446FFF7A8FF38B1A3
:100DE0002046FFF7D7FF18B12046BDE810409BE72B
:100DF000002010BD2DE9F04F002587B080460493F8
:100E00000195CDE90212039B4046EC0003EBC50AB5
:100E1000FFF78DFF024600286CD0002201214046DA
:100E2000FFF76FFF0246002864D098F80430990756
:100E300060D5F0214046FFF784FF0246002859D0D4
:100E4000A4F108024FF0000B0127039B5E461344F8
:100E50003C460593029B002B54D0082C52D804F139
:100E6000FF3943FA09F909F0010949464046FFF7FD
:100E700089FA024600283DD0002201214046FFF7B2
:100E800040FF0246002835D098F8041001F0600CAD
:100E9000C809BCF1600F16D0029B1BB1082C01D809
:100EA000814527D1002841D01AF8061039437F0028
:100EB00001340AF8061017F0FF07E4B2CAD1013670
:100EC000F6B2082E1CD1402C10D9072150460592AD
:100ED000FEF760FE9AF80710059A814206D10135A7
:100EE000EDB2BBF1000F05D0CDF804B0049B1B7828
:100EF000AB4288D8049B10461D7007B0BDE8F08F48
:100F00000127A7E75DB1019BA34208D9059B9A5D24
:100F1000174214BF4FF001094FF00009A5E7019BEC
:100F20001B1BD3F1000949EB03099EE7880940EA3E
:100F3000511111F0010F1AF8061008BFA34621EA5B
:100F40000701B4E7C90138B501F080010446154630
:100F5000FFF718FA08B9002038BD00220121204609
:100F6000FFF7CFFE0028F6D023795B092B70F3E75B
:100F700010B5021D0446FF210068FFF7A3FE18B15B
:100F80002079C04300F0010010BD38B50446154675
:100F900000680A46E121FFF7A5F928B12A46206832
:100FA000FF21BDE838408DE638BD0A46C321ECE795
:100FB00038B5021D0D46F0210446FFF7E6FF08B1E3
:100FC00023792B7038BD0A46E121DEE738B50446A7
:100FD0000D46FFF7CFF940B12046FFF7A5FE20B13F
:100FE00029462046BDE83840EDE7002038BD70B501
:100FF00006460C468D18AC4201D1012006E0214680
:1010000030460134FFF7E2FF0028F4D170BDF7B598
:10101000816B0546664F0F230468664A90F83500D9
:10102000B7FBF1F189B2FEF771F84388064600215B
:101030002046B7FBF3F72F64FEF73FFE0022762130
:101040002046FFF74FF90F224E212046FFF74AF9BD
:101050000F2003F048FC72794F21204602F00F0266
:10106000FFF740F90F2003F03EFC72795021204633
:1010700002F00F02FFF736F90F2003F034FC522183
:10108000FF222046FFF72EF90F2003F02CFC95F8E5
:101090003510072941D0484E96F8840CFEF782F8A7
:1010A0000546012276212046FFF71CF9AA780C217B
:1010B0002046FFF717F92A790D212046FFF712F98C
:1010C000AA79AB880E211201204642EA1322D2B23D
:1010D000FFF708F94FF4807196F8840CFEF762F878
:1010E0000546022276212046FFF7FCF8AA78032164
:1010F0002046520002F0FE02FFF7F4F82A7904219C
:101100002046FFF7EFF8AA79AB88052112012046A7
:1011100042EA1322D2B2FFF7E5F8002276212046F8
:10112000FFF7E0F8032214212046FFF7DBF80F2039
:1011300003F0D9FB002263212046FFF7D3F8642097
:1011400003F0D1FB082265212046FFF7CBF80DF113
:10115000070264212046FFF7B5FD9DF807206421B2
:10116000204622F0100242F060028DF80720FFF7BF
:10117000B9F80F2003F0B7FB0DF106024D21204610
:10118000FFF7A0FD9DF806204D21204602F03F020A
:1011900042F040028DF80620FFF7A4F80F2003F07C
:1011A000A2FB03212046FEF788FD03B0F0BD00BF7F
:1011B00040420F0028150608B8770120F7B51546FC
:1011C0000DF107021C4606460F46FFF77BFD9DF812
:1011D000073005EA0302A24209D023EA0502394694
:1011E0003046224303B0BDE8F040FFF77BB803B0C0
:1011F000F0BD09230C211A4630B5044687B0FFF72D
:10120000DDFF282003F06FFB01AA08212046FFF72D
:1012100059FD9DF904209DF80430002A03DB0025C8
:10122000284607B030BD5D06F9D5122301AA10216A
:101230002046FFF72BFA05460028F0D09DF8052040
:101240009DF804301109120241EA0311DB09544BE5
:1012500002F4706218BFA1F5805110059DF80700D7
:1012600019839DF8061041EA02019DF8082048BF45
:10127000A1F580511201598342EA00329DF809100C
:1012800042EA11101203BDF80A204FEA014148BF9B
:10129000A0F5801052BA01F47021D86192B20A43CD
:1012A000090348BFA2F580121A62BDF80C2052BA99
:1012B00091B21204BDF80E2048BFA1F5803152BA98
:1012C0009984100491B2BDF8102048BFA1F5803177
:1012D00052BAD98491B21204BDF8122048BFA1F5C8
:1012E000803152BA1985100491B2BDF814202046FD
:1012F00048BFA1F5803152BA598591B212044FF01E
:10130000070248BFA1F58031998500230821FFF726
:1013100055FFA5220E212046FEF7E4FF96220F215D
:101320002046FEF7DFFF022262212046FEF7DAFFA9
:1013300000220E212046FEF7D5FF00220F21204675
:10134000FEF7D0FF0223072208212046FFF736FFD1
:10135000282003F0C8FA5423204606211A46FFF736
:101360002DFF0DF1030228212046FFF7ABFC9DF86D
:1013700003302046072123F07F0343F054031A462D
:10138000FFF71CFF0C23204609211A46FFF716FF22
:101390000723082120461A46FFF710FF40E700BF49
:1013A000B877012013B504466A4608210068FFF7A4
:1013B00089FC9DF8003013F010037ED006236A46A6
:1013C00000212068FFF762F9002874D09DF80130F1
:1013D0009DF800201B029DF804109FED396A03EB75
:1013E00002439DF8022009021A441C029DF80330B2
:1013F00048BF02F17F4201EB03419DF8053007EE43
:10140000902A0B440902F8EEE77A48BF03F17F43C4
:10141000C7EE866A07EE903A2A4BB3F92C20B8EE55
:10142000E77A07EE902AB3F92820F8EEE77AC7EEBC
:10143000065A06EE102AB3F92420B8EEC66AA6EEC4
:10144000A76AD3ED087AB8EEE77AD3ED077AF8EE1B
:10145000E77AA6EE867A26EEA55AE6EE877A07EEBA
:10146000102AB3F92A20B8EEC77A06EE102AB3F98B
:101470002620B8EEC66AE5EE877A07EE102AB3F9A1
:101480001820B8EEC77AA6EE867AF6EE006AE5EE88
:10149000077A07EE102AB3F91A20B8EEC77AC3ED1F
:1014A0000C7A07EE902AF8EEE77A67EEA57AE7EE77
:1014B000267AC3ED0D7A02B010BD1846FBE700BFD7
:1014C00000007848B877012013B5002204460A21AD
:1014D0000068FEF707FF142003F005FA0F220A2127
:1014E0002068FEF7FFFE0A2003F0FDF901AA03239E
:1014F00010212068FFF7CAF80A2003F0F4F99DF8DC
:101500000420154B0A218032206823F8542C9DF8C2
:101510000520803223F8522C9DF80620803223F8D3
:10152000502C0022FEF7DEFE0A2003F0DCF90DF15C
:10153000030202212068FFF7C5FB0DF10302092118
:101540002068FFF7BFFB11220A212068FEF7CAFEC0
:10155000012002B010BD00BFB088012037B504469D
:101560006A4602210068FFF7ADFB18B9002528463E
:1015700003B030BD9DF80030DA07F7D507236A467F
:1015800003212068FFF782F805460028EED01122DB
:101590000A212068FEF7A6FE9DF806301B07E5D459
:1015A0000B4A684632F9541CFCF7BAFA404232F949
:1015B000521CE0860DF10200FCF7B2FA32F9501C21
:1015C000208701A8FCF7ACFA40426087CFE700BF54
:1015D000B088012013B5002204460A210068FEF7F6
:1015E00081FE142003F07FF90F220A212068FEF704
:1015F00079FE0A2003F077F9032301AA102120685D
:10160000FFF744F80A2003F06EF900220A2120684F
:10161000FEF768FE0A2003F066F90DF103020221CD
:101620002068FFF74FFB0DF1030209212068FFF747
:1016300049FB01220A212068FEF754FE012002B076
:1016400010BD30B5002385B004460221C3860DF1DC
:10165000070283630068FFF735FB18B900252846A9
:1016600005B030BD9DF80730DB07F7D5062302AA89
:1016700003212068FFF70AF80DF10702092120680D
:10168000FFF720FB05460028E8D09DF8073013F04F
:101690000C0FE3D1BDF8083001220A212068C3EB0A
:1016A00083339B00E386BDF80A309B002387BDF897
:1016B0000C30C3EB83339B006387FEF713FECEE74A
:1016C0001FB5002304460DF10702272100688DF89D
:1016D0000730FFF7F7FA68B19DF8073013F00803F9
:1016E00020D0062302AA28212068FEF7CFFF18B9D0
:1016F000E086A06304B010BDBDF90830002BB8BF70
:1017000003339B10E386BDF90A30002BB8BF0333C7
:101710009B102387BDF90C30002BB8BF03339B10FF
:101720006387E7E71846E5E71FB5002104460DF19A
:101730000702C18681630068FFF7C4FAC0B19DF853
:10174000073013F0080315D0062302AA01212068F0
:10175000FEF79CFF60B1BDF808305BBAE386BDF8C8
:101760000A305BBA2387BDF80C305BBA5B426387F3
:1017700004B010BD1846FBE730B5002585B004461F
:101780000621C5860DF1070285630068FFF79AFA06
:10179000A0B19DF8073013F0040311D0062302AA6C
:1017A00029462068FEF772FF40B1BDF80830E38695
:1017B000BDF80A302387BDF80C30638705B030BD13
:1017C0001846FBE730B5002585B004463421C586B0
:1017D0000DF1030285630068FFF774FA40B39DF9C9
:1017E0000330AB4226DA092301AA24212068FEF740
:1017F0004DFFE8B19DF808209DF8073012049DF8D0
:101800000A109DF8045042EA03629DF80B301B0455
:10181000C2F30F4243EA01639DF8051022870904D1
:10182000C3F30F4341EA05616387C1F30F41E186CA
:1018300005B030BD2846FBE7130A13B504468DF802
:1018400004308DF80520032301AA8DF806100068E6
:101850006021FEF7D5FE142003F045F800210DF1BC
:10186000030220688DF80310FFF72CFA02B010BDB8
:1018700037B50446002514208DF8075003F033F8DF
:101880000DF1070229462068FFF71CFA0DF1070247
:1018900080212068FFF716FA294620467C22FFF7B0
:1018A000CBFF204646F2C4220421FFF7C5FF2046A5
:1018B0001D220821FFF7C0FF0DF107021E2120683D
:1018C000FFF700FA012003B030BD13B5084C0DF14D
:1018D0000702A02154F8680CFFF7F4F918B19DF83D
:1018E00007309B0602D541F079FBF0E702B010BD4E
:1018F000B0880120F0B51D4A8DB000234FF400518F
:10190000013322F8021BB3F5F07FF9D1184E194DBF
:101910003468A5F1610732343A46802155F8680CE5
:10192000FFF7D0F9F8B133689C42F5D810240022B3
:10193000012623460134222103A8E4B20096FCF7D5
:101940004BF90246202CF4D14C2303A80093012329
:10195000FCF742F903AA0346002155F8680C44F04D
:1019600019FD0DB0F0BD10240246E1E764880120A6
:1019700088330120B088012018B1838802681B04D5
:101980009361704710B504464069FFF7F5FF0120E9
:1019900002F0A9FF6069FEF772FC0A20BDE8104062
:1019A00002F0A1BF2DE9F043046889B00646B622D3
:1019B0007E212046FEF796FC642002F094FF02216F
:1019C0002046DFF82091FEF778F92046FFF7DAFF8E
:1019D00000227C212046FEF785FC012002F083FFD7
:1019E000002259212046FEF77DFC012002F07BFFFA
:1019F0005E2301254FF000088DF807300DF1070335
:101A000002A92046039309F2F633CDF80880069325
:101A10004FF4A473324F0793CDE9045842F018FBFA
:101A20000A2002F060FF2A4659212046FEF75AFCA0
:101A3000284602F058FF8C2240212046FEF752FC37
:101A4000284602F050FF032241212046FEF74AFCBF
:101A5000284602F048FFB16B09F23E52092396F87E
:101A60003500B7FBF1F189B2FDF750FB4388422105
:101A7000B7FBF3F737640279204642F0C002FEF765
:101A800031FC284602F02FFF082243212046FEF7B2
:101A900029FC284602F027FF042258212046FEF7A1
:101AA00021FC284602F01FFF0A2253212046FEF7A0
:101AB00019FC284602F017FF42467C212046FEF71B
:101AC00011FC284602F00FFF06227D212046FEF77A
:101AD00009FC284609B0BDE8F04302F004BF00BF8E
:101AE00040420F008C11060830B50C4687B0054601
:101AF000E0B103680E4A03F13F4303F57E0302EBB6
:101B0000932393F8740541F0EBF9002301A92868A9
:101B10000593AB88019304F013030293C4F34113BC
:101B2000C4F3810403930494F8F742FA07B030BD7C
:101B30008C11060870B50C4686B016460546D0B125
:101B400003680E4A03F13F4303F57E0302EB932340
:101B500093F8740541F0C4F9AB8801A92868019392
:101B600004F0130302936309C4F381040393CDE9E2
:101B70000446F8F71DFA06B070BD00BF8C110608C8
:101B800038B5040900F00F02013C032C1AD80E4DA1
:101B900005EB4403B3F87A1541FA02F313F00100A0
:101BA0000FD001232C4403FA02F2013A02EA0100A9
:101BB00045F0B8FF94F882350C221844034B02FB21
:101BC000003038BD0020FCE78C110608248C012071
:101BD0002DE9F04F002104468BB054225F484DF0B0
:101BE000C1FB5F4B611E0334184611F8012F551ECF
:101BF000052D88BF00228C4240F8042BF5D11946F0
:101C0000002251F8040B012800F029830132042A34
:101C1000F7D1002253F8041B022900F01683013289
:101C2000042AF7D103204F4EFBF780FE0420FBF778
:101C30007DFE4A4C05204FF01A094FF0000A06F5C8
:101C4000B167DFF83081FBF771FE0620FBF76EFE0F
:101C5000207B40B394F90D50FFF792FF28B1052384
:101C600080F807908371002303720321FFF73CFF84
:101C7000227B002317F8331091426AD106EBC3038D
:101C8000D3F88C352361C02303FB0585D5F8A83133
:101C90005A1C23750723C5F8A821A37501239A446C
:101CA000637585F8A43109F101090C345FFA89F9EB
:101CB000B9F1200FCCD1BAF1000F47D02A4B002543
:101CC0002A4C2B4E049394F8B830002B36D0607910
:101CD00041F006F9207941F003F90122D4F8BC1053
:101CE0004FF44033234FC020914263614FF0000313
:101CF000A2622264D8BF4FF0000CA361C8BF4FF0AE
:101D0000010CE361636200FB05720191E162C4F8BA
:101D100020C0C4E90E33C4E90C3323682361D2F830
:101D20003C1109B9C2F8401100FB0570D0F83C1114
:101D300011F0100120D0002384F84C30049B0135B1
:101D4000C03403F58C73032D0493BCD10BB0BDE8F4
:101D5000F08F0133102B8DD1002393E750840120A5
:101D6000FC7701208C110608A8840120CC150120E5
:101D700000230140E0140120D0F83C214FF400582A
:101D800022F4885222F0020242F00202C0F83C2102
:101D9000726822F440327260726842F440327260BB
:101DA0005A6822F480725A605A6842EA0C225A60D9
:101DB0005A6822F040725A605A685A609A6822F44F
:101DC00000629A609A689A609A6822F070629A60DB
:101DD0009A689A609A6822F040529A609A689A606B
:101DE0009A6822F002029A609A6842F002029A60AF
:101DF0005A6822F400625A60DA6A22F47002DA62E7
:101E0000019AD3F82CE002F1FF3C4EEA0C524FF459
:101E1000806EDA629A6822F400729A609A6842F4DC
:101E200000729A609A6822F480629A609A689A6056
:101E3000C0F84011D0F83C2122F0030242F0010228
:101E4000C0F83C214FF40062D4F80CC084F84C1068
:101E50006166C4F88810C4E91AE24FF48072DFF8B2
:101E6000A8E3C4E91C824FF40032C4E91E21032216
:101E7000C4E92021A268C4E917C1A265DEF8008088
:101E800084F88C10022180F87911116821F0010189
:101E900011601168C90700F137811168182022F418
:101EA0007F7EDFF8689321F0FF512EF0030E21F4BE
:101EB000772121F47C6141EA0C0C4CF40B3141F4A4
:101EC00080711160516921F007015161D1B210395F
:101ED000B1FBF0FCC3485F294FF03F01604488BF6D
:101EE0000EF1040E90F80806C4F8B0E08140C4F882
:101EF000B40004F15800CEF808100591C02101FB90
:101F000005770021C7F89811012187F87911A0649D
:101F100004F110000391C4F8900068B2079099F89A
:101F2000150000285CD099F90D00079FB84257D1E1
:101F300001F1010C94F84CA0D9F810005FFA8CF76D
:101F4000BAF1010F99F8168006974FF0000708972D
:101F50003FF4F4AE4FF00107092884F84C7087B2C3
:101F6000029740F2E98007EB470C4FF0070BD3F8DC
:101F70000CA0ACF11E0C9C4F0BFA0CFBB8422AEAE9
:101F80000B0AC3F80CA040F0D080D3F80CC04CEA88
:101F9000086CC3F80CC0062901EB810C00F2E1804B
:101FA000ACF1050C4FF01F08596B08FA0CF8029FB2
:101FB00021EA080107FA0CFC5963596B4CEA01014C
:101FC00059638A498B4206D1122840F021817168F9
:101FD00041F4800171604FF0000184F84C100699C3
:101FE000039809F10C0901300728039097D10021CB
:101FF000099194F84C1001293FF4A0AE012184F816
:102000004C109968CF0740F1D2809968C8077FF5D6
:1020100095AE774FC02000FB0570D0F83C1121F43D
:10202000E06121F0010141F48071C0F83C11596870
:10203000490507D5D0F83C1121F4405141F48051B5
:10204000C0F83C11C02101FB0571D1F83C0110F42E
:10205000805003D0D1F8400120F00600C1F84001C3
:102060000021644884F84C10C4F894006248C4F815
:1020700098006248C4F8A4006FF022001860586805
:1020800040F080605860986840F48070986001204B
:1020900084F88C00C02000FB057797F879010128AF
:1020A00040F09880022087F87901C7F898111168EC
:1020B000019821F4802111601421484303F14C015F
:1020C000506091600499D1600599CEF808101168AC
:1020D00041F016011160516941F0800151611168B0
:1020E00041F008011160116841F00101116072684E
:1020F000D20672D19A6812F0405F7FF41FAE9A68E0
:1021000042F080429A6019E6DEF80010A1EB080167
:1021100005297FF6BEAEC02303FB05772023C7F851
:102120009831032387F8793108E6D3F80CA008FA30
:102130000CFC4CEA0A0C2CE700EB400B4FF0070AB2
:10214000D3F810C00AFA0BFA08FA0BF82CEA0A0CBA
:10215000C3F810C0D3F810C048EA0C08C3F81080C8
:1021600019E70C294FF01F0110D8ACF1230CD3F85C
:102170003080029F01FA0CF107FA0CFC28EA0101F9
:102180001963196B4CEA010119631AE7ACF1410CB0
:10219000D3F82C80029F01FA0CF107FA0CFC28EA14
:1021A0000101D962D96A4CEA0101D96209E799684B
:1021B000134841F00101996012490968B1FBF0F13F
:1021C00001EB41010991099900293FF41EAF0999DA
:1021D0000139F7E784F88C1089E7044A93427FF4C9
:1021E000ADAD87E78C1106081200001000200140F9
:1021F000E014012001800008578000085980000881
:1022000040420F00BC010120E8260120508401203B
:102210001849884202D011287FF4DDAE716841F47C
:1022200000017160134988427FF4D5AE124913480A
:102230000968B1FBF0F10A2041430891089900298F
:102240003FF4C9AE08990139F7E70D4B312283F805
:10225000B02C93F8EC2C013283F8EC2CE2E4084A21
:10226000322182F8A41C92F8EC1C013182F8EC1C9B
:10227000CFE400BF12000010BC01012040420F005B
:10228000B87701202DE9F0471F46AB4DAB4B9D427F
:1022900021D26C798C4240F06D812C79844202D03D
:1022A000002840F06781EC79944240F063812C680B
:1022B000DCB11C220021201D4DF054F825602B7943
:1022C0002371012B95F80680C4F808802A7AE26011
:1022D00003D0022B0CD0002407E0E87AFFF750FC73
:1022E0006B7AA0612374AB7A63742046BDE8F087F3
:1022F000E87AFFF745FC95F90960A0612674A87A91
:10230000FFF73EFC6061002800F0308114238C4D03
:10231000734305EB0309EB58002B00F0278199F874
:102320001230002B40F0EE8099F8080040F0D8FD04
:1023300099F80830012103F01F025B09023B01FA02
:1023400002F2032B08D8DFE803F0827C02767D4995
:102350000B6923EA02020A61142306F1010A03FB56
:1023600006535FFA8AFA5879FFF70AFC814620B1D2
:1023700040F60A3380F808A0C380142303FB0653F9
:10238000D879FFF7FDFB20B140F60A5380F808A08A
:10239000C380142303FB06539879FFF7F1FB20B1A8
:1023A00040F60A4380F808A0C380142348464FF043
:1023B000140918F0040803FB065309FB065918BF5B
:1023C0004E215A7A08BF2E21FFF7B4FB99F8070077
:1023D000FFF7D6FB99F80A202E21FFF7ABFB99F8FF
:1023E0000600FFF7CDFB99F80B200E21FFF7A2FBAB
:1023F00099F8040050B1FFF7C3FB20B140F60A631F
:1024000080F808A0C3800D21FFF76EFB14237343EF
:10241000EA58136823F0400313604B4B9A421CD1D7
:1024200003F58433596A41F480515962596A21F4A1
:10243000805159622AE043494B6923EA02024A610A
:102440008AE740490B6A23EA02020A6284E73D49AF
:102450004B6A23EA02024A627EE73C4B9A420CD066
:1024600003F580639A425BD1364B196A41F400410F
:102470001962196A21F4004107E0324B196A41F4EC
:1024800080411962196A21F4804119625368B8F1D8
:10249000000F43F4805314BF0020022053601368E0
:1024A0005B0615D4116821F47F4121F0BF01B8F11A
:1024B000000F08BF41F00101014341F44571116073
:1024C000536823F4706323F0040343F4E063536020
:1024D000D36923F40063D361136843F040031360AE
:1024E000536843F480535360142303FB0653187955
:1024F00018B1FFF745FBFDF7C2FE142303FB065599
:102500000123AB74606920B10E238771C37100236E
:1025100003720D21FFF7E8FA6069FDF7B0FEE4E60B
:102520000B4B9A4216D1074B596A41F4005159623C
:10253000596A21F400517CE7E8010008980300087B
:102540000000012000380240003001400038004007
:1025500000340140084B9A4298D1084B596A41F423
:1025600080115962596A21F4801162E72046FDF713
:1025700097FBB0E60C358AE6005001400038024077
:1025800038B500221F2333210120FFF77BFE3D4B8E
:1025900043F86C0C10B90024204638BDAE20FDF77E
:1025A000B8FF04460028F6D0D4204FF48065FDF72C
:1025B000B0FF8020FDF7ADFFA820FDF7AAFF3F2068
:1025C000FDF7A7FFD320FDF7A4FF0020FDF7A1FF33
:1025D0004020FDF79EFF8D20FDF79BFF1420FDF7A7
:1025E00098FFA120FDF795FFC820FDF792FFDA20A4
:1025F000FDF78FFF1220FDF78CFF8120FDF789FF8B
:10260000CF20FDF786FFD920FDF783FFF120FDF7EE
:1026100080FFDB20FDF77DFF4020FDF77AFFA4203F
:10262000FDF777FFA620FDF774FFAF20FDF771FFE0
:10263000A620FDF76EFFAE20FDF76BFF2020FDF713
:1026400068FF0020FDF765FFB020FDF762FF402026
:10265000FDF75FFF0020FDF75CFF1020FDF759FF3D
:10266000013D002043F0BCFCADB2002DF8D181202B
:10267000FDF74FFFC820FDF74CFFAF20FDF749FFE6
:102680008AE700BFB0880120F7B52C4DC2B20E23F7
:1026900031210220FFF7F6FDC5F8DC00002841D00B
:1026A00003210024FDF709FB322002F01CF99F23CF
:1026B0006946D5F8DC00019304238DF801402646D5
:1026C0000DEB030243F066FE9DF802309DF80120F9
:1026D00020461B021A4943EA02439DF80320134394
:1026E000184A14809481C2E901440F68E7B90EB119
:1026F000108094811088A8B1002393734FF48073E5
:10270000538093891B0258435360B0F1807F9060DF
:1027100005D90123B72085F8E830FBF70FFB01202E
:1027200085F8E00003B0F0BDBB4201F1080102BF33
:1027300031F8040C012631F8024CD6E7B8770120B5
:102740009C170608E01401202DE9F84F694B93F817
:10275000F000002840F0CB80D3F8ECA09AF81030BD
:10276000002B40F0C480DFF894C186463C269CF8DC
:1027700076260CF27A699CF877369CF87856ACF895
:10278000740699F8021099F80370C1F1FF0189B23B
:10279000002900F0A880B9F80040C1F1FF01B4FBA6
:1027A000F6FB79430912BBF1050F1FD8DFE80BF0E8
:1027B000030D5E6C7D8B7B1ACDB26343B3FBF6F3E6
:1027C00053FA81F3DBB23A460FE0B4FBF6F206FBB4
:1027D00012427C1ACDB292B2C2F13C026243B2FB09
:1027E000F6F252FA81F2D2B23B46012017020021E2
:1027F00047EA034747EA05080127C1F1170B0EEB2B
:102800000104013107FA0BFB2A341BEA080FA4B2BA
:102810000CBFBB464FF0020B374F182947F824B0C6
:10282000EAD10EF1180E09F104091FFA8EFEBEF569
:10283000406FA6D1ACF87AE828B18CF876268CF8EF
:1028400077368CF878568023ACF874369CF87C3850
:10285000002B4CD0504640F62B41F9F78BFA254B14
:10286000D3F8EC00BDE8F84FF9F7DCBAB4FBF6F3A7
:1028700006FB13447D1ACAB2A4B26543B5FBF6F554
:1028800055FA81F1CDB2AFE7B4FBF6F306FB134383
:102890007C1ACAB29BB2C3F13C036343B3FBF6F3A9
:1028A00053FA81F3DBB23D469FE7B4FBF6F006FB3B
:1028B00010447A1ACBB2A4B26243B2FBF6F252FAD7
:1028C00081F2D2B2EFE7B4FBF6F506FB15457C1AB0
:1028D000CBB2ADB2C5F13C056543B5FBF6F555FA93
:1028E00081F5EDB26FE73D463B463A467DE7BDE8F0
:1028F000F88F00BFB877012080AF0120B088012099
:1029000070B500211820F9F7BBF8064608B3F9F7AF
:1029100055F8224B0446C3F8EC00D0B1204D1820E6
:10292000FFF72EF9C5F8800820B140F21523C380C7
:1029300000230372327A4E21FFF7FCF895F88438B1
:10294000022B07D1FBF716FB2046F9F7EBF9002322
:10295000036070BD032B06D1FBF70CFB2046F9F793
:10296000E1F96423F4E7FBF7E9FA10B985F87C088C
:10297000EFE743F2AC0200210A484CF0F3FC95F873
:102980008438012B02BF084BFF22C3F8A820012383
:1029900085F87C38BDE87040D6E600BFB8770120E6
:1029A000B088012080AF012080DF012038B5114BB5
:1029B000D3F8EC0058B193F8F02042B10E4C94F8E3
:1029C0008428032A04D1F9F7ADF96423036038BDE4
:1029D000022A4FF0000503D1F9F7A4F90560F6E7E4
:1029E00083F8F050FBF7AAFA0028F0D184F87C08AD
:1029F000EDE700BFB8770120B08801202DE9F04F46
:102A00000021464FA9B04FF00A0B0C4607F6880A82
:102A10003C225046FBF702FC051E57DB07EB450343
:102A2000C5F307295FFA85F833F84C2C13F84C6C82
:102A3000130A7007039317F8603C03F0400151D567
:102A400059B943F0400322468C2105A807F8603CA1
:102A500000930423FBF7C0F8044649F00203B600D4
:102A60008C212246009305A80523F6B2FBF7B4F8A3
:102A700006230246CDF8008005A8FBF7ADF8072332
:102A80000246009605A8FBF7A7F805230246CDF8F5
:102A9000009005A8FBF7A0F806230246CDF80080B9
:102AA00005A8FBF799F8039B024605A800930723A6
:102AB000FBF792F8294604465046FBF7A2FBBBF110
:102AC000010B03D0691CB1F5F07FA1D31CB357F8FB
:102AD000680C234605AA002143F05CFC012029B0C4
:102AE000BDE8F08F19B903F03801B1420DD023F0E1
:102AF00078038C2105A813432246DBB207F8603C1B
:102B000000930423FBF768F80446052322468C2132
:102B1000CDF80090BDE72046E1E700BFB088012076
:102B200073B5234C14F8623C002B3ED101230DF108
:102B30000702842154F8680C04F8623CFEF7C2F8DE
:102B400014F8602C042154F8680C42F00402FDF7DC
:102B5000C9FB0DF10702842154F8680CFEF7B2F8A6
:102B60009DF8073013F00405F3D1124E3C2229469C
:102B7000114804F8603C4CF0F5FB06F6D40036F83A
:102B8000023B1A0A03F0040322F02002134302D08E
:102B90002946FBF71DFB0135B5F5F07FEFD1FFF7B7
:102BA0002DFF0028FBD104F8620C02B070BD00BFFD
:102BB000B0880120648801203891012030B5254C6F
:102BC00085B054F8680C002841D014F8643C012BFF
:102BD00013D0022B13D00DF10B02A021FEF772F8D7
:102BE0009DF80B3003F00503012B06D043B11A4BBF
:102BF0001A6840F2DC539A4229D9402300E00023AE
:102C000043F008030025022203A804F8613C8DF874
:102C10000D3004238DF80C5019460093FAF7DCFFB1
:102C200003AA0346294654F8680C43F0B3FB3C2240
:102C3000FF210A484CF096FB14F8633C3BB954F86A
:102C4000683C0BB1FFF76CFF012304F8633C05B04F
:102C500030BD00BFB08801208833012038910120A9
:102C6000F8B51D4C05460F4614F8623C002BFDD10B
:102C7000012304F8623CFDF78FFCEAB20646092105
:102C800054F8680CFDF72EFBB5F5807F05D1402286
:102C90000A2154F8680CFDF725FB00255022082175
:102CA00054F8680CFDF71EFBFEF70FFEEAB20A218E
:102CB00054F8680CFDF716FB7A190135C02154F859
:102CC000680CFDF7FFFF362DF0D10EB9FDF764FC5F
:102CD000002304F8623CF8BDB0880120F0B5234E13
:102CE000C5B004460F4616F8625C002DFDD10123E5
:102CF00006F8623CFDF750FCFF2C8DF80D404FF0BC
:102D000009034FF002028CBFA4082C464FF00005C7
:102D10008DF80C3088BF04F0C00444EA05034FF47A
:102D2000827103A8DBB200930A23FAF755FF7B5D9B
:102D300001350246009303A80B23FAF74DFF362D09
:102D40000246EAD1A02303A800930823FAF744FF20
:102D500003AA0346002156F8680C43F01BFBFEF75C
:102D6000B4FD002306F8623C45B0F0BDB0880120F8
:102D7000002A4FF0200CBCBF80185242002BBCBF71
:102D8000C9185B420028BCBF121A00200029F0B508
:102D900000EB0204BCBF5B1800210E4E1D3C3C271B
:102DA000002CC8BF121BCC180F3C0244002CC8BF1B
:102DB0001B1B0B4490420CDC06EB40050C4604E068
:102DC00007FB04FE013425F80EC09C42F8DD0130FB
:102DD000F0E7F0BD64880120014B53F820007047F4
:102DE00050280040014B43F8201070475028004005
:102DF0001A4B07B51A6C1A4942F080521A641A6CC1
:102E000002F080520192019A0A6842F480720A60CC
:102E1000FF211A6C42F480621A641A6C02F4806218
:102E20000092009A0F4A5162CA21516253215162A5
:102E30005B6FDB0005D50020FFF7CEFF0A4B984201
:102E400009D000210120FFF7CDFF0749002003B082
:102E50005DF804EBC6E703B05DF804FB0038024000
:102E6000007000400028004076614E69F8B52A4D98
:102E70000646D5F8EC40002C49D095F8F030002BF0
:102E800040D16368254A1B69C3F3032352F823101A
:102E9000E3685868EFF31187102383F312886268A0
:102EA000D2F800C092F805E01D4ADCF80C3032F888
:102EB0001E2002F4F05223EA0203CCF80C30F7F79C
:102EC0005FFCE3681A69596820231F2A20D9203A39
:102ED0009340CB60FFB287F3118800212368022260
:102EE00021745B68186883F83D20026842F0010293
:102EF0000260012283F83D20D5F8EC30DB681977B9
:102F0000FBF738F8D5F8EC00F8F70CFF0660F8BDD1
:102F100093408B60DEE700BFB877012050040608BD
:102F2000700406087047034B53F820300BB19B68C0
:102F30001960704748F1012008B5FFF7F4FFBDE8BC
:102F400008401AF08FB8054B03EBC00040F2FF7346
:102F50009942A8BF1946A0F84410704748F10120D3
:102F60000C4A13787BB10C4B93F8A01059B193F82D
:102F7000A11059B150680021FA2883F8A110A8BF08
:102F80004FF0FF3070476FF0010070476FF00200A4
:102F9000704700BFF420012048F101200B4B93F84B
:102FA000A2206AB193F8A3206AB1002283F8A3207B
:102FB000074B9868B0F5967FA8BF4FF0FF30704779
:102FC0006FF0010070476FF00200704748F1012078
:102FD000F4200120014B1B685B681847D89801203A
:102FE000014B1B689B681847D8980120014B1B6850
:102FF000DB681847D8980120014BD868704700BF9C
:10300000F4200120044B93F8A43013B1034B18694A
:1030100070476FF00100704748F10120F420012053
:1030200020B10078B0FA80F0400970470120704765
:103030000A4B07EE901A03EBC00010B5046C5CB1AC
:10304000F8EEE77A94ED047A94ED030AA7EE870A86
:1030500047F0F2F9A368186010BD00BF48F10120E5
:1030600007B50DF10702FDF72DFE034B18709DF813
:10307000070003B05DF804FBF420012007B502232C
:1030800001AAFDF703FB044B1870BDF8040040BA19
:1030900080B203B05DF804FBF420012007B50223E1
:1030A00001AA00210068FDF7F1FA0F4B83F8A40094
:1030B00050B1BDF804300D4A5BBA9BB2B3F5FA6F5C
:1030C00005D34FF0FF33136103B05DF804FB0A2111
:1030D000B3FBF1F307EE903AF8EEE77AFDEEE77A0C
:1030E000C2ED047AF0E700BF48F10120F42001208E
:1030F00013B502230C4601AA00210068FDF7C6FAA9
:1031000060B15CB19DF805309DF90420DB0902EB4C
:10311000820203EB830303EB4203238002B010BD62
:1031200008B5FDF7DFF8014B187008BDF420012049
:10313000F8B5144E41F0010200210446124FFFF78A
:10314000EFFF3568C7F8A85013212046FFF788FF26
:1031500010F007000BD001220B212046FFF7E0FF03
:10316000002220461146FFF7DBFF012008E0D7F8D8
:10317000AC20002AE8D033689BB25B1B9A42E3D2B2
:10318000F8BD00BF8833012048F1012070B53B4CE9
:10319000054694F8A030002B36D094F8B060012E8C
:1031A00033D0022E4FD07EBB012280210068FFF772
:1031B000B7FF0122FF212868FFF7B2FF32463146F0
:1031C0002868FFF7ADFF94F8B12091212868FFF738
:1031D000A7FF012231462868FFF7A2FF3246FF21F0
:1031E0002868FFF79DFF324680212868FFF798FF87
:1031F000012231462868FFF793FF214B1B68C4F872
:10320000A830012384F8B03070BD00210068FFF7BA
:1032100027FFC20711D5D4F8AC20002AF4D0184BF0
:10322000D4F8A8101B689BB25B1A9A42ECD2154BDB
:103230004FF0FF325A600023E4E7114B1B68C4F8DB
:10324000A8300223DEE713210068FFF709FF4307D8
:10325000E1D01E212868FFF711FF012206460B214D
:103260002868FFF75DFF0A20064BB6FBF0F6B6B202
:103270005E60012384F8A130DDE700BF48F1012042
:1032800088330120F420012010B50023094C84F874
:10329000B230032384F8B310FF2184F8B42004F182
:1032A000B202FDF7ADF900280CBF6FF00C00002052
:1032B00010BD00BF48F10120F8B5124D002416469C
:1032C000022305F1B20285F8B310FF21074685F805
:1032D000B240FDF795F905F1B20210B96FF00C009C
:1032E000F8BD0223FF213846FDF7D0F90028F5D0BC
:1032F00095F8B220204695F8B33003EB02233380D3
:10330000EEE700BF48F101200023024A5121006886
:10331000FDF776B9FAF2012013B5022301AA04469B
:1033200051210068FDF7B2F9114AF0B1BDF804303F
:103330005BBA9BB2D360D368B3F5C87F02DD4FF0B0
:10334000FF33D3600B4B0C4A1968D2F8B4313233D7
:103350008B4208D2C2F8B411002302F5D972512170
:103360002068FDF74DF902B010BD6FF00103E8E7EA
:10337000F42001208833012048F1012037B5124D97
:10338000044695F8A230E3B10DF10501006842F062
:103390008BFD9DF805307BB10DF10602962120686A
:1033A000FFF78AFF0A22BDF80630B3FBF2F3074AA3
:1033B0009360012385F8A330012286212068FFF75E
:1033C00063FF03B030BD00BF48F10120F4200120AD
:1033D000FCF756BC0FB413B504AB094C094953F8BC
:1033E000042BD4F8B801019341F03CFBD4F8B801A8
:1033F000FCF73AFC02B0BDE8104004B0704700BFD3
:1034000048F10120D1330108202108B54CF009FF13
:10341000034618B11A780130202AF9D0184608BDA1
:1034200070B50D461446FFF7EFFF0646A0B1FCF756
:1034300007FA40F634039842A8BF1846B0F5617FFA
:10344000B8BF4FF46170A0F561731920B3FBF0F3BE
:103450002B702378013323703046FFF7D5FF0646E3
:10346000A0B1FCF7EDF940F634039842A8BF184626
:10347000B0F5617FB8BF4FF46170A0F5617319209A
:10348000B3FBF0F36B70237801332370304670BDCB
:1034900037B505460846019143F0B4FC019904464E
:1034A00002462846FBF746FF68B92B5DA3F13002C0
:1034B000092A06D923F02003413B192B01D90134F5
:1034C000281903B030BD0020FBE710B504460846BC
:1034D00021601946F8F7DAF9BDF808102068F8F706
:1034E000E7FA2068F8F734FC2068022203685B687A
:1034F000196883F83D200A6842F001020A6001223F
:1035000083F83D20F8F70EFC0023A060036010BD97
:103510002DE9F04F85B0994607468A469DF83C3024
:1035200090460393F8F74AFA054650B1224B93F8B8
:10353000BC11092909D90025204A00210420FBF7E4
:10354000E1FC284605B0BDE8F08F4A1C5C2003F57D
:10355000E0765FFA82FB01FB006683F8BCB100FBFA
:1035600001330021C3F8C01183F8C4113879FEF784
:1035700007FB044628B1022380F806A080F808B0B3
:10358000C371039B7BB13A7A02212046FEF7D2FA3F
:10359000BDF8383029464246304600934B46354602
:1035A000FFF793FFCDE720461121FEF79DFA204655
:1035B000FEF7E2F9ECE700BF48F101201AB4060873
:1035C0003A4B1B782DE9F3470746002B6CD0384E59
:1035D00096F8585596F859350135ED1A102D0DDD30
:1035E000344B0222002104201A701023324A009327
:1035F0002B46FBF787FC02B0BDE8F08796F86235F2
:10360000012B11D0022B13D02C4B96F86215C6F863
:10361000683511F0FD010FD0294A0221042002B0C3
:10362000BDE8F047FBF76EBC42F040F9254BECE7F4
:1036300042F03CF9244BE8E77B68AB4229DBDFF83A
:10364000708030370C46DFF88490DFF890A0AC42F1
:10365000D1DADAF800200321B6F85C35C2F3007243
:10366000B9FBF3F301929BB2B6F85A25009257F8D2
:10367000040B164AFFF74CFF014688B90D4B052293
:1036800004201A702346124A02B0BDE8F047FBF747
:1036900039BC084A0420107000932B460D4AA8E755
:1036A000013448F8040BD2E70B4AB6E72CE00120BE
:1036B00048F10120DC93012055B40608272F0108AA
:1036C00081B4060865D00208392F010840420F0076
:1036D000F3B40608BDB4060818B5060800000020BB
:1036E0001E4B30B51C68B4FBF1F303F57F43FF3389
:1036F0001B0CB4FBF3F4B4FBF1F52DED028B0023AE
:1037000083B00221F0EE408A019222460093ABB2D0
:10371000B0EE608AFFF7FCFEE0B1B5EE408A07EE3E
:10372000904A0123F8EE677AF1EE10FA03710ABFAE
:1037300007EE105A67EE880AF8EE470A9FED087AFE
:10374000C0EE876A27EE667AC0ED046AA7EEA87A13
:1037500080ED037A03B0BDEC028B30BDBC010120CB
:1037600000007A440023064910B51C46984200DC4C
:1037700010BD51F833200AB1926814600133F5E7A7
:1037800088F1012013B50F4C8DF80700A168D4E92A
:10379000042353438B4212D063680DF10701E068A4
:1037A000184449F037FC636822691344A268B3FBEC
:1037B000F2F102FB1133636063690133636102B0AC
:1037C00010BD00BF60A301200F4B93F86C35062B92
:1037D00014D8DFE803F0161304070A0D10004FF4A5
:1037E000FA607047094B988870474FF47A607047C9
:1037F0004FF4FA5070474FF47A5070474FF47A7094
:1038000070474FF4C870704748F10120D0930120F1
:103810006D4B2DE9F04F2DED028B93F8008085B0B4
:103820000546B8F10C0F0FDD684B01221A700C230E
:10383000674A0093434600210420FBF763FB05B071
:10384000BDEC028BBDE8F08F624B634F9979032981
:1038500087F86C1513D90B1F022B12D95F4BC7F8D1
:1038600070355F4B13F8113003BB5E4A0221042010
:1038700005B0BDEC028BBDE8F04FFBF743BB5A4BE4
:10388000EDE7FFF7A1FF594A80B207F5B0634FF0AB
:10389000000A4FF0000BB2FBF0F00022C7F87805E9
:1038A000C3E900ABC7F87C25514BD8E72B684345EB
:1038B00019DB504C08354FF00009DFF864B19FED7B
:1038C0004E8AC145BBDADBF8002097F86C3555F815
:1038D000046BC2F30072062B6FD8DFE803F0642993
:1038E000310B3B3B3B00394A0321117000934346A7
:1038F000424AA0E70392FFF767FFDFED410A014666
:10390000039AB0EE600A3046FFF7EAFE206054F8F2
:10391000081B002954D12D4B052204201A704B4658
:10392000384A05B0BDEC028BBDE8F04FFBF7EABAB0
:103930000392FFF749FFDFED340A0146039AE0E7FF
:103940000392FFF741FFDFED310A0146039A9FED35
:10395000300AD8E7052B24D02E492F48062B08BF64
:1039600001464FF0000A3046019214230A46CDF872
:1039700000A00221FFF7CCFD064680B100F1140340
:1039800012220068194603933FF044FC039B30B1B8
:103990001846482251464BF0E5FC0123337126605E
:1039A000B5E71E49DDE70392F0EE480AFFF70CFF8A
:1039B0009FED110A0146039AA5E700232360A6E7BD
:1039C00009F101097DE700BF2C000020DC930120F4
:1039D00032B50608D093012048F10120252F0108B7
:1039E000701B06085EB506083130010840420F0022
:1039F000472F010888F101206F12833A7CB5060831
:103A000000000000B5B506086F120339ACC5A73732
:103A1000ACC5A736C0C62D00001BB700808D5B006B
:103A200000000020034AD2F8682512B10F2800D800
:103A30001047704748F10120130A07B58DF804308C
:103A400002238DF8052001AAFCF7DAFD024B18705D
:103A500003B05DF804FB00BFF420012050B1013831
:103A6000002330F0FF019AB203F1010303D140EAD1
:103A7000022080B270474008F3E710B50C460121E0
:103A8000FFF7EEFAC0F300132370C0F3C003A37076
:103A9000C0F380036370C0F38013C0F3C010E37001
:103AA000207110BD2DE9F047884650211446064686
:103AB000FFF7D6FA01304621304F40004FF47A79B3
:103AC0004FF4FA6AC0B220803046FFF7C9FA237873
:103AD000013051217B4380B203F5FA73A080B3FB20
:103AE000F9F2B3FBFAF300FB02333046B3FBF9F310
:103AF000E360FFF7C3FAC0F30F22C3B22578304664
:103B000003FA02F27D43013293B205F5FA72B2FB79
:103B1000F9F1B2FBFAF203FB01227021E380B2FB60
:103B2000F9F22282FFF79CFA013071214000C0B205
:103B300060803046FFF7A2FA98F80320C3B2C0F3C2
:103B40000F20834001339BB2238112B1E2889B1A7C
:103B50002381A3784FF47A724FF4FA6520897B436E
:103B600003F5FA73B3FBF2F1B3FBF5F300FB01339A
:103B7000B3FBF2F36382BDE8F08700BF002F3A0089
:103B80002DE9F0434FF4FA730026844F8DB00446BC
:103B900089210068C7F8AC3087F8A060FFF760FAA9
:103BA00040F001008921DFF8F881C2B22068FFF7F8
:103BB000B7FA324688212068FFF7B2FA0122802145
:103BC0002068FFF7ADFA0122FF212068FFF7A8FA6D
:103BD000324631462068FFF7A3FA91212068FFF7AB
:103BE0003FFA3146012287F8B1002068FFF798FAC2
:103BF0003246FF212068FFF793FA32468021206881
:103C0000FFF78EFA60212068FFF72AFA40F01200D1
:103C10006021C2B22068FFF783FA20224421206885
:103C2000FFF70AFFFF2201212068FFF779FA2568D4
:103C3000012280212846FFF773FA0122FF2128463E
:103C4000FFF76EFA324631462846FFF769FA062238
:103C5000FF212846FFF764FA83212846FFF700FA80
:103C600040F004008321C2B22846FFF759FA072228
:103C7000FF212846FFF754FA012281212846FFF749
:103C80004FFA012280212846FFF74AFA6B2294213D
:103C90002846FFF745FA324683212846FFF740FAC7
:103CA000D8F80060C7F8A86083212846FFF7D8F944
:103CB000002800F05583012228468321DFF8E480A4
:103CC000FFF72EFA92212846FFF7CAF90022C0F327
:103CD000C716814681212846FFF722FA0622284688
:103CE000FF21FFF71DFA8321284609F07F09FFF71E
:103CF000B7F9832100F0FB022846FFF711FA2846A6
:103D00000122FF21FFF70CFA284601220021FFF7CC
:103D100007FA28460022FF21FFF702FA2846002270
:103D20008021FFF7FDF9062305AAB02120680025B0
:103D3000FCF7ACFC0122FF2188F800002068FFF7A7
:103D4000EFF900224F212068FFF7EAF92C224E21DB
:103D50002068FFF7E5F90022FF212068FFF7E0F96E
:103D6000B422B6212068FFF7DBF9002E2A464FF077
:103D7000010C18BF0C26C5F3C4005FFA85FE05F0E0
:103D8000070100F1300376450DEB030010F81C3CF1
:103D90000AD8914540F0EF8206E000BF48F10120CB
:103DA00088330120F42001200CFA01F123EA0103F9
:103DB00000F81C3C0135302DDDD1062305AAB021C9
:103DC0002068FCF71DFC0122FF2188F80000206814
:103DD000FFF7A6F9002220681146FFF7A1F900229B
:103DE000FF212068FFF79CF9002209212068FFF7D6
:103DF00097F9002210212068FFF792F90022112183
:103E00002068FFF78DF9012224212068FFF788F947
:103E1000FF2225212068FFF783F900227521206801
:103E2000FFF77EF90122FF212068FFF779F92C22A4
:103E30004E212068FFF774F9002248212068FFF71F
:103E40006FF9294620222068FFF76AF90022FF2136
:103E50002068FFF765F9294609222068FFF760F915
:103E6000002254212068FFF75BF9042231212068E9
:103E7000FFF756F9032232212068FFF751F9832218
:103E800040212068FFF74CF9252246212068FFF7E2
:103E900047F9002260212068FFF742F9002227211C
:103EA0002068FFF73DF9062250212068FFF738F916
:103EB000002251212068FFF733F996225221206811
:103EC000FFF72EF9082256212068FFF729F92A4624
:103ED00057212068FFF724F9002261212068FFF7AD
:103EE0001FF9002262212068FFF71AF900226421DD
:103EF0002068FFF715F9002265212068FFF710F907
:103F0000A02266212068FFF70BF90122FF2120681B
:103F1000FFF706F9322222212068FFF701F9142267
:103F200047212068FFF7FCF8FF2249212068FFF7AE
:103F3000F7F800224A212068FFF7F2F80022FF215B
:103F40002068FFF7EDF80A227A212068FFF7E8F8E9
:103F500000227B212068FFF7E3F8212278212068E6
:103F6000FFF7DEF80122FF212068FFF7D9F834229D
:103F700023212068FFF7D4F8002242212068FFF7B0
:103F8000CFF8FF2244212068FFF7CAF826224521F6
:103F90002068FFF7C5F8052246212068FFF7C0F822
:103FA000402220681146FFF7BBF806220E21206848
:103FB000FFF7B6F81A2220212068FFF7B1F8402257
:103FC00043212068FFF7ACF80022FF212068FFF7AB
:103FD000A7F8032234212068FFF7A2F844223521F4
:103FE0002068FFF79DF80122FF212068FFF798F86D
:103FF000042231212068FFF793F809224B21206821
:10400000FFF78EF805224C212068FFF789F804227B
:104010004D212068FFF784F80022FF212068FFF778
:104020007FF8002244212068FFF77AF820224521FA
:104030002068FFF775F8082247212068FFF770F81D
:10404000282248212068FFF76BF8002267212068AA
:10405000FFF766F8042270212068FFF761F801225B
:1040600071212068FFF75CF8FE2272212068FFF7BB
:1040700057F8002276212068FFF752F800227721B6
:104080002068FFF74DF80122FF212068FFF748F86C
:1040900001220D212068FFF743F80022FF2120684C
:1040A000FFF73EF8012280212068FFF739F8F82257
:1040B00001212068FFF734F80122FF212068FFF773
:1040C0002FF801228E212068FFF72AF80122002113
:1040D0002068FFF725F80022FF212068FFF720F86D
:1040E000002280212068FFF71BF804220A212068A3
:1040F000FFF716F8256884212846FEF7B1FF8421D2
:1041000000F0EF022846FFF70BF801220B21206890
:10411000FFF706F8206803A90190FFF7AEFC07AA95
:1041200003A90198FFF7BEFC9DF80C30002B00F0AE
:1041300028810A9D05F684559DF80E30002B00F06D
:1041400023810A9B03F2B22305EB43059DF80F3050
:1041500023B1BDF82C3003F525731D449DF81030B4
:1041600023B1BDF82E3003F226231D44E82201219D
:104170002068C7F88855FEF7D3FF44F61F639D42B9
:1041800003D92946206841F0AFFE0122206811467C
:10419000FEF7C6FF40212068FEF7CAFF002800F0A6
:1041A000E780012120680222FEF7BAFF0021206883
:1041B000FEF7BEFF002800F0DB80E8220121206826
:1041C0004FF47A79FEF7ACFF202244212068FFF7F4
:1041D00033FC256803A948F20E662846DFF8C08143
:1041E000FFF74BFC07AA03A92846FFF75BFC502208
:1041F00057212846FEF794FF082256212846FEF74D
:104200008FFF082250212846FEF78AFFBDF82C00B8
:1042100009FB0060B0FBF8F080B2FFF71FFC5121F2
:1042200002462846FFF708FC0A9A5C4B462109FB28
:10423000026628469E429BBFB6FBF8F202F1FF32AF
:10424000FF22D2B2FEF76CFFD7F8881544F61F6341
:10425000994202D9284641F047FE01212846FEF73F
:10426000FFFE0222064601212846FEF759FF0021E3
:104270002846FEF75DFF324601212846FEF750FF33
:10428000246803A92046FFF7F8FB07AA03A92046E4
:10429000FFF708FC482220461146FEF741FF08229E
:1042A00047212046FEF73CFF032232212046FEF73D
:1042B00037FF072230212046FEF732FF0122FF217F
:1042C0002046FEF72DFF202230212046FEF728FF52
:1042D0000022FF212046FEF723FF06222046702100
:1042E000FEF71EFFBDF82E304FF47A7246F64400FA
:1042F00002FB03004DF28803B0FBF3F09DF80F3092
:1043000080B21BB1BDF82230184480B2FFF7A6FB83
:10431000712102462046FFF78FFBD7F8881544F637
:104320001F63994202D9204641F0DEFD012120465B
:10433000FEF796FE0222054601212046FEF7F0FE1A
:1043400000212046FEF7F4FE2A4601212046FEF712
:10435000E7FE6423C7F8AC30012387F8A03007E0FC
:10436000D8F800309BB29B1BB3F5FA7F7FF69CAC6C
:104370000DB0BDE8F0830B41DB0744BF0132D2B280
:1043800018E540F63635D7E69DF80D30002B3FF4A2
:10439000DDAE0A9B03F525731D44D7E61B280D01EE
:1043A0001C0C010010B500230A4C84F8B230130A2B
:1043B00084F8B310FF2184F8B430042384F8B520C6
:1043C00004F1B202FCF71CF900280CBF6FF00C00DE
:1043D000002010BD48F101202DE9F3410023744D68
:1043E00006460468DFF8D4812D2785F8A230B9B2DB
:1043F000013718F8012B2046FEF746FF882FF6D12B
:10440000402287212046FEF73FFF00238DF806302B
:104410000DF10601204641F047FD9DF80630002BC6
:10442000F6D0012286212046FEF72EFF00228721AA
:104430002046FEF729FF092208212046FEF724FF27
:1044400000220B212046FEF71FFF002851D13768BC
:104450000DF106025E213846FEF72EFFBDF806304C
:10446000B3F5D77F00F09F8053D8512B00F099808F
:1044700047D81D2B6AD01E2B00F093802121306875
:1044800041F081FC34680DF10602DE212046FEF782
:1044900013FFBDF8063028229FED467AC3F30903C7
:1044A000FF212046ADF806305343002207EE903A34
:1044B00085F8B2206C22F8EEE77A85F8B32067EE33
:1044C000877AFCEEE77A17EE903A1A0E85F8B73045
:1044D00085F8B4201A0C85F8B5201A0A062385F849
:1044E000B620354AFCF78CF8402287213068FEF769
:1044F000CBFEB0FA80F0400985F8A20002B0BDE81A
:10450000F081AD2B4FD0D62B01D0602BB6D121241A
:104510001DE040F2E132934247D00CD840F2D9225C
:10452000934242D040F2E122934202D0B3F5E67FBB
:10453000A4D164240BE040F28F42934203D040F2B6
:10454000915293429AD14FF4FA7400E00F2400285C
:1045500094D10A224B213846FEF796FE0F226021A5
:104560003846FEF791FE0D2263213846FEF78CFE99
:10457000B82269213846FEF787FE40F60D72782191
:104580003846FFF70FFF40F60E627A213846FFF7F4
:1045900009FF00287FF472AF2146384641F0F3FB53
:1045A0006CE71424D3E73224D1E7C824CFE700BF57
:1045B00048F101209A99893FFAF101207E1B0608F3
:1045C00038B50B0A15460C4A044682F8B23002236D
:1045D00082F8B310B232FF21FCF712F810B96FF075
:1045E0000C0038BD01232A46FF212046FCF74EF877
:1045F0000028F4D00020F4E748F1012003681B688C
:10460000184703685B68184703689B681847036886
:10461000DB6970B506460C46154683B1BDE87040AF
:1046200018473046FFF7F0FF0028FAD014F8011BB6
:104630003046FFF7E3FF2B1B002BF2DC70BD0D446F
:10464000F9E7E4E70368DB68184708B5194B1A4C2B
:10465000D3F88C55A0681CF0E7FC28461CF0E4FC5D
:10466000A06841798B0704D4036841F002019B697B
:10467000984700203EF056FCA068FFF7C2FF60B1EB
:1046800001203EF04FFCA068FFF7DCFF0146284602
:10469000FFF7B4FF00203EF045FC2846FFF7B1FFCE
:1046A0000028E9D02846FFF7CDFF0146A068FFF7B4
:1046B000A5FFE1E748F10120A895012003681B69E7
:1046C000184703685B69184703689B6A03B118477A
:1046D00070470368DB6A03B118477047134B014604
:1046E0001B68DB0606D5124BB3F8903513F0040FA8
:1046F00018BF00210F4B9B7A73B10F4B1B68A3B1FE
:104700009A6839B10D4B19880D4BB3FBF1F35B106F
:1047100013607047116070470A4B18680A4B1B788A
:104720000BB981F00101FBF7A2BD70470800002022
:1047300048F10120AC940120B89401201895012083
:1047400040420F00A4940120A8940120BFF34F8F92
:104750000549064BCA6802F4E0621343CB60BFF31D
:104760004F8F00BFFDE700BF00ED00E00400FA0539
:1047700008B572B600224FF0FF319300013203F109
:104780006043082A03F56143C3F88010C3F8801121
:10479000F3D1FFF7DBFF012108B50846FEF722FB46
:1047A000FFF7E6FFEFF31183102282F312880B4923
:1047B000DBB20A6801320A604FF0E02208499069D2
:1047C000C1F8A0050020C1F8A405126983F311887F
:1047D000044A136801331360704700BF8833012017
:1047E00048F10120E8260120064B074A1B68516862
:1047F00058434FF47A73B0FBF3F053685B1A83426B
:10480000FBD97047802F0120001000E010B5EFF3B6
:104810001182102383F312884FF0E0239C691969F9
:1048200011F4803F0D4903D00120C1F8A4059C6913
:104830000B4BD2B21868D1F8A43582F31188094A1B
:10484000034411684FF47A7202FB01F0001BB0FBC5
:10485000F1F00021E3FB020110BD00BF48F101208F
:1048600088330120802F0120124B5B68C3F30803BB
:1048700030B4EBB9EFF31183D3B90F4B4FF0E02510
:104880000E481968AC691A688A42FAD1D0F8A015A6
:10489000A142F6D30A4B19684FF47A7303FB01F077
:1048A000001BB0FBF1F0002130BCE2FB03017047BC
:1048B00030BCABE700ED00E08833012048F1012077
:1048C000802F0120F8B506460D46FFF7CDFF0446C0
:1048D0000F46FFF7C9FF031B61EB0702B34272EB00
:1048E0000503F6D3F8BD10B50446013C00D210BD57
:1048F0004FF47A700021FFF7E5FFF6E708B50122D3
:1049000009210068FBF7EEFC6420BDE80840EAE7F7
:1049100006460B2580B5013D01D1FFF73CFF771C12
:104920004FF03208052400203EF0FCFA3EF056FB22
:104930000120FFF7D3FE4046FFF7D5FF3EF04EFBC8
:104940000020FFF7CBFE4046FFF7CDFF7CB1013CD6
:1049500005D14FF0FA084FF4FA70FFF7C4FF54EA9C
:104960000703E3D14FF47A70FFF7BDFFD3E7013FB0
:10497000F5E718B103685B6803B11847FF2070477B
:1049800018B103689B6803B118470020704770B4E2
:1049900050B106798E4207D34579954204D3036816
:1049A000DB680BB170BC184770BC704710B440B1E5
:1049B00084798C4205D303681B6913B15DF8044BFD
:1049C00018475DF8044B704718B103685B6903B181
:1049D0001847704718B10368DB6903B11847002016
:1049E000704718B103681B6A03B11847002070476D
:1049F00030B568B1041D0A4600F11403206808347C
:104A000054F8041C15469C4203C52A46F6D10120E1
:104A100030BD10B50C4670B92D23002023750A4B0C
:104A20002061C4E906333023C4E90000C4E9020070
:104A300084F8203010BD0368DB6A002BECD0984767
:104A40000028E9D0F6E700BFA600070838B5441EE5
:104A5000044D14F8011F01B938BDD5F8B801FBF7B2
:104A60000FF9F6E748F1012013B50C4C01900C4802
:104A70000091FFF7EBFF0B49D4F8B801DDE90032F4
:104A80003FF0F0FFD4F8B801FBF7EEF894F8A83542
:104A900013B1012384F8A93502B010BD48F10120FB
:104AA000DAB50608D1330108084D0446084808B5B0
:104AB000FFF7CCFFD5F8B801FBF7D6F8D5F88C0591
:104AC0001CF0B2FA204609F00BFD00BF48F10120AE
:104AD000E6B50608034808B5FFF7B8FF0120FFF761
:104AE000E3FF00BFF2B506087FB5184B93F8AA257F
:104AF000012A28D193F8AF350A2B04D0144807B007
:104B00005DF804EBA2E71122002101A84AF02AFC7B
:104B1000A623152168468DF8003041238DF8021038
:104B20008DF80130EB238DF803300A4B1B7D8DF897
:104B30000430B2238DF8053003238DF8063021F0C0
:104B4000CAF90548DBE707B05DF804FB48F101202E
:104B50000BB60608F42001201AB6060810B5044664
:104B60000B48FFF773FF06F05BFC20F061FFFAF7DC
:104B70009AFE20F067FF074B00220749204683F882
:104B8000A925FEF785FC08B9FFF78EFF10BD00BF11
:104B900034B6060848F101204BC30608054808B59D
:104BA000FFF754FF044BB3F8CA0510B1BDE8084045
:104BB00099E608BD0412070848F1012010B5074C1A
:104BC00002460B460649D4F8B8013FF04BFFD4F833
:104BD000B801FBF749F8BDE81040DFE748F10120D4
:104BE000D13301080FB407B504A951F8040B0191A2
:104BF000FFF73AFFFFF7D2FF03B05DF804EB04B014
:104C0000704770B5837916468EB0044603F00702EC
:104C1000062A52D8DFE802F00415181A1D1F4B00AF
:104C20000D7813F0C0034AD0402B3ED129462046D0
:104C300013F082F800285ED00EB0BDE87040FEF799
:104C4000C9BB91F90050ECE70D88EAE7B1F90050D3
:104C5000E7E70D68E5E791ED000A02A8FAF700FD25
:104C600001462A48FEF7B6FBFEB1A37913F0C00F48
:104C70001BD1204612F0AFFF00EE100A02A8B8EEDA
:104C8000C00AFAF7EDFC01462148FEF7A3FB2046D7
:104C900012F0B2FF00EE100A02A8B8EE400AFAF7CE
:104CA000DFFC01461A48FEF795FB0EB070BD1748B1
:104CB0000EB0BDE87040FEF78DBB0025B1E7042AB9
:104CC00029460CBF13481448FEF784FB002EECD095
:104CD000A37913F0C00FE8D1204612F07CFF0190B9
:104CE000204612F089FF019902460C480EB0BDE83B
:104CF0007040FEF76FBB02A9204612F07FFE02AAA9
:104D000029460748FFF76EFFCFE700BFF1B7060857
:104D100075BC060811BB0608ECFF0608301307082F
:104D20004AB6060813B50446019112F047FF019AEE
:104D30000146204602B0BDE8104062E7004851E756
:104D400067B606082DE9F04F87B00346FEF768F90D
:104D5000064618B107B0BDE8F04FEFE705AA47498E
:104D60001846344649F066F9B04605464FF0FF371D
:104D7000DFF83091DFF830A1DFF830B18DB97EB2C5
:104D800030461BF007FF10B14568002D5BD1B8F12C
:104D9000000F36D139463A48FAF783F807B0BDE834
:104DA000F08F012E0ED0022E11D01EB92846FAF730
:104DB00047FD074605AA31490020013649F03AF976
:104DC0000546DBE72846FAF73BFD8046F2E7494611
:104DD00028464BF080FA20B92A4928464BF07BFA46
:104DE00008B144F00104514628464BF074FA28B942
:104DF000594628464BF06FFA0028DBD044F00204F5
:104E0000D8E7002C4FF00003304608BF03241A46B1
:104E100019460293E4B2CDE900841CF088F80546F7
:104E200010B939461848B7E7424639461748FAF7E5
:104E300038F839461648FAF734F8164B2946D3F8AD
:104E40008C053EF077F839461348FAF72AF85CB13A
:104E50006979A14208D022461048FAF722F82B6857
:104E6000E1B228469B699847EB6A002BE1D00C48D9
:104E7000FAF717F80023EB62DBE700BF380B0708EF
:104E800076B60608FDED06089EB60608BDB606080D
:104E900028B7060848F10120DAB60608F2B6060877
:104EA00012B7060803C7060873B6060809CF060836
:104EB0002DE9F3474FF0000A4FF0FF35DFF8D090AF
:104EC00001AA57465446D0462E46314949F0B2F819
:104ED00068B9BAF1040F50D03ADCBAF1020F13DC12
:104EE0002B4632462B4901203CF0B4FF0EE0BAF1CC
:104EF000040F09D8DFE80AF0030D12171C00FAF7B7
:104F00009FFC064603281BD9FFF718FF02B0BDE837
:104F1000F087FAF795FC05469528F4E7FAF790FC38
:104F200080463F28EFE7FAF78BFC04463F28EAE784
:104F30000378482B03D0562BE6D1012700E0002749
:104F400001AA494600200AF1010A49F073F8BFE7B7
:104F5000BAF1050FD8D1A40108F03F08962304F454
:104F60007C6403FB06550C4E44EA080406EB450539
:104F700044EA4734A5F8CC45C8E7962303FB06521C
:104F8000054B03EB4203B3F8CC75C7F34037E2E7B8
:104F9000380B070814F7012048F1012013460A4690
:104FA000014601481EE600BF56B706082DE9F04F3E
:104FB00085B00546FEF734F8044630B100210120E3
:104FC00005B0BDE8F04F3CF0BDBE85492846FAF774
:104FD000CDF920B905B0BDE8F04F35F0B1BA81493F
:104FE0002846FAF7C3F928B9012005B0BDE8F04F0B
:104FF00035F012BC7C492846FAF7B8F9034680BB65
:105000007A4A82F8200E104692F9271E92F8D2545E
:10501000012D08D0033D052D05D9002C00F0D180CD
:1050200080F8271ECDE092F8D3540133A52D13D17B
:1050300001290ED16E4A80F8213E002380F8201EFF
:1050400082F87C3A80F8273E05B0BDE8F04F35F095
:105050002DBC0139012449B2782B02F11402D5D1BB
:10506000DBE72846FAF7ECFB614B834693F97C3A81
:1050700003FA80F60093772E00F2A7802846FEF709
:10508000C3F90746002800F08980FAF7D9FB01240C
:10509000C5B23846FEF7B8F90746002800F081800F
:1050A0000134FAF7CDFB0190E4B23846FEF7ACF9D3
:1050B0008046002877D00134FAF7C2FB0746E4B2F5
:1050C0004046FEF7A1F9814600286ED00134FAF778
:1050D000B7FB0290E4B24846FEF796F982460028F4
:1050E00065D00134FAF7ACFB0FFA80F9E4B2504610
:1050F000FEF78AF9824600285BD00134FAF7A0FB5C
:105100000FFA80F8E4B25046FEF77EF9002852D03C
:105110000390FAF795FB03990FFA80FA0846FEF719
:1051200073F90346002857D004F0FD04FAF788FB12
:10513000042C46D1C3B2012D02D9E91E052940D85D
:105140001BB1A52B01D0482B3BD1284C0EB984F8BC
:10515000276E1421019AA52B01FB0646C6F8C02430
:10516000029A86F8D254C6F8C474C6F8C824A6F8C1
:10517000CC94A6F8CE84A6F8D0A486F8D3340AD16D
:1051800000981B4B0130584483F87C0A94F8273E62
:10519000013384F8273E05B0BDE8F08F044605468C
:1051A00077E7019081E707468AE7029093E7814617
:1051B0009DE78046A7E75FFA88F382468046062C83
:1051C000B9D005B0BDE8F04FB8E5772221460948CF
:1051D00005B0BDE8F04FE1E60134E4B2EFE700BF0F
:1051E00073B7060879B7060815C5060830E0012030
:1051F00048F101207EB7060810B50F4C94F8A83589
:1052000073B194F8A9355BB10C48FFF7EBFC0C487F
:10521000FFF7E8FC002384F8A83584F8A93510BD11
:105220000848FFF713FC20F003FCFAF73CFB20F0E2
:1052300009FC0020FFF738FC48F1012087B7060879
:10524000BEB70608DCB706082DE9F04F01F02003D1
:105250008FB081460F464C4C4FF0000800934B4BEB
:10526000D3F8B801FAF700FD94F806B00BF0380354
:105270004B454BD1204612F03BFCFAF72BFC06467F
:10528000204612F057FCD6F808A005460AEB0006A7
:10529000204612F093FC0BF00702062A6BD8DFE8D9
:1052A00002F0043F44484D515D001AF80520007893
:1052B000111A4A424A41009B03B13ABB02A9204657
:1052C000019212F09BFB7B0615D5019A9AB902A9AF
:1052D0002F48FEF77FF82F4902A841F089FD0028EA
:1052E0004BD11AF80530202B47D131462A48FEF71A
:1052F00071F8FFF753FC02A92848FEF76BF800226B
:1053000031462046FFF77DFCFFF748FC08F1010815
:1053100040F266230B349845A1D10FB0BDE8F08F61
:105320001AF9052090F90000C2E73AF80520008834
:10533000BEE73AF90520B0F90000B9E75AF80520B0
:105340000068B5E796ED007AD0ED007AB4EE677AA2
:10535000F1EE10FA0CBF01220022ACE701902046CA
:1053600012F04AFC0199421C304649F08DFFB0FA18
:1053700080F252099FE700229DE700223146204635
:10538000FFF73FFCB5E700BF1F25060848F10120E5
:10539000E3B7060802130708CBBA0608E4B7060805
:1053A000F8B50C4C34250C4E0C4F2068FFF74EFB23
:1053B000616811B13046FEF70DF8A16811B13846A9
:1053C000FEF708F8FFF7EAFB013D04F11004ECD109
:1053D000F8BD00BFDC1B06083ED50608EEB7060880
:1053E00008B5FFF733FBBDE80840FFF7D7BB10B5A2
:1053F00004460348FFF72AFB2046BDE81040EFE7CC
:10540000F4B7060810B527F0EBFC134CD8B11348DD
:10541000FFF7EDFF1248FFF719FBD4F8B801FAF7D0
:1054200023FC4FF47A70FFF75EFAD4F88C051BF07A
:10543000FBFD0C4B1878FEF795F902210120FDF7D2
:10544000D1FCFFF795F90848FFF700FBD4F8B80145
:10545000BDE81040FAF708BC48F10120F9B706088A
:10546000E6B506082C00002019B8060808B5FAF7BA
:105470009DFE83681BB90948BDE80840B0E70848AD
:10548000FFF7AEFF27F052FCFAF787FE08B1054898
:10549000F2E76420FFF727FAF6E700BF48B80608EE
:1054A0005CB8060867B806080A4D00240A4808B523
:1054B000FFF796FFD5F8B801FAF7D6FB85F87D4AD5
:1054C000C5F8C04A85F8C44A13F0E4FE2046FFF749
:1054D000EBFA00BF48F101206DB8060810B50522AF
:1054E000184904464AF0B2FE60B9174B93F8A82554
:1054F00022B9012183F8A92583F8A8151348BDE82E
:1055000010406DE70322124920464AF09FFE98B9E9
:105510000D4C94F8A8355BB194F8A93543B10D480A
:10552000FFF760FB002384F8A83584F8A93510BD87
:105530000948FFF755FFF5E70848BDE81040FFF7B9
:1055400051BB00BF13C3060848F1012097B80608F5
:1055500036C5060887B70608ADB80608C1B80608FC
:1055600010B504460648FFF771FA2046FFF76EFAB9
:10557000044B93F8A82512B1012283F8A92510BD88
:10558000DAB5060848F101200CB4830607B500D54A
:1055900051B905A904980191FFF710FB012003B050
:1055A0005DF804EB02B070470020F8E7024B0146BB
:1055B000D3F8B801FAF764BB48F101200CB407B581
:1055C00010F0400009D069B92320FFF7EFFF05A9CB
:1055D00004980191FFF7F2FA012003B05DF804EBA3
:1055E00002B070470020F8E72DE9F04F074687B07A
:1055F00016460C4615464FF0000B4FF019094FF4B4
:105600006178DFF8A4A0002E4BD02378287883425D
:10561000EB7844D161786A78914240D1A178AA7838
:1056200091423CD1E178CA1A51425141CDE904136B
:1056300011F0F0FA059B0499524619FB038303937A
:10564000AB7819FB038302936B7801934379384657
:1056500000935B46FFF7B2FF04992078043504916C
:1056600011F0D8FAE37852460499043419FB038305
:10567000039314F8023C19FB0383029314F8033CD0
:1056800001934379384600935B460BF1010BFFF71A
:105690007BFFBBF1280FB6D107B0BDE8F08F00212A
:1056A000C4E73146D9E700BFD0B80608F7B50746CA
:1056B000FDF7B6FC044630B100222749012003B0B3
:1056C000BDE8F04090E73846FAF7BAF827280546D3
:1056D0003ADC8600781C8DF80740FDF795FE0446FD
:1056E00078B1FAF7ADF800280BDBC0B211F0A4FADC
:1056F00038B11A4B0279334483F8C52A01238DF857
:1057000007302046FDF780FE044660B1FAF798F8AE
:105710000D2808D8114B334483F8C60A9DF807308A
:1057200001338DF807300C4FB11C0DF107022046F4
:105730003944FDF775FE9DF80730042B02D0002395
:1057400047F8253003B0F0BD27222146044803B0B6
:10575000BDE8F04022E400BF0DFC012048F101202B
:10576000E6B906082DE9F04F804689B00C4615468B
:1057700002F1540B334EDFF8D490069294F90410E2
:1057800000230C2202FB03F02F4FC057884254D055
:105790000133072BF6D10C350C345D45EED109B041
:1057A000BDE8F08F95F904302A689942687995F838
:1057B00006C095F808E095F807A03CD12168914211
:1057C00039D16179814236D1A179614533D1217ACC
:1057D000714530D1E179A1EB0A077942794156F858
:1057E0002A7056F82000049756F82E7007910397F8
:1057F00056F82C70CDE9002002974A464046FFF744
:10580000DDFE0799E279404694F9043056F82220EB
:105810000492227A56F822200392A27956F8222086
:105820000292627956F822200192226800924A463A
:10583000FFF7AAFEAFE70021D1E7069B002BB1D10D
:105840001946DFE7F4180608F0910120E3B80608CE
:10585000F0B585B00346FDF7E3FB30B100224049C7
:10586000012005B0BDE8F0407CE718465E1CF9F762
:10587000E7FF044640B21BF00DFB054630B9214658
:10588000384805B0BDE8F040FFF7ACB9006801AB9F
:10589000696803C3A86818603046FDF7B5FD044683
:1058A00000284CD003782B2B05D02D2B3CD0F9F7BA
:1058B000C7FF019009E001342046F9F7C1FF01223A
:1058C000019B02FA00F003430193022600272046C1
:1058D000FDF79AFD044600B3F9F7B2FF2249002212
:1058E0008C4651F804EBD3B2704503D00132112A33
:1058F000F7D100235CF8232090420ED1022F20D054
:10590000032F21D0012F14BF8DF809308DF80A30F4
:1059100001370136042FF6B2D9D1012E17D805B0C0
:10592000BDE8F040FFF70ABA01342046F9F788FFD6
:105930000122019B02FA00F023EA0003C4E70126DA
:10594000C4E78DF80C30E3E78DF80B30E0E701ABEE
:1059500003CB286018686960A86005B0F0BD00BF7F
:105960008CA0012000B90608F41806082DE9F04FB4
:10597000804689B017460C46154600264FF0190A96
:105980004FF46179DFF8B4B0002F54D06979A8786A
:105990000791A1782B7881426A7895F803C095F831
:1059A00004E0069345D12178994242D16178914231
:1059B0003FD1E17861453CD12179714539D1617997
:1059C000079BCB1A59425941069B1AFB029206913A
:1059D0001AFB039303925A46CDE90103079B404605
:1059E00000933346CDE904CEFFF7E8FD069923790D
:1059F0005A46404606340593063514F8033C049392
:105A000014F8053C1AFB0393039314F8063C1AFBA5
:105A10000393029314F8043C019314F8013C00939F
:105A200033460136FFF7B0FD142EADD109B0BDE805
:105A3000F08F0021C8E73946D9E700BF13B906083F
:105A40002DE9F3478246FDF7EBFA064630B1002216
:105A50003B49012002B0BDE8F04787E75046F9F71F
:105A6000EFFE1328054663DC364C06278DF80760E9
:105A7000474304F665390AF10100FDF7C5FC09EB5F
:105A80000708064648B1F9F7DBFE03289FBFE31974
:105A900083F86A0B01238DF807303046FDF7B4FC1C
:105AA000064668B1F9F7CCFE0D2809D8062303FB9A
:105AB000054383F8670B9DF8073001338DF80730F5
:105AC0000DF1070241463046FDF7AAFCFDF79CFCAC
:105AD000064668B1F9F7B4FE3B2809D89DF80730AF
:105AE0000622013302FB05428DF8073082F8680B6D
:105AF0003046FDF789FC68B1F9F7A2FE0D2809D8F8
:105B00009DF807300622013302FB05448DF807306B
:105B100084F8690B9DF80730062B06D0002349F85E
:105B20000730A8F80430FFF709F902B0BDE8F087A4
:105B300013223146044802B0BDE8F047FFF72EBA01
:105B4000ADFC012048F10120E6B906082DE9F04F2F
:105B5000074690460C4615460026DFF80CA12DEDB1
:105B6000088B97B094ED008AB5EE408AF1EE10FAFA
:105B700071D0D4ED019A94ED029AD4ED038AB8F174
:105B8000000F40D095ED000A95ED01BAB4EE408AC1
:105B9000D5ED02AA95ED03AAF1EE10FA60D1F4EE6C
:105BA0004B9AF1EE10FA5BD1B4EE6A9AF1EE10FA6C
:105BB00056D1F4EE4A8AF1EE10FA0CBF4FF001090B
:105BC0004FF0000912A8F9F74BFDB0EE4B0A8346DF
:105BD0000EA8F9F745FDB0EE6A0A05900AA8F9F794
:105BE0003FFDB0EE4A0A049006A8F9F739FD049A81
:105BF000059B49460390384602925246CDE900B3D0
:105C00003346FFF7DBFCB0EE480A12A8F9F728FD8F
:105C1000B0EE690A81460EA8F9F722FDB0EE490AF6
:105C200083460AA8F9F71CFDB0EE680A049006A89E
:105C3000F9F716FD049B0390524600213846CDF833
:105C4000009010341035CDE901B333460136FFF72B
:105C50009BFC0C2E86D117B0BDEC088BBDE8F08FF5
:105C60004FF00009AEE700BF31B9060870B5054630
:105C7000FDF7D6F9064660B1404B4FF4C872404973
:105C80009B7802FB0311002210310120BDE8704017
:105C90005CE705223B492846F9F74CFB68B9374BCE
:105CA0004FF4C8719A78364B01FB02330022013061
:105CB00043F8102F0C28FAD170BD2846F9F7C0FD23
:105CC0000B28044653D82846FDF79EFB06460028BD
:105CD00038D0F9F729FD294B192201259B7802FBC1
:105CE0000342274B03EB021383ED040A3046FDF712
:105CF0008BFB064660B1F9F717FD204B19220135E1
:105D00009B7802FB03421E4B03EB021383ED050A53
:105D10003046FDF779FB064660B1F9F705FD174BF4
:105D2000192201359B7802FB0342154B03EB02134A
:105D300083ED060A3046FDF767FB28B9BDE87040E1
:105D4000FEF7FCBF0546D1E70C4B9E78F9F7ECFC5B
:105D500019200B49032D00FB064401EB041484EDCC
:105D6000070AEBD14FF4C87303FB06118BE73146EA
:105D70000B220548BDE87040FFF710B9BD91012026
:105D800028FD012073B70608E6B906082DE9F0439F
:105D9000804685B00D46164602270024DFF858904D
:105DA0003EB336F8242035F82430F05B93421ED100
:105DB000EB5B191A4B424B4119462346CDE90020B3
:105DC0004A4640460391FFF7F9FB0399EB5B4A46CD
:105DD00040460437019335F82430009323460134BC
:105DE000FFF7D2FB042CDBD105B0BDE8F083002324
:105DF000E2E73146EAE700BF45B90608F8B50446D0
:105E0000FDF70EF9054628B100222A490120BDE818
:105E1000F840BBE728492046F9F7A8FAA8B9274B6C
:105E20004FF47A714FF4FA62A3F8001FA3F8022F1F
:105E3000A3F8041FA3F8062FA3F8081FA3F80A2F3E
:105E4000A3F80C1FA3F80E2FF8BD2046F9F7F8FCB5
:105E50000328074627D82046FDF7D6FA044670B136
:105E6000F9F7EEFC012506462046FDF7CDFA10B104
:105E7000F9F7E6FC2DB9BDE8F840FEF75FBF05462F
:105E8000F2E7A6F2EE2240F2DC539A42F3D8A0F2F7
:105E9000EE229A42EFD8094B03EB8703A3F8006F79
:105EA000A3F8020FD0E7294603220548BDE8F840D1
:105EB000FFF774B84800022073B7060848F10120C4
:105EC00056B906082DE9F04F834691B091460C462D
:105ED00015460026DFF8F0A004F11508042209A8F1
:105EE0000BAF41464AF0D4F900238DF82830D4E9AD
:105EF0000232082B72F1000155D21A462E4938465B
:105F0000F8F7EAFFB9F1000F54D02B780793079AFE
:105F1000237893424CD1D4E90202D5E902139A4284
:105F200008BF884244D1227D2B7D9A4240D1042271
:105F300005F1150140464AF055F9002838D121698C
:105F40002B69CB1A594259411C4B5246584605936E
:105F500000230493B5F912300393B5F9103002937E
:105F6000174B0193079B079100933346FFF726FBDE
:105F7000079909AB5246584620350593237D049373
:105F8000B4F912300393B4F91030CDE9017314F869
:105F9000203B009333460136FFF7F6FA082E9BD1DB
:105FA00011B0BDE8F08F07493846F8F795FFA9E72B
:105FB0000021C9E74946DCE7ECFF06083CD40608A7
:105FC0002DF206085EB9060869B906082DE9F74FF3
:105FD0000446FDF725F8074630B100226D4901203F
:105FE00003B0BDE8F04F6DE76B492046F9F7BEF905
:105FF000014638B94FF48072664803B0BDE8F04FEF
:1060000049F0B0B92046F9F71BFC054683B2072BCF
:1060100000F2B8802046FDF7F7F9824600284CD000
:10602000F9F70EFC01240FFA80F95046FDF7ECF960
:1060300068B14FF00008411E00F1100C464611F8FF
:10604000013F13F0DF0F3BD101270134E4B2FDF72C
:10605000DBF9824600284CD00134F9F7F1FB0FFA46
:1060600080FBE4B25046FDF7CFF90346002842D04A
:1060700001340190F9F7E4FB019B0FFA80FAE4B2D6
:106080001846FDF7C1F90346002836D001340190C7
:10609000F9F7D6FB019B42B2E4B218460192FDF734
:1060A000B3F9019A034650B30134E4B2032C28D863
:1060B00003B0BDE8F04FFEF741BE04468146B4E7A9
:1060C0006145C2D0A3F13002D2B2092A05D9A3F1A9
:1060D0006102052A07D8573BDAB2360146EA18763C
:1060E00042EA0818ABE7A3F14102052AADD8373BD5
:1060F000F2E78346B6E78246C2E70246CDE7274B82
:10610000D4E71FFA89F10229D2D80BF2262189B2ED
:10611000B1F5E16FCCD80AF2262189B2B1F5E16F71
:10612000C6D8D4B2062CC3D81846019340F06AFEF4
:106130000428BDD8002FBBD02DB2164A019B6801A0
:1061400002EB451102F8009002EB4512A1F810B0E5
:10615000A1F812A015320C75114DC1E90286591E25
:10616000033311F8010F445D04F00304022C08BF4F
:10617000203802F8010B087808B18B42F1D103B046
:10618000BDE8F08F07223946064803B0BDE8F04F5E
:10619000FEF704BF9897012073B706083CD40608A1
:1061A000691807088AB906082DE9F04F804689B0BA
:1061B00017460C4615460026DFF89C90002F48D065
:1061C000687A627AB5F90AC08242B5F90CE095F8AE
:1061D00008A0D5E900B33AD122685A4537D16268A0
:1061E0009A4234D1B4F90A20624530D1B4F90C2076
:1061F00072452CD1217AA1EB0A02514251414A4603
:106200000791CDE9020CCDE900B340463346CDE914
:1062100004EAFFF7D3F90799237A4A464046103536
:106220000593B4F90C300493B4F90A300393637AFC
:1062300002936368019354F8103B00933346013690
:10624000FFF7A2F9112EB9D109B0BDE8F08F0021F6
:10625000D5E73946E0E700BF97B906082DE9F74FC3
:106260000446FCF7DDFE054630B100224E49012010
:1062700003B0BDE8F04F97E74C492046F9F776F8B0
:1062800030B94FF0FF3003B0BDE8F04F36F018B929
:106290002046F9F7D5FA8346C3B2102B07D910224E
:1062A0002946434803B0BDE8F04FFEF777BE2046CD
:1062B000FDF7AAF80646E8B1F9F7C2FA01248246CA
:1062C0003046FDF7A1F80646B8B10134F9F7B8FA3F
:1062D0008146E4B23046FDF797F8064600285CD0C8
:1062E000F9F7AEFA0128804609D903B0BDE8F04FAE
:1062F000FEF724BD04468246E2E78146EAE7013420
:10630000E4B23046FDF780F80646002847D0F9F79A
:1063100097FA00F5B4730746B3F5347FE5D8013436
:10632000E4B23046FDF770F80346002839D00190FA
:10633000F9F786FA00F5B4720646B2F5347FD4D880
:106340000134019BE4B21846FDF75EF8034640B104
:1063500001340190F9F774FA051EE4B2019B18BFED
:1063600001251846FDF750F808B10134E4B2062CB7
:10637000BBD14FFA8BFB0F4B03EB0B13C3F810AFE2
:10638000C3F8149F83F8198FA3F81A7FA3F81C6F22
:1063900083F8185F03B0BDE8F08F8046B1E7074689
:1063A000BFE70646CFE700BF5800022073B70608D4
:1063B000B7B9060848F101202DE9F047814686B0BB
:1063C00090460D4617460026DFF868A0B8F1000F8A
:1063D0002DD03B782A789A42D7E9010C25D16A68FA
:1063E000824222D1AC68A4EB0C02544254412146B3
:1063F0000093524633460594CDE9010C4846FFF719
:10640000DDF80599AB68524648460C3702936B6835
:10641000019315F80C3B009333460136FFF7B4F8AF
:10642000082ED3D106B0BDE8F0870024DFE741464F
:10643000E8E700BFC8B906082DE9F8430446FCF7B1
:10644000EFFD054628B100222D490120BDE8F843A3
:10645000B2E72C492046F8F789FF014628B96022A7
:106460002748BDE8F84348F07DBF2046F9F7E8F932
:106470000646C3B2072B06D9294607222248BDE8A3
:10648000F843FEF78BBD2046FCF7BEFF074630B34E
:10649000F9F7D6F9051E4FF0010418BF012538465B
:1064A000FCF7B2FF0746E0B10134F9F7C9F98046BD
:1064B000E4B23846FCF7A8FF0746A0B10134F9F76B
:1064C000BFF98146E4B23846FCF79EFF08B10134BB
:1064D000E4B2032C09D0BDE8F843FEF72FBC044614
:1064E000DDE78046E5E78146EDE776B2074B0C2015
:1064F00000FB063606F8D85C46E93589BDE8F88326
:106500006801022073B70608DDB9060840020220C0
:106510002DE9F04F91B007468846164600240DF14C
:106520002C0ADFF8789004EB8405514608EB05034C
:1065300058F805001B79029002A88DF80C303BF04A
:1065400095FB4EB373197059052204A91B790DF1FF
:10655000180B049002A88DF8143049F043FEB0FAED
:1065600080F5594604A86D093BF080FB23464A4656
:1065700029463846CDF800B0FFF720F8234601340D
:106580004A4629463846CDF800A0FEF7FDFF802C8C
:10659000C9D111B0BDE8F08F3546EFE7ECB9060878
:1065A0002DE9F04F89B00546FCF73AFD044630B1BD
:1065B00000226749012009B0BDE8F04FA8E728464E
:1065C000F9F73EF97F28074600F3BA802846A2462D
:1065D000FCF71AFF5E4ABB0006462546A346039316
:1065E00007EB8703A046A146D118D450594B0C7134
:1065F00002930194029B05AA13F801CB96460293DD
:106600000023304616F8011B19B18C4501D00A2B26
:106610000CD120334FF000068C456B4403F80C6C12
:1066200008D009B0BDE8F04FFEF788BB01330EF883
:10663000011BE6E709F1FF33461C032B03D8DFE813
:1066400003F02D446D7605A8F9F7FAF8019009F1E9
:1066500001095FFA89F9B9F1050FCBD1039A05F069
:106660000F003D4B04F00F043A44019944EA08142A
:1066700017469A18783B40EA01104FEA281802F8AA
:1066800077BC1F4402F8780C02F876ACFC7087F8EF
:10669000048009B0BDE8F04F27F0EEBF05A8F9F778
:1066A000CFF80546D3E74E2B14D0452B14D0532BEF
:1066B00014D0572B14D0552B14D0442B05D10523BF
:1066C000012101FA03F348EA030812F8013B002B09
:1066D000E9D1BCE70023F3E70123F1E70223EFE769
:1066E0000323EDE70423EBE7DFF874C0002319462A
:1066F0001CF8013B834204D0072901F10103F6D1C4
:106700005946DFF860C000231CF801EB70450AD140
:10671000012000FA03F34AEA030A8B4612F8010B40
:106720000028E1D193E70133072BEDD1F5E705A868
:10673000F9F786F810280446B4BF0446002486E71B
:106740007F222146054809B0BDE8F04FFEF726BC80
:10675000C80102201C1F060840020220E6B90608F4
:10676000211F0608291F06082DE9F047814686B03B
:1067700090460D4616460027DFF860A0B8F1000FDE
:106780002AD033882A889A4224D16C887188621A68
:1067900054425441F2782146484605940292B27818
:1067A000CDE900323B465246FEF708FF0599EB78EB
:1067B0005246484604360293AB78019335F8043BC1
:1067C00000933B460137FEF7DFFE102FD6D106B00F
:1067D000BDE8F0870024DDE74146E8E7F6B90608A2
:1067E0002DE9F8430546FCF71BFC044628B10022BE
:1067F00025490120BDE8F843B6E72846F9F720F817
:106800000F28064630DCA0362846FCF7FDFD1F4F5A
:106810000546DFF884804FEA86092846F9F710F824
:1068200037F8023B984226DC012C08EB090311D013
:10683000022C12D023F8780C28462C2149F0F1FCC8
:10684000054668B1013501230134A3B1032CE4D11D
:10685000BDE8F88303F8760CEEE703F8750CEBE778
:10686000A21E53425341EFE721460F220848BDE8DC
:10687000F843FEF793BB074B002243F82620BDE800
:10688000F843FEF75BBA00BF48040220301F060839
:10689000E6B90608C8010220400202202DE9F04FA7
:1068A000144685B00646894600274FF0060B294A54
:1068B0000BFB07F54FF0000805F5307519F805A03A
:1068C000002C42D0635DAAEB0300414241413046B7
:1068D000CDE900833B460391FEF770FE03991D4A04
:1068E0003B4630460135CDE9008A08F10108FEF744
:1068F0004BFE184AB8F1060FE0D10137062FD7D169
:106900004FF43975134FA5F5397819F805A0F4B18E
:10691000635D3046AAEB0302514251413A46CDE94C
:10692000008306230391FEF749FE039906233A46A6
:1069300030460135CDE9008AFEF726FE40F2ED2310
:106940009D42E0D105B0BDE8F08F2146C8E7214661
:10695000ECE700BF08BA06082DE9F043804687B08F
:1069600017460C4615460026DFF88C90002F40D0C5
:10697000B5F90030B4F90010B5F902209942B5F923
:10698000040095F906C032D1B4F9021091422ED11B
:10699000B4F9041081422AD194F90610A1EB0C0E2F
:1069A000DEF1000141EB0E010591CDE90032CDE9A8
:1069B000020C33464A464046FEF700FE059994F91C
:1069C00006304A46404608350393B4F90430029332
:1069D000B4F90230019334F9083B00933346013691
:1069E000FEF7D2FD102EC1D107B0BDE8F083002123
:1069F000DAE73946E3E700BF1CBA06087FB505466B
:106A0000FCF70EFB00285ED000223049012004B0C4
:106A1000BDE87040A0E72D2B03D0A3F13002092A76
:106A20004CD8042C04DD04B0BDE87040FEF786B9F4
:106A30002846F8F705FF04AB621C03EB440424F876
:106A40000C0C15F8013F303B092BFAD914462B7872
:106A5000002BE0D1052CE6D1BDF80430BDF904606F
:106A60000F2BE0D8BDF90610A1F5FA7292B2B2F57B
:106A7000FA6FD8D8BDF90820A2F5FA7080B2B0F547
:106A8000FA6FD0D8BDF90A008142CCDC8242CADB61
:106A90009142C8DCBDF90C5005F17D04A4B2FA2C7A
:106AA000C1D80B4B03EBC603A3F87612A3F87822E8
:106AB000A3F87A0283F87C5204B070BD202BB2D1C7
:106AC00001352246C2E70446C1E700BFB6040220F2
:106AD000400202202DE9F04F80468FB017460C4649
:106AE00015460026DFF8A8B0A3882068ADF82C3042
:106AF0002378B4F902900893637894F905A006937B
:106B000023790A900793B9F1000F3AD0002F3DD0B6
:106B10002868BDF828100C9080B2AB8881422A7892
:106B2000ADF8343095F801C0B5F9023095F804E0BD
:106B30002AD14B4528D1BDF82C10BDF83400081AD5
:106B400041424141009240465A460991CDE901C374
:106B5000CDE903EA3346FEF731FD0999079B5A4612
:106B60004046CDF810A006340635CDE90293069BC9
:106B70000193089B009333460136FEF705FD202E56
:106B8000B2D10FB0BDE8F08F0021DBE73946E5E771
:106B900031BA0608F0B589B0044640F033F910F078
:106BA000FF020CD13A4B4FF4C8703A499B7800FB76
:106BB00003110120D03109B0BDE8F0408AE7052279
:106BC00035492046F8F7B6FBA8B9314B4FF4C871E8
:106BD00006269A782F4B01FB0233304AD0331568D2
:106BE000948806FB00F20130991820289D508C8073
:106BF000F7D109B0F0BD204601AA294902AD47F0FE
:106C000019FA00244FF0FF33254E079378B1062C74
:106C100002D1FEF793F8ECE7F8F712FE01AA45F867
:106C2000040B31460020013447F004FAEEE7042C4F
:106C3000EFDD029A1F2AECD8039E0F2EE9D8049D9F
:106C4000262DE6D8059C04F57A73B3F5FA6FE0D8E3
:106C50000698FF28DDD807994B1C402BD9D80C4B40
:106C60004FF4C8779B787B43062707FB02320D4B16
:106C7000134483F8B40C83F8B06C0B4883F8B15C10
:106C8000A3F8B24C83F8B51CFFF784FFB1E700BF4F
:106C9000BD91012028FD012073B70608361F0608A4
:106CA000380B070848F101203CD406082DE9F04FC5
:106CB00007469BB093460C4615460026DFF804A114
:106CC0000E930E9B5A1C01D0B3426FD1A6460DF114
:106CD000400C94F8048094F81390BEE80F00ACE8E0
:106CE0000F00DEF800300890CCF80030237B0992CA
:106CF0000A93237C0B9394F911300C93A37C0D938E
:106D0000BBF1000F5CD0AE460DF1540CBEE80F0095
:106D1000ACE80F00DEF80030149ACCF8003023F015
:106D20007F4322F07F420F9095F804E09A42A868D2
:106D300095F80CC0E97C41D1F0453FD1089B0F9AF2
:106D400093423BD10A9B634538D1099B834235D19D
:106D5000A9EB010359425941099B52463846CDF8E7
:106D60001C9006930A9B0F910593089BCDE9038322
:106D70000D9B02930C9B01930B9B00933346FEF7F4
:106D80001DFC0F99099B52463846CDF81C9006937E
:106D90000A9B0593089BCDE903830D9B02930C9BF3
:106DA00001930B9B00933346FEF7EEFB0136143440
:106DB0001435402E85D11BB0BDE8F08F0021CBE704
:106DC0005946DFE748BA06082DE9F0418AB0044683
:106DD0000D4640F017F810F0FF0210D13F4B93F82A
:106DE000A81541B94FF0FF330A463D4901200AB0CA
:106DF000BDE8F0415AE76B1C6CD02B46F5E7052245
:106E000038492046F8F796FA38B94FF47E7134487D
:106E10000AB0BDE8F0413FF005BB204601AD0024BB
:106E2000314E6A46304947F005F978B1092C02D154
:106E3000FDF784FF4EE0F8F703FD6A4645F8040BC2
:106E400031460020013447F0F5F8EEE7092CEFD188
:106E500001993F29ECD8DDF808E0BEF1010FE7D831
:106E6000DDF80CC00CF10103402BE1D8049F342F56
:106E7000DED8059E072EDBD8069D1C4A05F5742337
:106E800003F510739342D3D8079C072CD0D80898E9
:106E900000F5742303F510739342C9D8099AFF2AA9
:106EA000C6D8134B4FF0140808FB013309B2C3F8DE
:106EB000000383F808E30F4883F809C383F80A73D3
:106EC00083F8FC62C3F8F85283F8044383F80B2379
:106ED000FFF77AFF0AB0BDE8F08100BF48F101205A
:106EE0003805022073B70608380B070880841E0097
:106EF000400202203CD406084FF0FF3164E72DE940
:106F0000F04F1646154687B007460C464FF0000B6B
:106F1000194AD4F80880D4E9009A56B3AB6898456A
:106F2000D5E9000123D1814521D1AAEB01035942C2
:106F300059415B463846CDF800800591CDE9019A6C
:106F4000FEF73CFB05990C4A5B460BF1010B3846FA
:106F5000CDF800800C340C35CDE9019AFEF714FB16
:106F6000BBF1080F044AD4D107B0BDE8F08F00216F
:106F7000DFE73146E8E700BF69BA060870B586B0BA
:106F800004463FF03FFF10F0FF0205D120490120E9
:106F900006B0BDE87040B2E705221E492046F8F76A
:106FA000C9F938B940F2FF31194806B0BDE8704060
:106FB0003FF038BA204602AD0024174E01AA164908
:106FC00047F038F878B1042C02D1FDF7B7FE1CE089
:106FD000F8F736FC01AA45F8040B314600200134CD
:106FE00047F028F8EEE7042CEFD1029B072BECD8F2
:106FF0000C22074903985343CA1890600498C8505C
:10700000059B06485360FFF7B9FF06B070BD00BF8F
:107010007093012073B70608380B07083CD40608A4
:107020002DE9F04F8046A1B017460C4615460026C4
:10703000DFF8F8B0A6460DF1480C94F80C9094F8DF
:1070400018A0BEE80F00ACE80F0023680C9323796A
:107050000A93A3680B93238A0D93638A0E93A38AE2
:107060009EE807000F93E38A8CE807001093002F37
:107070005AD0AE460DF1640CBEE80F00ACE80F002C
:107080002B7E9EE8070053458CE807004AD12B79F8
:107090000A9A934246D12B680C9A9A4242D12B7B92
:1070A0004B453FD1AB680B9A9A423BD1169A82422C
:1070B00038D117991E9BCB1A59425941109B5A46F9
:1070C0004046119108930F9B07930E9B06930D9BCF
:1070D00005930B9BCDE903930C9B02930A9BCDE98F
:1070E00000A33346FEF76AFA1199109B5A464046B0
:1070F0001C3408931C350F9B07930E9B06930D9B26
:1071000005930B9BCDE903930C9B02930A9BCDE95E
:1071100000A333460136FEF737FA042E8AD121B098
:10712000BDE8F08F0021C9E73946DEE77ABA0608E4
:107130002DE9F0438DB004463FF064FE10F0FF02ED
:1071400005D13E4901200DB0BDE8F04368E70522B6
:107150003B492046F8F7EEF838B94FF47E713748CE
:107160000DB0BDE8F0433FF05DB9204602AD00240C
:10717000344E01AA334946F05DFF78B10A2C02D1A2
:10718000FDF7DCFD57E0F8F75BFB01AA45F8040BBF
:1071900031460020013446F04DFFEEE70A2CEFD1D6
:1071A000DDF80880B8F1030FEAD8DDF80CE0BEF195
:1071B000010FE5D8DDF810C0BCF1070FE0D8059F3E
:1071C000214B07F5742202F510729A42D8D8069E18
:1071D000072ED5D8079D05F5742202F510729A4244
:1071E000CED8089CB4F5004FCAD20998B0F5004F2C
:1071F000C6D20A99B1F5004FC2D20B9AB2F5004F30
:10720000BED2124B4FF01C0909FB0833A3F80A0841
:1072100083F810E80E4883F8FCC7C3F8F87783F8C2
:107220000468C3F80058A3F80848A3F80C18A3F89A
:107230000E28FFF77DFF0DB0BDE8F083380A02206D
:1072400073B70608380B070880841E00400202202E
:107250003CD406082DE9F04FA1B00646154600249F
:1072600014AFDFF844810D910D9A63010DF1400ECA
:1072700002EB441202F120091068083252F8041C93
:10728000F4464A45ACE80300E646F5D1002D00F08F
:1072900089802B440DF1600C03F1200E186808332F
:1072A00053F8041C6246734503C29446F6D19DF818
:1072B00040309DF860100A930A98BDF84230814230
:1072C000BDF846900B939DF844309DF848A00C9370
:1072D000BDF84AB09DF84C30BDF84E2060D1BDF8E5
:1072E00062100B9881425BD19DF864100C9881422A
:1072F00056D1BDF86610494552D19DF868105145E8
:107300004ED1BDF86A1059454AD19DF86C1099428A
:1073100046D1BDF86E10914242D11CA93846CDE944
:107320000E323FF065FDB0FA80F1DDE90E32490919
:107330003046CDE905B30C9B02930B9B01930A9B4E
:107340000A9100932346CDE90727CDE9039A4246E7
:10735000FEF734F90A99BDF84E3042463046089798
:1073600007939DF84C300693BDF84A3005939DF87D
:1073700048300493BDF8463003939DF8443002939F
:10738000BDF8423001939DF840300093234601340C
:10739000FEF7FAF8032C7FF467AF21B0BDE8F08F59
:1073A0000021C5E72946D6E79CBA06082DE9F04139
:1073B00090B004463FF026FD10F0FF0205D146498B
:1073C000012010B0BDE8F04144E706AE01AA4349F0
:1073D000204635460024424F46F02CFE6A4640497E
:1073E00046F028FE00286FD0092C62D101AA3B4943
:1073F000002046F01FFE064600286AD03FF002FD3E
:107400000F28044628BF0F2420B12246314602A887
:1074100045F000FE04F14003DDF818800DEB030495
:10742000B8F1020F4FF0000304F8383C4ED8DDF8F5
:107430001CE0BEF1070F49D8DDF820C0BCF1FF0FFA
:1074400044D8099F072F41D80A9EFF2E3ED80B9C97
:10745000072C3BD80C98FF2838D80D99022935D82D
:107460000E9AFF2A32D81F4B03EB481383F870485B
:1074700002AC83F868E803F6780323F80ECC03F82F
:107480000C7C23F80A6C23F8060C03F8041C23F880
:10749000022C2246083303CAAA4243F8080C43F8D8
:1074A000041C1446F5D11048FFF780FF10B0BDE86A
:1074B000F081F8F7C5F96A4646F8040B3946002012
:1074C000013446F0B7FD8DE7092C8FD0FDF736FC6F
:1074D000ECE704469EE700BFA80A0220C5D40608D0
:1074E000380B0708400202203CD406082DE9F04F73
:1074F000064685B0894615461F460024DFF858A089
:10750000DFF858B0002F01DBA7421DD119F8048025
:1075100005B32B5D3046A8EB03020AEB830351420F
:10752000D3F8CC33514100935A4623460391FEF7DA
:1075300045F803990AEB88085A463046D8F8CC3308
:1075400000932346FEF720F801340E2CDAD105B063
:10755000BDE8F08F2946EDE7701B0608D0BA060893
:107560002DE9F04385B0002425494FF0FF3903AAE7
:10757000254646F05FFD234E0246234FDFF89080FC
:1075800042B9012D35DD022D07D120494B4601F8C6
:10759000094030E035B1012D12D0FDF7CFFB05B029
:1075A000BDE8F0831046F8F74BF90D288146F4D872
:1075B00003AA13490020013546F03CFD0246DFE7EF
:1075C000114630460192F7F7D1FE019A0446002891
:1075D000EED011463846F7F7C9FE019A38B1114688
:1075E0004046F7F7C3FE0028D7D10224E0E72C4637
:1075F000DEE74B4605490120FFF778FFCFE700BFE4
:10760000380B0708E8BA06085ED30608A9780120F7
:107610002BFB06080FB407B504A951F8040B019120
:10762000FDF7CCFA03B05DF804EB04B07047F7B592
:107630008479054614F0C00303D0402B18D003B062
:10764000F0BD04F0070410F0D7FA062C05D101466E
:10765000164803B0BDE8F040DCE70190284610F082
:10766000BAFA019A0146124803B0BDE8F040D1E7EA
:107670000024104E104F10F04FFB05460F48FDF749
:10768000E5F92B79A34204D803B0BDE8F040FDF73B
:1076900085BA14B13046FDF7D9F92B68384653F84E
:1076A00024100134FBF796FEEBE700BFEDBA0608A5
:1076B000FDBA060824BB060875BC060814BB0608FC
:1076C0002DE9F0478CB0074610F8013B202BFAD08B
:1076D00000251F4CDFF880802E46DFF88090DFF811
:1076E00080A06946204610F089F93946684648F07E
:1076F000F2FDE0B169464046FBF76CFE494668463C
:107700003FF076FBF8B9204610F058FA114B0146CD
:10771000007820280CBF50461846FBF75BFE013668
:10772000FDF73CFA2046FFF782FFFDF737FA0135F7
:1077300040F266230B349D42D3D10EB93AF0ECFAF5
:107740000CB0BDE8F08700212046FDF7EBFAE6E734
:107750001F250608F1B70608E8B706080213070850
:10776000CBBA06082DE9F04F2DED028B8FB00578CE
:1077700006460130202DFAD030463FF043FB044648
:1077800018B1012821D12A2D1FD1934D0026DFF8F1
:10779000648240F266279148FDF722FE284602A93E
:1077A00010F02CF9013602A94046FBF713FE2846DB
:1077B00021460B35FDF7B6FAFDF7F0F9BE42EDD1E3
:1077C0000FB0BDEC028BBDE8F08F3D21304648F094
:1077D00028FD002800F0F9800346994613F8012D92
:1077E000202AFAD0A9EB060901308046074610F896
:1077F000013B202BF9D0784D4FF0000A5FFA89F950
:1078000040F2662B02A9284610F0F8F802A83FF0D3
:10781000F9FA02A9024601903046F7F78BFD6E4B4C
:10782000044658BB019A4A4528D10B2202FB0A3371
:107830009B7903F00706062E36D140463FF0E2FA68
:107840008442064622D3664902A83FF0D1FA20B10D
:10785000644902A83FF0CCFA18BB98F80030222BFC
:107860001FD108EB060313F8013C222B19D1B21EDD
:1078700008F10101284610F06BFAA1E70AF1010AAC
:107880000B35DA45BED13AF047FA99E718F80430DB
:10789000A3F16102192A9CBF203B08F8043001348F
:1078A000CBE732464146E5E713F0C0030AD0402B50
:1078B0005BD04D48FDF754FE2846FFF7B8FEFDF7B4
:1078C0006DF97DE798F80030002BF2D0474940462B
:1078D00048F0F1FC044640463FF094FA8442E8D177
:1078E0004046F7F721FF2846B0EE408A10F073F9C2
:1078F00007EE900AF8EEE77AF4EEC87AF1EE10FAA5
:10790000D7D8284610F078F907EE900AF8EE677A93
:10791000F4EEC87AF1EE10FACBDB052E0BD118EE9F
:10792000104A284610F04AF9052E3FD8DFE806F045
:107930003D3D4747494B042E12D13A4617F8013BCB
:10794000202BFAD0092BF8D0013A00240A2112F892
:10795000013F303BDBB2092BE3D801FB0434F6E7EF
:107960004046F7F76DFF0446DBE72846274610F050
:10797000D3F9A246814690F804B02346BB4500D90E
:107980001BB1BAF1000F94D0CBE7D9F800304146D3
:1079900053F82700F7F7EAFC002805BF3C4601230F
:1079A00000234FF0010A0137E8E7047002A91048EC
:1079B000FBF710FD00212846FDF7B4F900E704802D
:1079C000F4E70460F2E70460F0E730460FB0BDEC86
:1079D000028BBDE8F04F73E61F25060826BB06089C
:1079E0000213070838BB06085CBB060843BB060841
:1079F00051BB0608E8B7060870B586B00346FBF72A
:107A00000FFB044638B100221949012006B0BDE839
:107A10007040FEF743BF03AD164E02AA1549184643
:107A200046F008FB80B1032C03D1FDF787F906B0BF
:107A300070BDF7F705FF02AA45F8040B3146002098
:107A4000013446F0F7FAEDE7032CEED1059BDDE9B2
:107A500003451A4601932946E0B226F06BFF002841
:107A6000E3D0019B2A4621460348FFF7D3FDDEE71A
:107A7000C8010220380B070808BA060810B50346EB
:107A8000FBF7CEFA30B1FAF791FF0848BDE8104095
:107A9000FDF7A6BC1846F7F7D3FE044680B2FBF705
:107AA000E5F921460248BDE81040B3E56CBB060885
:107AB00078BB060808B50346FBF7B2FA40B10C4B99
:107AC00000220C48A3F8CA25BDE80840FDF788BC91
:107AD0001846F7F7B5FE014630B1054BA3F8CA05C5
:107AE0000548BDE8084095E5BDE80840FDF726B922
:107AF00048F101208ABB0608A0BB06082DE9F04327
:107B000085B0F8F753FB826804462AB9224805B0CD
:107B1000BDE8F043FDF764BC83890025018801922C
:107B200042881E4EDFF888801D4FDFF88890009253
:107B300042681C48FFF76EFD15B94046FDF750FC42
:107B40003B689D4215DA3378294601351648062BE5
:107B500006F1060696BF09EB83030022D3F8DC2367
:107B600036F8023C009336F8043CFFF753FD092D2C
:107B7000E2D10220F8F724FB81884388CB1A6168A0
:107B800003FB0111039125F007FA03990246074808
:107B900005B0BDE8F0433DE548B806080888012077
:107BA00040880120B7BB060810BC06081FBC0608A9
:107BB00005BC0608701B06082DE9F84305463FF092
:107BC00021F90446D0B9304B0127304DDFF8C88089
:107BD0002F481E68FCF73AFF55F8041B51B10B788B
:107BE00033B107FA04F3334202D04046FBF7F2FB0D
:107BF0000134F1E7BDE8F843FCF7D0BF0246254960
:107C00002846F7F797FB78B9204C234D2348FCF71B
:107C10001DFF54F8041B0029ECD00B78002BF8D082
:107C20002846FBF7D7FBF4E72B780026DFF85C90BB
:107C30002D2B03BF013504F1FF344FF001084FF045
:107C4000000859F8047B1FB9BDE8F8433AF064B85E
:107C5000224639462846F7F76DFB90B90120B0401F
:107C6000B8F1000F09D0F7F72BFF0D48FCF7EEFE37
:107C700039460C48BDE8F843CCE4F7F717FF0A484B
:107C8000F4E70136DDE700BF4C840120681F0608D9
:107C90003CBC060896CA0608FE0E070846BC060845
:107CA00052BC060875BC06085BBC06082DE9F84FF7
:107CB000344F05463FF0A6F80446BE68C8B9324DB9
:107CC0000127DFF8D4803148FCF7C0FEE3B205EBB2
:107CD0008302D2F87C1441B107FA03F3334202D095
:107CE0004046FBF777FB0134F0E7BDE8F84FFCF7BF
:107CF00055BF024626492846F7F71CFB60B9254CBC
:107D0000254D2648FCF7A2FE54F8041B0029ECD0B0
:107D10002846FBF75FFBF7E72B784FF00009DFF809
:107D200074B02D2B03BF013504F1FF344FF0010A6D
:107D30004FF0000A5BF8048BB8F1000F03D1BDE8E7
:107D4000F84F39F0E9BF224641462846F7F7F2FAE4
:107D5000A0B9012303FA09F3BAF1000F0AD026EA09
:107D600003030F48BB60FCF771FE41460D48BDE8B8
:107D7000F84F4FE433430C48BB60F4E709F10109C5
:107D8000D8E700BF1C950120701B06083CBC060804
:107D900096CA0608EC1F0608FE0E070846BC060831
:107DA00052BC060875BC06085BBC06082DE9F04706
:107DB0004E4E81463FF026F80446376800BB4C4DD6
:107DC0004FF00C084B4E4C48FBF704FB08FB04F348
:107DD0005B5D5A1E012393403B4206D0204618F0BB
:107DE00019FD01463046FBF7F5FA0134182CEDD1A8
:107DF00017B94248FCF72AFEBDE8F047FCF7CEBEB3
:107E000002463F494846F7F795FA054678B92C46A9
:107E1000384D3C48FCF71AFE2046013418F0FAFCB5
:107E200001462846FBF7D6FA1A2CF5D1E4E799F873
:107E300000304FF000082D2B03BF09F1010904F1B8
:107E4000FF344FF0010A4FF0000A404618F0E2FC00
:107E50002246054601464846F7F76CFA00283BD112
:107E6000BAF1000F1FD0B8F1180F0BD16FF07F439C
:107E700033602548FCF7EAFD29462448BDE8F04771
:107E8000FFF7C8BBB8F1190F01D17368F0E7204BB9
:107E90000C2202FB083898F8B4345A1E0123934090
:107EA0001F433760E5E7B8F1180F03D1C6F800A00B
:107EB0001848DFE7B8F1190F01D17760F8E7144BE4
:107EC0000C2202FB083898F8B4345A1E0123934060
:107ED00027EA03073760EBE708F10108B8F11A0F4A
:107EE000B3D1BDE8F04739F017BF00BFAC94012013
:107EF0002420060874BC060863BC06086DBC06088E
:107F000096CA060879BC060852BC060875BC060865
:107F1000701B06085BBC0608F0B585B004463EF051
:107F200071FF04283DD1631E2546E11C13F8012F83
:107F3000A2F16100192898BF203A8B421A70F5D13E
:107F4000261D1A4F15F8011B3846019148F069F9B2
:107F500020B10199284648F064F920B105B0BDE888
:107F6000F040FCF7EBBEB542ECD120461DF07CFDA5
:107F70000F48FCF76BFD0F4C0C4901231A5D0133D0
:107F800011F8010B1032052B6A4402F8080CF5D1E8
:107F9000002302A908488DF80C30FFF73BFB05B021
:107FA000F0BD0028E4D0FCF7C9FEE1E75C2106083B
:107FB00084BC0608F2F60120F1B70608F7B50346BF
:107FC000FBF72EF8044620B103B0BDE8F040FCF703
:107FD000B5BE264625461D4F01AA1C49184646F047
:107FE00029F840B90B2D18D901460B221848FCF787
:107FF000D5FF03B0F0BD44B1012C0AD001AA394627
:108000000020013446F016F8EBE7F7F719FC0546B7
:10801000F4E7F7F715FC0646F0E7022C0DD1A6F5BC
:108020007A73B3F57A7F05D94FF4FA624FF47A7117
:108030000848DCE7084B23F81560074B294607483A
:1080400033F91520FFF7E6FAD3E700BF380B07082E
:10805000E6B906081CD70608501100208ABC06089D
:1080600070B50346FAF7DCFFC0B11F4B9E690136BD
:108070003046344618F0CEFB0546E8B901341A2CD8
:10808000A8BF0024204618F0C5FB0546A0B9B4429D
:10809000F4D11648BDE87040FDF7A2B91846F7F7CD
:1080A000CFFB044618F0B6FB054628B92146104818
:1080B000BDE87040FFF7AEBA0B4B9C6119F066FA51
:1080C0000C4821462A46FFF7A5FA192C9BBF0A48FF
:1080D0000C21002001FB0400BDE8704098BF90F81F
:1080E000B40419F06BBA00BFF420012097BC060855
:1080F000ABBC0608C1BC0608701B060810B50346D9
:108100000C4C1846FAF78CFF38B10B4B0B4819781A
:10811000BDE810400131FFF77DBA1846F7F790FB34
:108120000138022804D8C0B203F0C2FB2346E8E7B6
:1081300010BD00BF3CD40608BD91012014BD060847
:10814000022810B50C4618D803F04AF90B48FDF781
:108150004EF90B4B0B4819780131FFF75BFA2146BA
:108160000820FDF771F821461020FDF76DF8214633
:108170002820BDE81040FDF767B810BD0BCA0608FF
:10818000BD91012079C2060810B503460C4C184673
:10819000FAF746FF38B10B4B0B485978BDE8104051
:1081A0000131FFF737BA1846F7F74AFB01380228C2
:1081B00004D8C0B203F08FFB2346E8E710BD00BF30
:1081C0003CD40608BD910120D6BC0608022810B593
:1081D0000C4610D803F05AF90748FDF708F9074B89
:1081E000074859780131FFF715FA21461820BDE8F4
:1081F0001040FDF729B810BDE9BC0608BD9101206B
:10820000F9BC060810B503460C4C1846FAF708FFEF
:1082100038B10B4B0B489978BDE810400131FFF79E
:10822000F9B91846F7F70CFB0138012804D8C0B299
:1082300003F064FB2346E8E710BD00BF3CD406080A
:10824000BD9101200EBD06082DE9F04FBB4BA1B03A
:10825000BB4A00250293BB4BBB490193BB4BBC48B7
:108260000093BC4BFFF7D6F9BB49BC48FFF7D2F9E6
:10827000BB4BBC4819684FF47A73BB4CBB4E04F23D
:108280000468DFF8949304F5C46AB1FBF3F1FFF7D7
:10829000C1F908A8F7F766F9B54B08A914A8B3F90E
:1082A00000203BF069FE14A9B248FFF7B3F91EF0B5
:1082B00059F9B14B64221B78B0FBF2F104EB830354
:1082C00002FB110289B2AD48D3F8F43592B20093A3
:1082D000AB4B1B78FFF79EF9AA4B3168AA48B1FB5C
:1082E000F3F1FBF777F8A94B1F680123AB403B4242
:1082F0000BD058F8253043B119F805205AF825104D
:1083000053F82220A248FBF765F80135072DECD180
:108310009C4DFCF743FC9F48FDF762F8F2F762F8CA
:10832000B0FBF5F19C48FFF775F931689B48B1FB4C
:10833000F5F1FFF76FF9F2F78FF8B0FBF5F1984818
:10834000FFF768F9F2F7A2F8B0FBF5F19548FFF7EF
:1083500061F91EF0F7FC04EB8000D0F84816079195
:108360001EF0FAFC04EB8000D0F8482606921EF0BE
:1083700003FD04EB8000D0F8483605931EF020FD85
:1083800004EB8000D0F848761EF03CFD05461EF058
:1083900083FD06461EF068FD04EB8000079904EBA0
:1083A0008606D0F8480604EB85050390D6F8480603
:1083B0000290D5F84806DDE90532CDE900707A482B
:1083C000FFF728F9794B1B68DB0317D5784B1E782C
:1083D000A6B10025774F31467748FFF71BF9E8B281
:1083E0001FF098F829460135B0F902203846FAF70F
:1083F000F1FFEBB2B342F2D3FCF7D0FB6F4B704A04
:108400001D88704B7049ADB21B687048C3F500738E
:10841000DFF808826E4F9B006E4EFFF7FBF86E4A46
:108420006E4B29466E480425D31A6E4ADFF8F0A138
:108430001288DFF8F0B1FFF7EDF8DFF8EC916A4849
:10844000FCF7CEFF58F8041B5046FAF7C3FF584616
:10845000FCF7FCFA17F8011B002940F09D816348E6
:10846000FCF7F4FA6248FCF7F1FA56F8041B00290D
:1084700040F096815D48FCF7B3FF013DE2D15D4BD2
:108480005D48198BFAF7A6FF5C490A6F5AB107EEEF
:10849000902ADFED5B6AF8EEE77A86EEA77AFDEECA
:1084A000C77A17EE902AD1F800315BB107EE903A07
:1084B000DFED536AF8EEE77A86EEA77AFDEEC77A2B
:1084C00017EE903A896A59B107EE901ADFED4C6ABF
:1084D000F8EEE77A86EEA77AFDEEC77A17EE901AE5
:1084E000484E4FF0010848480091484FB6F8C81868
:1084F000FFF790F84648FCF7A9FA3D68DFF82C91A1
:1085000025F0004525F07F05002D40F04D81FCF75A
:1085100045FB3B685F0140F194800BA80FF082FBA4
:10852000002840F08E800B9B40F2652214A99342F4
:108530009ABF38480B2528467AE000BF80B106086C
:10854000A4B1060889B106087BB0060892B10608F6
:10855000E8C106089EB1060852BD060800C206081A
:10856000883301206CBD0608701B0608BC01012081
:108570004884012086BD060805A3012097BD060892
:1085800006A3012040420F00BCBD060840010020A8
:10859000CCBD0608D4BD0608E9BD0608FBBD06082B
:1085A0000DBE06081FBE060831BE060804000020E6
:1085B0002C000020A9BE060884BE0608C42B01209A
:1085C00000000120B07B012000180000B8BE0608A2
:1085D00028950120FC770120008000080040000859
:1085E000F0BE0608B87801202ABF06086FBC06084E
:1085F0005BBF06085011002065BF0608D81801208F
:10860000002474494002022075BF060808000020BB
:10861000B2BF06081F2506089C960120C82106083F
:108620003DBF060845BF060854BF060875BC0608CE
:1086300098BF05FB03000FF0E1F914A97148FCF79E
:10864000D1FA7148FCF702FA704B1968002900F062
:10865000BE800B7B4A7B6E488968FAF7BBFE6D4D86
:10866000FCF79CFA6C48FCF7F1F92868FCF788F9EC
:10867000002800F0B0800BA92868FCF7CAF99DF823
:1086800040109DF84C30129A6448FAF7A3FE0F99F7
:1086900011B16348FAF79EFE0D9911B16148FAF7DE
:1086A00099FEFCF77BFA604B1B68180667D55F4B99
:1086B0001B78012B63D85E48FCF7C8F95D48C36896
:1086C000B3F5487F00F0958000F28980B3F5167FFE
:1086D00000F09180B3F52F7F00F08F805649574A04
:1086E000B3F5FA7F08BF1146437C027CC07C0728A3
:1086F00096BF04EB80000020D0F8C80600905048D8
:10870000FAF768FEFCF74AFA4E48FEF783FF4E4838
:10871000FCF766FE4D48FCF763FE96F8CC38190767
:108720000AD596F8D42896F8D518C2F3C00248485E
:10873000C1F3C001FEF76EFF96F8CC385A070AD590
:1087400096F8D42896F8D518C2F380024148C1F3B0
:108750008001FEF75FFF96F8CC389B070AD596F8A4
:10876000D42896F8D518C2F340023B48C1F3400123
:10877000FEF750FF96F8D0183848FEF74BFF384BFD
:108780001B7833B104EB83043648D4F8E816FEF7BF
:1087900041FF21B0BDE8F08F4846FAF71BFE61E6C5
:1087A0004846FEF737FF68E695FAA5F3B3FA83F378
:1087B00008FA03F2062B25EA02057FF7A5AE04EBC3
:1087C00083034846D3F84C16FAF704FE9CE6264885
:1087D000FCF73CF943E72548FCF738F961E7B3F5C6
:1087E000617F0CD01449224AB3F57A7F08BF114645
:1087F0007AE7204978E7204976E7204974E720495D
:1088000072E700BFC9BF0608DDBF060828A4012023
:10881000E3BF060880A20120FCBF060802C00608CC
:1088200020C0060829C006084C840120DC950120E0
:1088300045C00608A89501201FBD060835BD0608DD
:108840004BC0060872C0060887C00608A8C0060804
:10885000B4C00608C6C00608D7C00608E9C00608A6
:10886000DC93012000C10608F0BF060838C00608E6
:108870004ABD060827BD06082EBD060843BD0608EA
:108880003CBD06082DE9F04F00274E4D4E48B94635
:10889000BA462DED028B9FED4D8A8BB0FEF7BAFEE6
:1088A0004B4BD96903F1200200238B4226DB0137B1
:1088B00048351A2FF4D146494FF47A73D1E925028D
:1088C000D1F88C404009D1F89C10B4FBF3F340EA96
:1088D000C2624048FEF79EFE0A2299FBF2F39AFB21
:1088E000F2F102FB139002FB11A200903A48FEF74E
:1088F00091FE0BB0BDEC028BBDE8F08F52F8040B7B
:10890000A84201D00133D0E7AC6A4CB107EE904ADF
:10891000B8EEE77AC8EE077AFDEEE77A17EE904AEE
:10892000AB6B4FEAE47BD5E90C6108934A09EB6B2A
:1089300076096343099246EAC166089AA4FB020CD1
:1089400002FB0B3141F288334FF47A72C0184FF0BA
:10895000000341EB0C013FF0CDF8099A804641F24B
:10896000883304FB02F14FF47A7206FB0B1BA4FB65
:108970000601C0184FF000034BEB01013FF0BAF8BD
:108980002B6C4FF47A72042F394601961CBF814438
:10899000C244B3FBF2F306930A2390FBF3F203FB0A
:1089A0001200CDE9042098FBF3F203FB12830B487D
:1089B000CDE90223089B2A6800932346FEF72AFE8E
:1089C00075E700BFD81801201AC1060800247449B1
:1089D0005011002096C10608B8C1060861C10608FA
:1089E0001FB5094B094A0293094B0A4901930A4BE7
:1089F0000A4800930A4BFEF70DFE0A490A4805B0E3
:108A00005DF804EBFEF706BE80B10608A4B10608C7
:108A100089B106087BB0060892B10608E6C10608CF
:108A20009EB1060852BD0608FEC10608F8B500242E
:108A30000B4D0C4E0C4F0D48FEF7ECFD6CB9326837
:108A4000C2F50072920022B157F824100848FEF7D0
:108A5000E1FD0134222CF1D1F8BD55F82420F2E7D4
:108A6000B4830120B07B01207022060807C20608EB
:108A70001DC206082DE9F3411A4C00251A4E1B4F62
:108A8000DFF870801A48FEF7C5FDE279216806EB31
:108A90008202A37901F13F4194F808C0D2F8880717
:108AA00006EB8303A28801F57E01D3F80037B2FA02
:108AB00082F2890AC2F11F024131BCF1000F0BD0D2
:108AC000CDE900C04046FEF7A5FD01350C34402D30
:108AD000DBD102B0BDE8F08100903846FEF79AFD88
:108AE000F3E700BF248C0120701B060857C206085C
:108AF0002BC2060847C206082DE9F843264D0C464E
:108B000002F0D4FC2548FCF772FCA97824484FF405
:108B1000C8770131DFF89C90FEF77CFD21462020CC
:108B200009F6D806FCF790FB1E48FCF760FCAB7812
:108B30001D4A204607FB0363DFF87C80D3ED047AEF
:108B4000F5EE407AF1EE10FA0CBF01210021FCF79E
:108B50001BFDA97820467943103108EB010231440E
:108B6000FCF7F4FF1148FCF742FCAB78104A2046B2
:108B700007FB0399B9F9AA19B1FA81F14909FCF780
:108B800003FDA97820467943D03108EB0102314436
:108B9000BDE8F843FDF79EBFBD91012065C2060800
:108BA00073C2060886C2060899C20608A8C206084B
:108BB000BBC206084002022028FD01202DE9F04F2B
:108BC0000D468DB0B4490446FAF762FC064600280B
:108BD00040F0B780B1492046FAF75AFC0646002813
:108BE00040F0B180AE492046FAF752FC0646002814
:108BF00040F0AB80AB492046FAF74AFC0646002815
:108C000040F0A5802046A849FAF742FC0028064615
:108C100012BF1024264601240DB144F02004A34DB8
:108C2000A34F95F800A095F8019095F80280DFF821
:108C3000ECB25F45C0F08D8002F0F2FB504602F0CE
:108C4000CFFB484602F022FC404602F02FFC994937
:108C50003046FAF71DFC08B144F0400414F011034B
:108C6000009300F0A1829448FCF7C1FB0020FFF7BD
:108C7000B7FE9248FCF7BBFB9148FCF7B1FB04F050
:108C80003003302B02D18F48FCF7B1FB8E484FF0F8
:108C9000000AFCF7ACFB8D48FCF7A9FB4FF0FF3353
:108CA0008B4A20468B49FEF721FC8B48FCF79FFB43
:108CB0008A4A2046DFF8689202F68211FDF74CFEE0
:108CC0008748FCF794FB874A2046CB4602F555615E
:108CD000FDF772FB8448FCF78AFB844A84492046EE
:108CE000FDF762FA8348FCF782FB834B834A1E68D8
:108CF000834B1F6867EA060301935BF8043B002B74
:108D000034D01978D1B14FF001080199204602936F
:108D100008FA0AF811EA080F14BF01210021FCF734
:108D20004DFC66EA0701754A204611EA080F029BCE
:108D300014BF01210021FCF727FC704A0AF1010A47
:108D4000DBE7012468E7022466E7042464E70824DB
:108D500062E77B88C3F30B021B04D7E9011048BF0D
:108D600002EB4202143744F055F962E79846654A2F
:108D700067EA0603019359F804BBBBF1000F26D044
:108D80009BF8001001B34FF0010A0AFA08FA17EA3B
:108D90000A0F0BD066EA07015B46204611EA0A0F6C
:108DA00014BF01210021FCF709FC564A16EA0A0FFC
:108DB0000AD0019B204613EA0A0F5B4614BF01212B
:108DC0000021FCF7E1FB4F4A08F10108D3E74E48C8
:108DD0005E46FCF70CFB4D4ADFF848A1D2F8009044
:108DE0004B4ADFF844B1126889EA02086FEA0808C2
:108DF00001273046B740013618EA070F14BF01219A
:108E0000002119EA0707039114BF52465A460192FE
:108E100017F000FD03990346019A02902046019144
:108E2000FCF7CCFB002F14BF5A465246029B019917
:108E30002046FCF7A9FB182EDAD136480026FCF7AD
:108E4000D6FA354BDFF8E4A09F68DFF8E480DFF85E
:108E5000E490F3B20AEB8302D2F87CB4BBF1000FCA
:108E60006AD0012199405B4639400CD04A46002126
:108E70002046FCF789FB5B464A4600212046013626
:108E8000FCF79CFBE5E7424620460191FCF77CFBA2
:108E90005B4642460199F1E7DDC206080BCA0608A7
:108EA000E9BC060865C20608E4C20608BD910120B7
:108EB0003C400708E8C2060820CE0608F5C20608AE
:108EC0000DC3060819C3060866CA060854C3060877
:108ED000A97801202DA4012064C30608B60402204D
:108EE00074C30608680102207DC3060858000220EA
:108EF000180F022048C80608F0AD012091C30608EB
:108F00004C8401209DC30608E4C60608B0AC0120CD
:108F1000AC940120A8C3060840AF0120784507089B
:108F2000681F0608C8C20608D2C20608701B0608D9
:108F3000BDC30608B1C30608A348FCF758FA0123CD
:108F4000A2481F46DFF844C3DFF844E38DF820B0A1
:108F50008DF810B08DF821B08DF811B08DF822B0D9
:108F60008DF812B08DF823B08DF813B013F80C20E3
:108F700010F8016B02F13001694401F8206C13F81C
:108F80000E1001F13008E84408F8106C2FB1A2EB84
:108F90000108D8F1000747EB08070133052BE5D19D
:108FA0000026394608AB8A4A20468DF81460FCF743
:108FB00005FB04AB3946864A2046FCF7E5FA8548AE
:108FC000FCF715FA844A85492046FCF7CBFB844818
:108FD000FCF70DFA834A204602F56861FDF798FA1E
:108FE0008148FCF704FA814A204602F56861FDF7E2
:108FF000BBFB7F48FCF7FBF97A4A204602F5686123
:10900000FDF74CFC7B48FCF7F2F97B4A7B49204694
:10901000FCF7EAFA7A48FCF7EAF97A4A7A492046F4
:10902000FCF7A4FC7948FCF7E2F9794A7949204633
:10903000FCF7ACFE7848FCF7DAF9784A7849204624
:10904000FCF740FF7748FCF7D2F97749204638F023
:1090500079FE7648FCF7CBF94FF0FF337449204690
:109060001A4638F0F7FE7348FCF7C1F94FF0FF33AA
:10907000714A20467149FDF719FE7148FCF7B7F9AE
:10908000704A71492046FDF73AFF7048FCF7AFF986
:109090006F4A70492046FDF7C3FF6F48FCF7A7F9F8
:1090A0006E4A6F492046FEF7D5F86E48FCF79FF9E7
:1090B00021463046FCF7C8F8E70665D5214630461C
:1090C00095F800806F7895F80290FFF715FD21461E
:1090D0000120FFF711FD21463046FFF731F8214608
:1090E0000120FFF72DF821460220FFF729F821463D
:1090F0003046FFF76BF821460120FFF767F821465D
:109100000220FFF763F8404602F06AF9384602F0A1
:10911000BDF9484602F0CAF95348FCF768F909F16D
:1091200001015248FEF776FA08F101015048FEF7B6
:1091300071FA791C4F48FEF76DFA200705D5A8781B
:10914000012802D82146FFF7D7FCA10703D5214605
:109150002878FEF7F5FF620703D521466878FFF708
:1091600035F8009B13B14448FCF741F92EB1434850
:10917000FCF73DF94248FCF733F9424C424DAC4212
:1091800014D30DB0BDE8F08FA878012802D821468D
:10919000FFF7B2FC21462878FEF7D2FF2146687817
:1091A0000126FFF713F8C8E7009EC6E76388C3F3FC
:1091B0000B021B04D4E9010148BF02EB4202143444
:1091C00043F028FFDBE700BFCAC306085C2106089E
:1091D000E0C30608E7C306088CA00120C4AE012046
:1091E000EDC30608C8010220F2C3060848040220A5
:1091F000FCC306080BC406080DFC01203613022030
:1092000017C40608ADFC0120D61302202EC40608A0
:10921000480002204E1402203FC4060898970120FF
:1092200098AB01204BC40608601402206AC40608EB
:10923000C01D02207BC406083805022070220220CF
:109240008EC406087093012028AB0120ACC4060828
:10925000380A022070270220C9C40608A80A022082
:10926000E0270220DDC20608DEC406080EBD06089F
:1092700014BD0608D6BC060801C506081AC50608AE
:1092800030C506083C40070878450708281002202A
:10929000F2F60120002191E401218FE408B5054890
:1092A000FBF7D4FB044BD3F8B801BDE80840F6F750
:1092B000DBBC00BFF4B7060848F10120704700BFCF
:1092C000114B014603F1180210B553F8044B9342B9
:1092D00041F8044BF9D11B880B8000F11A030A49AD
:1092E00051F8044B914243F8044BF9D111883430C2
:1092F0001980054B53F8041B934240F8041BF9D125
:109300001B88038010BD00BF843F0608104A117AF5
:10931000537A0B43D17C0B4351780B4391780B4329
:10932000D1780B4311790B43917B0B43917E0B4317
:1093300092F823100B4392F82F100B4305D192F8AB
:109340003D00013818BF012070470120704700BF61
:10935000C831022070B5244C05460E4694F84C30B6
:1093600043B1D4E91423904271EB030324BF0023DB
:1093700084F84C30E36E1D48984710F0010321D06B
:1093800080F00203C3F3400384F84C30D4E9183171
:109390005B1946EB0106C4E91436012384F88030DA
:1093A0004307D4F8880048BF0123A5EB000548BF58
:1093B00084F88130002D0EDD012084F8800000F05B
:1093C000010070BD8207EBD594F84C20002AE7D04D
:1093D00084F84C30E4E794F8803013B994F88100B5
:1093E000EDE70120EBE700BFC83102202032022068
:1093F000A0F2DC50164BB0F5FA7FA8BF4FF4FA701C
:10940000984210B5B8BF18460C46114638F025FEF4
:109410009FED107A00B2FBEE096AE4B207EE900A03
:10942000F8EEE77A87EE870A07EE904A9FED0A7A10
:10943000F8EE677AE0EE006AA7EEA67AF3EE097A14
:1094400020EE070A80EE270A40F0F6FF00B210BDBA
:109450000CFEFFFF0000C84200401C452DE9F0470C
:10946000854E864C70792DED028BB0EE408A68B344
:1094700027460025DFF8188206F13009DFF814A22C
:1094800096F82C30062202FB03832B441B7F4BB142
:10949000012B0BD001350237042DF1D1BDEC028B2D
:1094A000BDE8F08739F815303B80F3E7032D01D094
:1094B0000023F9E7DAF80030DA0404D40FF076FE7E
:1094C00000B2E080E6E740F2DC50FAE71CF0ECFA8C
:1094D0006B4FA368D7F8905013F4807897F89420D6
:1094E00014BF697B297AFFF783FF208001201CF0DD
:1094F000DBFAB8F1000F00F08280697B97F89420C6
:10950000FFF776FF608002201CF0CEFAB8F1000F62
:1095100077D0A97B97F89520FFF76AFF404200B209
:10952000A080B8F1000F6ED02288EB7B618813FB1E
:1095300002F3642293FBF2F323802B7C13FB01F3F1
:1095400093FBF2F363806B7C13FB00F090FBF2F073
:10955000A0800DF0A5FF3379E0802BB9B4F9043079
:109560002268B3863263F086A3685B0696D5B4F9A9
:109570001030F2EE046A07EE103AB7F9A030B8EEF8
:10958000C77A08EE103AB8EEC88AC7EE267A37EEE8
:10959000C88ADFED3C7ABDEEC88A18EE103A1BB2DD
:1095A00008EE103AB8EEC88A28EE278AB0EE480ACC
:1095B000F4F784FFF0EE408AB0EE480AF4F71CFF9F
:1095C000B4F9023007EE903AB4F9003006EE903A62
:1095D000F8EEE77AF8EEE66A26EE807AA7EEA87A49
:1095E00060EE677AE6EEA87ABDEEC77AFDEEE77A1E
:1095F00017EE903A238017EE103A63804EE7297AEF
:109600007CE7697A86E7204DB0EE480AB4F900009D
:1096100000212B78122B04BF1C4B186046F0C8FEAB
:109620002B7800B2B0EE480A122B4FF001012080D7
:1096300001BFB4F90220154B9A605860B4F90200DA
:1096400046F0B6FE2B7800B2B0EE480A122B4FF06F
:109650000201608001BF0D4BB4F90420D8601A618B
:10966000B4F9040046F0A4FE2B7800B2122BA080BF
:1096700004BF064B58616CE758990120F81100208F
:10968000C831022035FA8E3CE59101209CA30120CF
:10969000843F06080000002038B52C4B1B68580397
:1096A0004ED5D90608D42A4B30211A78294B01FB14
:1096B00002335B6CDA0544D4274B5D79002D3FD033
:1096C000264A926893073BD02DB20FF06FFD0446F7
:1096D0000EF034FD9FED227AF7EE007AB4EEC70A61
:1096E000F1EE10FA2FD4B4EE670AF1EE10FA37FE5D
:1096F000800A07EE105AC7EE806ADFED1A5A002181
:10970000164DB5F90630B8EEC77A1B1B87EE256AF1
:1097100076EEE76AE6EE867AB0EE677A07EE903A82
:10972000F8EEE76A07EE904AF8EEE77AE6EE877A17
:10973000FCEEE77A17EE903A98B20FF03DFEE88023
:1097400038BD6425C1E7B0EE470AD2E70400002027
:1097500030E00120843F0608BD910120F81100206F
:109760009A99193F0000C842F8B5734B0E4605465A
:109770001B68D9062DED028B40F1A6806F4C636902
:109780000BB12046984762684FF47A73534305D073
:109790006B4A0A2B1268B8BF0A23D3600EF0CEFCC6
:1097A000A369B0EE408A002B00F09B806348984785
:1097B000C21C00F089800028C0F28980614B2062C1
:1097C0001B68A362604B5B78002B38D05F49D1F8EF
:1097D000A43001EB83020133052BC2F8A800C1F8C5
:1097E000A43027D10023C1F8A430012381F8BC3074
:1097F000D1F8B800D1E92A32D1E92C7C9A42A2BF33
:1098000011461A460B468445DEBF014660468C462B
:109810009042B8BF10466345A8BF63469F42A2BFAF
:109820003A461F4613469842A8BF1846B842B8BFEA
:10983000384603E091F8BC30002BD9D12062D4ED3A
:10984000077AB4EEE78AF1EE10FA4DD4236A002BC2
:109850004ADB07EE903AF8EEE77A27EE888AFDEECB
:10986000C87A17EE903A636207EE903A374CB8EE3A
